:020000040000FA
:10000000084804000100000010EF000010EF00009D
:1000100010EF000010EF000010EF000010EF0000E4
:1000200010EF000010EF000010EF000010EF0000D4
:1000300010EF00006674000010EF000010EF0000E9
:1000400010EF00008C740000B274000010EF00008C
:1000500010EF000010EF000010EF00007AC9000060
:1000600010EF000010EF00007ACC000012C1000079
:1000700010EF0000CAE500007EDE000010EF000077
:1000800010EF00001CE6000010EF000010EF000071
:1000900010EF0000E67400000C750000BEDE0000EA
:1000A00010EF000010EF000010EF000010EF000054
:1000B00010EF000010EF000010EF000010EF000044
:1000C00010EF000010EF000010EF000010EF000034
:1000D00010EF000010EF000042A9000010EF000038
:1000E00010EF000010EF000010EF000000CD000046
:1000F000A8C1000010EF000010EF000096B700004C
:100100001269000010EF000010EF000010EF000077
:1001100010EF000010EF000010EF000010EF0000E3
:1001200010EF000010EF000010EF000010EF0000D3
:1001300010EF000010EF000010EF000010EF0000C3
:1001400010EF000010EF000082B7000010EF000079
:1001500010EF000010EF000010EF000010EF0000A3
:1001600010EF000010EF000010EF000010EF000093
:1001700010EF000010EF000082CD00003EC2000032
:1001800080E9000010EF000010EF000010EF000009
:1001900010EF000010EF000010EF000052E0000030
:1001A00010EF000010EF000010EF000010EF000053
:1001B00010EF000010EF000010EF000010EF000043
:1001C00010EF000010EF000010EF000010EF000033
:1001D00010EF000010EF000010EF000010EF000023
:1001E00010EF000010EF000010EF000010EF000013
:1001F00010EF000010EF000010EF000010EF000003
:10020000000000000000000010EF000010EF0000F0
:1002100010EF000010EF000010EF000010EF0000E2
:1002200010EF000010EF000010EF000010EF0000D2
:1002300010EF00006674000010EF000010EF0000E7
:1002400010EF00008C740000B274000010EF00008A
:1002500010EF000010EF000010EF00007AC900005E
:1002600010EF000010EF00007ACC000012C1000077
:1002700010EF0000CAE500007EDE000010EF000075
:1002800010EF00001CE6000010EF000010EF00006F
:1002900010EF0000E67400000C750000BEDE0000E8
:1002A00010EF000010EF000010EF000010EF000052
:1002B00010EF000010EF000010EF000010EF000042
:1002C00010EF000010EF000010EF000010EF000032
:1002D00010EF000010EF000042A9000010EF000036
:1002E00010EF000010EF000010EF000000CD000044
:1002F000A8C1000010EF000010EF000096B700004A
:100300001269000010EF000010EF000010EF000075
:1003100010EF000010EF000010EF000010EF0000E1
:1003200010EF000010EF000010EF000010EF0000D1
:1003300010EF000010EF000010EF000010EF0000C1
:1003400010EF000010EF000082B7000010EF000077
:1003500010EF000010EF000010EF000010EF0000A1
:1003600010EF000010EF000010EF000010EF000091
:1003700010EF000010EF000082CD00003EC2000030
:100380009E48010010EF000010EF000010EF000089
:1003900010EF000010EF000010EF000052E000002E
:1003A00010EF000010EF000010EF000010EF000051
:1003B00010EF000010EF000010EF000010EF000041
:1003C00010EF000010EF000010EF000010EF000031
:1003D00010EF000010EF000010EF000010EF000021
:1003E00010EF000010EF000010EF000010EF000011
:1003F00010EF000010EF000010EF000010EF000001
:1004000000480400010000006F422300607D2400CA
:1004100000018800000000000B00070060252B0091
:100420000100200010000700000020000000E00094
:10043000020032000000020000000000CEB70200FF
:10044000000000000000FE004440A90040772100A9
:100450000000E0000300320000002000A00188003E
:100460004440A80000000600F8FF2000591C2100AD
:1004700091018800800078000000EB001A0037002E
:100480008180E80032A0B4009101BA00E28040000F
:1004900032A0B4009102BA00E280400032A0B40061
:1004A0000002EB00472BDE00F507B200602CE100F4
:1004B00009003A00330007000700E00002003200A4
:1004C0000059EB00010037000201E8008301E90058
:1004D000F8FF3E00040037006128E100010032000F
:1004E0000082EB00040007001101BA000200E000E6
:1004F000E3FF3A0000000600220007000700E000CA
:10050000020032003159BA00020037008100E800D1
:100510000201E8008301E90017003200190007001A
:100520000700E000020032002159BA000200370043
:100530008100E9000201E8008301E9000D003200BA
:100540000400E00003003A00E280400032A0B40062
:10055000E9FF37000B0007000700E000020032004F
:1005600011D9BA00010037000201E8008301E90057
:10057000F5FF3A008100E800E180400032A0B400BD
:10058000000006000810E600020037000910E6002F
:10059000020037008083EB00000006008003EB00C0
:1005A0000000060091018800800078000000EB0048
:1005B00015003700E280400032A0B4009101BA007B
:1005C000E280400032A0B4009102BA00E280400014
:1005D00032A0B4000002EB00472BDE00F507B200AA
:1005E000602CE10004003A000059EB008301E900AF
:1005F000FDFF3E00040037006128E10001003200E9
:100600000082EB00040007001101BA000200E000C4
:10061000E8FF3A00000006003159BA008301E90002
:100620000C0032002159BA008301E90008003200B1
:100630000400E00003003A00E280400032A0B40071
:10064000F5FF370011D9BA008301E900FAFF3A003B
:100650008100E800E180400032A0B4000000060004
:1006600002EF040000000000EED2040000000000D1
:10067000BC8C040000000000D28D040000000000CB
:10068000BAC8040000000000D4B604000000000056
:1006900004B60400000000001EB6040000000000C4
:1006A00070B6040000000000A8E404000000000090
:1006B000B0DC0400000000003CE00400000000008A
:1006C000E8BC040000000000C8AA0400000000000C
:1006D0009CAE04000000000098AE04000000000082
:1006E0003EAF0400000000000CAF0400000000005A
:1006F000A0AE040000000000167704000000000017
:100700004877040000000000787704000000000033
:10071000BA77040000000000FE770400000000002B
:10072000427804000000000084780400000000000B
:10073000F078040000000000387904000000000098
:100740008079040000000000DC7904000000000053
:10075000527A040000000000CE7A0400000000007D
:10076000227B0400000000003E7B0400000000002B
:10077000D07B0400000000001C7C0400000000008E
:10078000587C040000000000947C0400000000007D
:10079000487D040000000000707E0400000000009E
:1007A000229B040000000000969B04000000000053
:1007B000569B040000000000D69B040000000000CF
:1007C000169C0400000000005C9C04000000000077
:1007D000E89C0400000000004C9D040000000000A4
:1007E0001A9D0400000000000C9F0400000000009F
:1007F0007E9D040000000000DC9D0400000000005D
:10080000689E0400000000009E9E0400000000009E
:10081000BA9E040000000000D69E04000000000004
:100820003E9F040000000000769F040000000000CE
:10083000929F04000000000000A0040000000000DF
:1008400032A004000000000064A0040000000000CA
:100850004EB70400000000006022B800060220002D
:100860000000D0008180D2000482D2008582D200B4
:100870000000A0000202520083825A0003003100EF
:100880000202420083824A000000A1000603E90040
:10089000F3FF3A0000000600020AB900001BB9008D
:1008A0000200B80081004200810043000000060001
:1008B000889FBE008A9FBE008C1F78000006EB0058
:1008C000E00F5000E08F5800E00F5900E08F590012
:1008D00007003D006044B8006055B80000005400B7
:1008E00081805C0002015D0083815D001C002000AE
:1008F000E00F5200E08F5A00E00F5B00E08F5B00DA
:1009000007003D006044B8006055B8000402540080
:1009100085825C0006035D0087835D000C00A200F9
:100920000B010700E00F5600060032006022B800FD
:100930006033B8000000520081805A0002015B0061
:1009400083815B004F0678004F05BE004F04BE0058
:1009500000000600889FBE008A9FBE003004BE00D3
:100960002005BE000404440085844C0006054D00AB
:1009700087854D000898BE000A90BE0095000700CC
:1009800002003100680040001008E8004F05BE007A
:100990004F04BE0000000600889FBE008A9FBE0074
:1009A0008C1F7800000678003C04BE002C05BE00B9
:1009B0000400540085805C0006015D0087815D00B5
:1009C000009EBE00029EBE001000200081000700B5
:1009D000010039000000EB001C0E10004F067800EB
:1009E0004F05BE004F04BE00000006001200FA00D2
:1009F000889FBE008A9FBE008C9FBE000205BE007D
:100A00000004BE00E4B79F00F5B79F0086BF9F00BB
:100A100097BF9F000000EB00D0B79F00C0B79F00BA
:100A2000B0B79F00A0B79F0090B79F000006780066
:100A3000FD032000DFB197004FB097000381410014
:100A4000BFB09700E08F510004003D006600070032
:100A50007E805700BFFF07000300370062000700D9
:100A60007E805700CCFF0700DFB09700E08F50007A
:100A70000700350014002000050020006033B80096
:100A800008047200898472000A0573008B85730064
:100A90000C06E8008D0F5600E6FF3400E08F500092
:100AA00006003D006FB29700FFB297000FBB9700A2
:100AB0009FBB97007E805700A6FF07005FA89700A6
:100AC000E00F500004003A001FB49700AFB4970045
:100AD0003FB59700CFB597000800BE000A01BE00E1
:100AE0004F06BE004F05BE004F04BE000080FA0056
:100AF00000000600881F780018002000881F78007A
:100B0000BAFF07008F87E9004F0478000000060055
:100B1000801FEB00B5FF07008F87E900000006008B
:100B2000889FBE008A9FBE008C1F78004E00070081
:100B300005003D005100070009003D005B00070073
:100B40000006EB00060037005D00070004003D00D2
:100B50006044B8006055B800540007001C00200035
:100B6000E4FF0700E00F5600010032005A000700C2
:100B70004F0678004F05BE004F04BE00000006007F
:100B8000889FBE008A9FBE008C1F78003600070039
:100B900003003D003900070006003D000400370057
:100BA0004700070003003D006044B8006055B800EE
:100BB0003E000700D6FF0700E00F5600010032009C
:100BC000450007004F0678004F05BE004F04BE00E9
:100BD000000006000440E10005C8E10006D0E10085
:100BE00007D8E10000000600CF01DE00028171009D
:100BF000B2B79F004F09DE00000040000000710006
:100C0000A0B79F000FB097004F01DE008180400029
:100C10008100710091B79F007FAA9700CF20DE006E
:100C2000000040000080700080B79F000800BE00F8
:100C30000A01BE004F18DE000402420000027200EA
:100C4000F4AF9F000804440089844C000A054D005D
:100C50008B854D004FB29700DFB297006FB39700BE
:100C6000FFB3970000000600E00F5000E08F58002F
:100C7000E00F5900E08F5900000006006044B80002
:100C80006055B8000000540081805C0002015D00E6
:100C900083815D001C0020000820E10009A8E1001C
:100CA0000AB0E1000BB8E1000000060004025400A5
:100CB00085825C0006035D0087835D0000000600FE
:100CC0000006EB00E00F5200E08F5A00E00F5B00DF
:100CD000E08F5B00000006006022B8006033B800BF
:100CE0000000520081805A0002015B0083815B009A
:100CF00000000600839F68000100E00002003D0044
:100D000060001000E08018000300E00002003D00D9
:100D100060011100E0811900CFFE07004F00E000E4
:100D200002003B0060001000E08018000000060098
:100D300080017800110009008280D8008001FD0048
:100D4000110009004288D8008300780000000600E6
:100D5000889FBE008A9FBE008C9FBE000404B8001E
:100D60000506B8008904460060854E000606B800F6
:100D70000A054600E0854E000706B8008B054600D0
:100D8000040EB800890446000A854E00E0854D0037
:100D9000050EB8000A0546008B854E00060EB80009
:100DA0008B0546000416B8000A0546008B854E00E8
:100DB0000516B8008B054600041EB8008B054600DA
:100DC0000800BE000A01BE004F06BE004F05BE006F
:100DD0004F04BE00000006008001780002003700CA
:100DE000B1597800040178000202E900E00F5100D7
:100DF000FBFF3A0000000600800178000200370087
:100E000081597800040178000202E900E00F5100E6
:100E1000FBFF3A0000000600800078000041EB0074
:100E2000B14F1100FDFF3A000080EA000080400051
:100E300000000600E68747008E1F7800D0BF9F00A5
:100E400066875700012F78000E003700DFB9970042
:100E5000134178006FB8970090407800814F51009F
:100E6000040032000280FB008180FB000100500082
:100E7000080037008301E800D3BF9F00000FE8009F
:100E8000040178000202E900E00F5100EFFF3A0090
:100E9000020078004F0778006F00B10000000600E4
:100EA0006D610000746800002E6300006F70000028
:100EB00079000000636F0000706900006573000036
:100EC0002073000072630000207400006F20000097
:100ED0006465000073740000206500006C6500000C
:100EE0006D6500006E740000206200007920000033
:100EF000656C0000656D0000656E00007400000008
:100F000064650000737400000073000072630000E9
:100F100000000000508700005A870000FFFF00001B
:100F200080870000FFFF00008587000000000000B0
:100F3000000000006D610000746800002E66000073
:100F4000696C00006C000000666900006C6C0000B9
:100F500073200000646500007374000020770000B7
:100F60006974000068200000636F00006E73000069
:100F7000746100006E74000020760000616C000057
:100F80007565000000760000616C0000756500006A
:100F9000000000009A870000A4870000FFFF000007
:100FA0008087000001000000C387000000000000EF
:100FB000000000006D610000746800002E610000F8
:100FC0006464000073630000616C000061720000E3
:100FD0000061000064640000207300006361000091
:100FE0006C61000072200000746F0000206500003A
:100FF0006163000068200000656C0000656D000002
:10100000656E0000742000006F6600002073000011
:1010100072630000206100006E6400002073000015
:10102000746F00007265000020720000657300009C
:10103000756C000074200000746F000020640000D4
:10104000657300007400000073630000616C0000B1
:101050006172000000000000DA870000E9870000EC
:10106000FFFF000080870000FFFF00008587000071
:1010700001000000248800000000000000000000C3
:101080006D610000746800002E610000646400005F
:1010900000610000646400007320000073720000AF
:1010A00063310000206100006E64000020730000C6
:1010B0007263000032200000746F000020640000A2
:1010C00065730000742C0000206500006C65000052
:1010D0006D6500006E740000206200007920000041
:1010E000656C0000656D0000656E00007400000016
:1010F000737200006331000000730000726300002F
:10110000320000004088000049880000FFFF000016
:1011100080870000FFFF000078880000FFFF0000CC
:101120007D88000000000000000000006D610000EC
:10113000746800002E7300007562000000730000E8
:101140007562000073740000726100006374000037
:1011500073200000737200006332000020660000FC
:10116000726F00006D200000737200006331000098
:10117000207400006F20000064650000737400009C
:101180002C200000656C0000656D0000656E00009D
:101190007420000062790000206500006C6500008A
:1011A0006D6500006E74000000000000968800006D
:1011B0009F880000FFFF000080870000FFFF000005
:1011C00078880000FFFF00007D880000000000001C
:1011D000000000006D610000746800002E6D0000CA
:1011E000756C0000006D0000756C000074690000F3
:1011F000706C0000696500007320000073720000CD
:1012000063310000206100006E6400002073000064
:101210007263000032200000746F00002064000040
:1012200065730000742C0000206500006C650000F0
:101230006D6500006E7400002062000079200000DF
:10124000656C0000656D0000656E000074000000B4
:10125000EA880000F3880000FFFF0000808700009C
:10126000FFFF000078880000FFFF00007D8800007D
:1012700000000000000000006D61000074680000C4
:101280002E640000697600000064000069760000AA
:101290006964000065730000207300007263000041
:1012A00031200000627900002073000072630000AA
:1012B00032200000746F000020640000657300009D
:1012C000742C0000206500006C6500006D65000056
:1012D0006E7400002062000079200000656C000040
:1012E000656D0000656E0000740000003C89000020
:1012F00045890000FFFF000080870000FFFF00001D
:1013000078880000FFFF00007D88000000000000DA
:10131000000000006D610000746800002E6D000088
:10132000696E0000007700007269000074650000BB
:101330007320000074680000652000006D690000E3
:101340006E6900006D7500006D2000006F66000082
:10135000207300007263000031200000616E000005
:1013600064200000737200006332000020740000EB
:101370006F20000064650000737400002C200000E2
:10138000656C0000656D0000656E00007420000053
:1013900062790000206500006C6500006D6500004A
:1013A0006E740000000000008A890000938900002C
:1013B000FFFF000080870000FFFF0000788800002A
:1013C000FFFF00007D88000000000000000000001A
:1013D0006D610000746800002E6D000061780000EF
:1013E000007700007269000074650000732000003F
:1013F00074680000652000006D61000078690000DD
:101400006D7500006D2000006F6600002073000005
:101410007263000031200000616E00006420000053
:101420007372000063320000207400006F2000001F
:1014300064650000737400002C200000656C0000DF
:10144000656D0000656E0000742000006279000088
:10145000206500006C6500006D6500006E74000082
:1014600000000000E8890000F1890000FFFF000093
:1014700080870000FFFF000078880000FFFF000069
:101480007D88000000000000000000006D61000089
:10149000746800002E6300006C6100006D70000035
:1014A000006300006C6100006D700000207300009C
:1014B00072630000207400006F2000006C6F000059
:1014C000772F000068690000676800002062000054
:1014D0006F7500006E64000073200000696E0000EC
:1014E000746F00002064000065730000742C00001D
:1014F000206500006C6500006D6500006E740000E2
:101500002062000079200000656C0000656D00001D
:10151000656E0000740000006C6F00007700000032
:10152000686900006768000000000000468A00004B
:10153000518A0000FFFF000080870000FFFF0000CD
:1015400085870000FFFF00008C8A0000FFFF00007D
:10155000908A000000000000000000006D610000A3
:10156000746800002E6400006F74000000770000B3
:101570007269000074650000732000007468000048
:1015800065200000646F000074200000707200008D
:101590006F64000075630000742000006F66000037
:1015A000207300007263000031200000616E0000B3
:1015B0006420000073720000633200002074000099
:1015C0006F20000064650000737400002C20000090
:1015D0006166000074650000722000006120000058
:1015E0007368000069660000740000007368000002
:1015F0006966000074000000AE8A0000B78A00002F
:101600000100000080870000FFFF000078880000D4
:10161000FFFF00007D88000001000000F68A000046
:1016200000000000000000006D6100007468000010
:101630002E730000746100007400000070650000EB
:10164000726600006F7200006D730000207300006E
:101650007461000074690000737400006963000025
:10166000732000006F6E00002073000072630000A2
:10167000006D0000696E0000006D000061780000E0
:10168000006D0000656100006E000000148B00001A
:101690001E8B0000FFFF0000858700000100000096
:1016A000398B0000010000003D8B000001000000AC
:1016B000418B000000000000000000006D61000090
:1016C000746800002E61000072670000626F000005
:1016D000756E000064730000006700006574000010
:1016E0002074000068650000206900006E6400003E
:1016F000696300006573000020280000617200002B
:10170000676D0000696E00002C200000617200000F
:10171000676D000061780000292000006F660000FE
:101720002074000068650000206C0000696D0000F6
:101730006974000020760000616C0000756500008F
:10174000732000006F6600002073000072630000C9
:1017500000610000726700006D6900006E0000000B
:1017600061720000676D00006178000000000000F9
:101770005E8B00006D8B0000FFFF0000858700007E
:1017800001000000A98B000001000000B08B0000E8
:1017900000000000000000006D610000746800009F
:1017A0002E7300006F72000074000000736F000061
:1017B0007274000020610000727200006179000004
:1017C000206900006E200000706C00006163000062
:1017D0006500000061720000726100007900000085
:1017E000CC8B0000D68B0000FFFF0000EA8B0000CE
:1017F00000000000000000006D610000746800003F
:101800002E6D0000756C0000646900007600000019
:1018100070650000726600006F7200006D7300005A
:101820002064000065730000742000003D2000006B
:10183000286100002A620000292F000063200000B8
:10184000696E000020330000322000006269000051
:1018500074730000206500006C6500006D65000079
:101860006E7400002062000079200000656C0000AA
:10187000656D0000656E00007400000061000000EE
:101880006200000063000000FC8B0000088C000078
:10189000FFFF000080870000FFFF00003E8C00007B
:1018A000FFFF0000408C0000FFFF0000428C0000A2
:1018B00000000000000000006D610000746800007E
:1018C0002E610000746100006E32000000700000A4
:1018D00065720000666F0000726D000073200000EA
:1018E0006465000073740000203D0000206100006A
:1018F000746100006E320000287900002C7800002E
:1019000029200000656C0000656D0000656E000018
:101910007420000062790000206500006C65000002
:101920006D6500006E740000007900000078000012
:10193000000000005C8C0000678C0000FFFF0000CE
:1019400080870000FFFF0000958C0000FFFF000073
:10195000978C000000000000000000006D61000096
:10196000746800002E730000696E000000700000B3
:1019700065720000666F0000726D00007320000049
:101980006465000073740000203D000020730000B7
:10199000696E00002878000029200000656C0000B6
:1019A000656D0000656E0000742000006279000023
:1019B000206500006C6500006D6500006E7400001D
:1019C00000000000AE8C0000B78C0000FFFF00009C
:1019D00080870000FFFF0000978C000000000000DF
:1019E000000000006D610000746800002E630000BC
:1019F0006F7300000070000065720000666F0000E9
:101A0000726D0000732000006465000073740000B4
:101A1000203D0000206300006F7300002878000064
:101A200029200000656C0000656D0000656E0000F7
:101A30007420000062790000206500006C650000E1
:101A40006D6500006E74000000000000F28C000064
:101A5000FB8C0000FFFF000080870000FFFF0000FC
:101A6000978C000000000000000000006D61000085
:101A7000746800002E7200006F74000032000000D5
:101A8000726F000074610000746500007320000034
:101A9000762000006F660000206100006E67000085
:101AA0006C65000020610000207400006F200000C1
:101AB0006465000073740000007600000000000000
:101AC000368D0000408D000002000000808700007D
:101AD000020000005D8D0000010000003E8C00004F
:101AE00000000000000000006D610000746800004C
:101AF0002E73000071720000740000007065000019
:101B0000726600006F7200006D73000020640000B8
:101B100065730000742000003D2000007371000018
:101B2000727400002878000029200000656C000015
:101B3000656D0000656E0000742000006279000091
:101B4000206500006C6500006D6500006E7400008B
:101B500000000000748D00007E8D0000FFFF00007B
:101B600080870000FFFF0000978C0000000000004D
:101B7000000000006D610000746800002E6E00001F
:101B80007A73000065710000007700007269000040
:101B900074650000207400006F2000006465000080
:101BA000737400002074000068650000206D000060
:101BB00069640000646C000065200000696E00002C
:101BC00064650000782000006F660000207400004B
:101BD00068650000206C000061720000676500000D
:101BE00073740000207300006571000075650000CB
:101BF0006E630000652000006F660000206E00002C
:101C00006F6E00002D7A0000657200006F200000EA
:101C1000656C0000656D0000656E00007473000067
:101C200020660000726F00006D20000073720000DB
:101C3000632C0000202D00003120000069660000A8
:101C4000206E00006F740000206600006F750000B9
:101C50006E640000206F00007220000069660000C2
:101C6000207300006D6100006C6C00006572000064
:101C700020740000686100006E2000006D690000A3
:101C80006E4C0000656E0000677400006800000084
:101C90006D6900006E4C0000656E00006774000006
:101CA00068000000BA8D0000C58D00000100000032
:101CB00080870000FFFF0000858700000100000012
:101CC000488E000000000000000000006D61000070
:101CD000746800002E720000616E00006400000055
:101CE000666900006C6C00002061000072720000E8
:101CF000617900002077000069740000682000000E
:101D0000726100006E6400006F6D000020760000BC
:101D1000616C00007565000073000000668E0000B5
:101D2000708E0000FFFF00008087000000000000B0
:101D300000000000000000009301000024030000E8
:101D4000B704000048060000DA0700006B09000035
:101D5000FC0A00008C0C00001C0E0000AB0F000001
:101D60003B110000C812000056140000E3150000EB
:101D70006E170000F9180000831A00000C1C000008
:101D8000941D00001A1F0000A02000002422000063
:101D9000A723000029250000A8260000272800000E
:101DA000A4290000202B0000992C0000122E000016
:101DB000872F0000FC3000006F320000DF3300008E
:101DC0004E350000BA360000253800008D3900007D
:101DD000F33A0000573C0000B93D0000173F0000F7
:101DE00074400000CE410000264300007B44000008
:101DF000CD4500001D4700006A480000B4490000BE
:101E0000FC4A0000404C0000824D0000C04E000023
:101E1000FC4F000034510000695200009B53000049
:101E2000CA540000F65500001E5700004358000039
:101E300064590000835A00009D5B0000B45C000000
:101E4000C85D0000D75E0000E45F0000EC600000A9
:101E5000F1610000F2620000EF630000E96400003D
:101E6000DE650000D0660000BD670000A7680000C6
:101E70008C6900006E6A00004B6B0000246C00004F
:101E8000F96C0000CA6D0000976E00005F6F0000E3
:101E900023700000E37000009E7100005572000086
:101EA00008730000B6730000607400000575000040
:101EB000A575000042760000D97600006C7700001E
:101EC000FB77000084780000097900008A7900001F
:101ED000067A00007D7A0000EF7A00005D7B00004A
:101EE000C67B00002A7C0000897C0000E47C0000A6
:101EF000397D00008A7D0000D77D00001D7E000036
:101F0000607E00009D7E0000D67E0000097F0000FC
:101F1000397F0000627F0000877F0000A77F0000FC
:101F2000C27F0000D87F0000EA7F0000F67F00003B
:101F3000FE7F0000FF7F00008C020000DF02000037
:101F40003003000080030000D103000022040000E1
:101F500073040000C204000014050000B305000073
:101F600054060000F10600008F0700002D08000055
:101F7000CA08000063090000FC090000340B0000DF
:101F80005C0C0000820D0000A40E0000BD0F0000DC
:101F9000D3100000E2110000E7120000EF1400006F
:101FA000CC16000092180000401A0000D61B00005A
:101FB000531D0000B51E00000B2000007922000018
:101FC0008D2400006F2600001428000090290000D6
:101FD000E02A0000112C0000252D0000052F000034
:101FE00089300000D3310000EC320000DD33000006
:101FF000AE340000673500000D36000020370000C9
:10200000FB370000B23800004A390000CC3900002C
:102010003B3A00009B3A0000F33A0000833B00008B
:10202000F43B0000513C00009F3C0000E13C0000FC
:102030001A3D00004B3D0000783D0000C03D00000F
:10204000F93D0000283E00004F3E0000703E0000B9
:102050008D3E0000A53E0000BC3E0000E03E0000BA
:10206000FD3E0000143F0000283F0000383F000004
:10207000473F0000533F00005E3F0000703F0000FC
:102080007F3F00008A3F0000943F00009C3F00001B
:10209000A43F0000AA3F0000AF3F0000B83F00008F
:1020A000C03F0000C53F0000CB3F0000CE3F000016
:1020B000D23F0000D53F0000D83F0000DC3F0000C9
:1020C000E03F0000E33F0000E53F0000E83F000084
:1020D000E93F0000EB3F0000EC3F0000EE3F000056
:1020E000F13F0000F13F0000F33F0000F43F00002B
:1020F000F53F0000F53F0000F73F0000F73F00000C
:10210000F93F0000F83F0000FA3F0000FA3F0000EE
:10211000FA3F0000FB3F0000FB3F0000FC3F0000D7
:10212000FC3F0000FC3F0000FE3F0000FD3F0000C0
:10213000FD3F0000FD3F0000FE3F0000FE3F0000AD
:10214000FE3F0000FE3F0000FE3F0000FE3F00009B
:1021500000400000FF3F0000FF3F0000FF3F000085
:10216000FF3F0000FF3F0000FF3F0000FF3F000077
:10217000FF3F0000FF3F0000FF3F0000FF3F000067
:10218000004000000040000000400000004000004F
:10219000004000000040000000400000004000003F
:1021A000004000000040000000400000004000002F
:1021B00000400000004000000040000041640000BA
:1021C0006472000065730000732000006F750000EA
:1021D000742000006F66000020730000657400002A
:1021E000746900006E67000073000000536C00000B
:1021F00065650000702000006D6F000064650000E0
:10220000206E00006F7400002073000075700000E5
:10221000706F0000727400006564000000450000EB
:10222000727200006F7200003A2000006D690000B9
:102230006E2000003D3D0000203000007846000088
:102240004646000046460000464600004620000084
:102250002100000045720000726F0000723A000019
:10226000205500006E610000626C000065200000D7
:10227000746F0000206600006C610000736800004D
:102280002062000079740000656300006F64000044
:1022900065200000283100002920000021000000F6
:1022A00045720000726F0000723A00002055000075
:1022B0006E610000626C000065200000746F000019
:1022C000206600006C61000073680000206200005E
:1022D00079740000656300006F64000065200000F1
:1022E0002832000029200000210000004572000073
:1022F000726F0000723A0000205500006E6100000D
:10230000626C000065200000746F00002066000011
:102310006C610000736800002062000079740000A6
:10232000656300006F640000652000002833000032
:102330002920000021000000466C000061730000AD
:10234000686900006E670000204F00004B0000002D
:1023500074680000796D0000696F00002D4900006D
:10236000490000005F69000064000000657600001D
:10237000656E0000742E0000736F0000757200001F
:102380006365000000650000766500006E74000063
:102390002E61000072670000730000005F6600009D
:1023A0007776000065720000736900006F6E0000B0
:1023B000005F0000707200006F6400007563000031
:1023C000744900006400000062750000747400002D
:1023D0006F6E0000732E00005F72000061770000D6
:1023E0000062000075740000746F00006E2E000023
:1023F00062610000636B000077610000726400009E
:102400000062000075740000746F00006E2E000002
:102410006C650000667400000062000075740000C6
:10242000746F00006E2E0000636500006E74000083
:10243000657200000062000075740000746F000097
:102440006E2E0000666F000072770000617200005F
:102450006400000062750000747400006F6E00007C
:102460002E720000696700006874000000620000BE
:1024700075740000746F00006E7300002E5F000022
:102480006D650000616E0000006200007574000060
:10249000746F00006E7300002E5F00006E6F00000E
:1024A0006973000065000000707200006F78000022
:1024B0002E6800006F720000697A00006F6E0000E5
:1024C000746100006C000000707200006F78000002
:1024D0002E6300006F6D00006D2E0000727800000A
:1024E0002E5F000070610000796C00006F610000D9
:1024F0006473000000700000726F0000782E00000E
:10250000636F00006D6D00002E720000782E0000D9
:102510005F6900006E740000656E00007369000062
:10252000746900006573000000700000726F0000A5
:10253000782E0000636F00006D6D00002E720000A9
:1025400078000000707200006F7800002E630000B9
:102550006F6D00006D2E00007478000000700000A8
:10256000726F0000782E0000677200006F75000027
:102570006E6400002E6100006D6200006961000061
:102580006E74000000700000726F0000782E000072
:10259000677200006F7500006E6400002E7200000C
:1025A000656600006C6500006374000065640000EF
:1025B00000700000726F0000782E0000677200004B
:1025C0006F7500006E6400002E640000656C0000F2
:1025D00074610000006D00006F7400006F720000F5
:1025E0002E6C000065660000742E0000746100000F
:1025F0007267000065740000006D00006F740000D9
:102600006F7200002E72000069670000687400009D
:102610002E74000061720000676500007400000005
:102620005F76000062610000740000005F690000D6
:102630006D6F0000740000006D6F0000746F00008B
:10264000722E00006C650000667400002E7300009E
:102650007065000065640000006D00006F7400008C
:102660006F7200002E72000069670000687400003D
:102670002E7300007065000065640000006D0000AE
:102680006F7400006F7200002E6C00006566000021
:10269000742E0000707700006D0000006D6F000068
:1026A000746F0000722E00007269000067680000FD
:1026B000742E0000707700006D0000006163000060
:1026C00063000000746500006D700000657200001A
:1026D0006174000075720000650000007263000004
:1026E000352E000061640000647200006573000014
:1026F0007300000072630000352E0000636F00005D
:102700006D6D0000616E0000640000006D690000E6
:10271000632E0000696E0000746500006E73000097
:1027200069740000790000006D690000632E0000EC
:102730007468000072650000736800006F6C000030
:10274000640000006D690000632E00005F6D0000F2
:10275000656100006E000000746900006D65000096
:10276000722E000070650000726900006F64000046
:1027700000610000636300002E5F000074610000D0
:1027800070000000A891000001000000B29100005C
:1027900001000000B691000020000000C39100007D
:1027A00002000000CE91000001000000D99100005D
:1027B00005000000E491000001000000F19100001C
:1027C0000100000001920000010000000D920000D5
:1027D000010000001B920000010000002A9200008E
:1027E000050000003792000005000000459200003F
:1027F00007000000549200000700000064920000EF
:10280000070000007B92000001000000959200008C
:1028100001000000A292000002000000AF92000040
:1028200002000000C392000002000000D9920000E4
:1028300001000000EB92000001000000FD9200008A
:102840000200000010930000020000001693000038
:10285000010000001C930000010000002D93000007
:10286000010000003F930000010000004E930000B3
:10287000030000005E93000001000000629300006E
:10288000010000006E930000010000007A93000038
:1028900001000000869300000100000094930000F6
:1028A00001000000A293000002000000AC930000B1
:1028B00001000000B99300000000000000000000CB
:1028C000DE000000AD000000CA000000FE000000B5
:1028D000BE000000EF000000040000000200000045
:1028E00098AE00003EAF00000CAF0000A0AE0000AC
:1028F000167700004877000078770000BA7700006C
:10290000FE7700004278000084780000F078000034
:102910003879000080790000DC790000527A0000EC
:10292000CE7A0000227B00003E7B0000D07B0000BE
:102930001C7C0000587C0000947C0000487D000056
:10294000707E0000229B0000969B0000569B0000BA
:10295000D69B0000169C00005C9C0000E89C0000D8
:102960004C9D00001A9D00000C9F00007E9D000001
:10297000DC9D0000689E00009E9E0000BA9E000044
:10298000D69E00003E9F0000769F0000929F0000B0
:1029900000A0000032A0000064A000004EB70000BC
:1029A00042610000636B0000776100007264000008
:1029B0002062000075740000746F00006E2000003B
:1029C00073740000617400007573000020630000E0
:1029D000686100006E67000065640000004C000044
:1029E00065660000742000006275000074740000C9
:1029F0006F6E0000207300007461000074750000A9
:102A00007320000063680000616E000067650000CD
:102A100064000000436500006E74000065720000F1
:102A20002062000075740000746F00006E200000CA
:102A3000737400006174000075730000206300006F
:102A4000686100006E6700006564000000460000D9
:102A50006F72000077610000726400002062000065
:102A600075740000746F00006E2000007374000025
:102A7000617400007573000020630000686100004D
:102A80006E67000065640000005200006967000086
:102A9000687400002062000075740000746F00000C
:102AA0006E200000737400006174000075730000F4
:102AB00020630000686100006E670000656400002C
:102AC0000062000075740000746F00006E730000F7
:102AD0000042000075740000746F00006E73000007
:102AE00020760000616C0000756500007320000016
:102AF00075700000646100007465000064000000EF
:102B0000707200006F78000000500000726F0000CB
:102B1000786900006D69000074790000207600007B
:102B2000616C000075650000732000007570000086
:102B300064610000746500006400000070720000B1
:102B40006F7800002E6300006F6D00006D000000C4
:102B500044610000746100002072000065630000A1
:102B60006569000076650000642000006F6E00005B
:102B7000207400006865000020700000726F000083
:102B8000786900006D69000074790000206300001E
:102B90006F6D00006D7500006E69000063610000DC
:102BA000746900006F6E0000007400006170000026
:102BB00000410000207400006170000020690000E6
:102BC00073200000646500007465000063740000F9
:102BD000656400000041000063630000656C000054
:102BE000657200006F6D0000657400006572000082
:102BF00020760000616C0000756500007320000005
:102C000075700000646100007465000064000000DD
:102C10006D690000630000004669000072650000F5
:102C20006420000077680000656E0000206D0000E1
:102C300069630000726F0000706800006F6E000032
:102C400065200000696E0000746500006E7300006E
:102C500069740000792000006973000020610000A1
:102C6000626F00007665000020740000687200004A
:102C700065730000686F00006C6400000073000062
:102C80006F7500006E6400002E660000696E000023
:102C90006973000068650000640000004669000078
:102CA000726500006420000077680000656E000017
:102CB0002074000068650000207000006C61000056
:102CC00079620000616300006B2000006F66000005
:102CD0002061000020750000736500007220000074
:102CE000696E00006974000069610000746500008D
:102CF00064200000736F0000756E00006420000007
:102D00006973000020660000696E000069730000AE
:102D10006865000064000000546500006D700000EC
:102D2000657200006174000075720000652000008B
:102D3000766100006C750000652000007570000071
:102D400064610000746500006400000072630000AC
:102D50003500000052430000352000006D65000082
:102D60007373000061670000652000007265000059
:102D7000636500006976000065640000006D000076
:102D80006F7400006F720000004D00006F7400004F
:102D90006F72000020740000696D00006572000011
:102DA00000740000696D00006572000030000000D2
:102DB000546900006D6500007220000030000000C2
:102DC000746900006D65000072310000005400005D
:102DD000696D0000657200002031000000000000F5
:102DE000F1910000D094000001920000EF940000E7
:102DF0000D9200000A9500001B920000279500002C
:102E00002A92000045950000619500006995000038
:102E100080950000859500009E950000A895000013
:102E2000D5950000D99500005E930000EB95000059
:102E3000089600000C9600003F9600004E96000099
:102E4000629300008C960000A6960000AA960000EF
:102E5000BF960000C5960000D1960000D8960000ED
:102E6000E0960000E796000000000000000000006F
:102E70005F73000079730000746500006D2E000020
:102E800072650000626F00006F7400000052000065
:102E9000656200006F6F000074200000746800001D
:102EA000652000006D690000637200006F63000020
:102EB0006F6E0000747200006F6C00006C650000A3
:102EC000720000005F7300007973000074650000F9
:102ED0006D2E00007365000074740000696E0000C0
:102EE000677300002E72000065610000640000003E
:102EF0005265000061640000206100002073000042
:102F000065740000746900006E67000000610000D5
:102F100064640000726500007373000000760000B6
:102F2000616C000075650000005F000073790000AF
:102F300073740000656D00002E730000657400005E
:102F4000746900006E670000732E00007772000045
:102F50006974000065000000577200006974000089
:102F6000652000006120000073650000747400009B
:102F7000696E0000670000005F7300007973000055
:102F8000746500006D2E000073650000747400000D
:102F9000696E0000677300002E6600006C6100001F
:102FA000736800000057000072690000746500003B
:102FB0002074000068650000207300006574000044
:102FC000746900006E67000073200000696E0000E5
:102FD000746F0000206600006C61000073680000E0
:102FE0000000000045720000726F0000723A00009D
:102FF00020730000616D0000706C000065730000BC
:10300000206D0000757300007420000062650000F0
:10301000206900006E2000005B2D000031320000AE
:10302000382C000031320000375D000020720000B3
:10303000616E000067650000005F00006C650000C5
:10304000647300002E7300006574000000530000DC
:10305000657400002074000068650000206C0000AA
:1030600065640000006C0000656400000062000000
:103070007269000067680000746E000065730000EC
:1030800073000000736F0000756E0000642E000076
:1030900072650000636F000072640000005300005E
:1030A000746100007274000020720000656300000B
:1030B0006F720000646900006E670000206F0000FE
:1030C00066200000724E00002E770000617600003E
:1030D000004E0000007300006F7500006E64000079
:1030E0002E7000006C610000790000005374000035
:1030F0006172000074200000706C000061790000B3
:1031000062610000636B0000206F00006620000019
:10311000704E00002E770000617600000073000002
:103120006F7500006E6400002E7200006570000074
:103130006C610000790000005374000061720000AF
:1031400074200000706C0000617900006261000072
:10315000636B0000206F000066200000724E0000CC
:103160002E77000061760000007300006F7500008C
:103170006E6400002E730000797300007465000017
:103180006D000000537400006172000074200000A4
:10319000706C00006179000062610000636B0000E8
:1031A000206F000066200000737900007374000037
:1031B000656D0000207300006F7500006E640000F4
:1031C000204E0000006C000065640000732E0000BB
:1031D00063690000726300006C650000005300002A
:1031E00065740000206300006972000063750000D0
:1031F0006C61000072200000726900006E670000C0
:10320000206C000065640000730000006C3000005A
:10321000006C0000310000006C320000006C000007
:10322000330000006C340000006C0000350000002A
:103230006C360000006C0000370000006C65000078
:10324000647300002E7400006F70000000530000D3
:103250006574000020520000474200002074000006
:103260006F700000206C00006564000000720000B8
:10327000656400000067000072650000656E000074
:10328000006200006C750000650000006C650000C5
:10329000647300002E6200006F740000746F000001
:1032A0006D2E000072690000676800007400000065
:1032B00053650000742000005247000042200000C7
:1032C000626F0000746F00006D20000072690000E2
:1032D00067680000742000006C6500006400000056
:1032E0006C650000647300002E6200006F740000C3
:1032F000746F00006D2E00006C65000066740000A5
:103300000053000065740000205200004742000096
:10331000206200006F7400006F6D0000206C0000E0
:1033200065660000742000006C6500006400000009
:103330006C650000647300002E620000757400006C
:10334000746F00006E73000000530000657400008D
:103350002062000075740000746F00006E7300003E
:10336000206C000065640000730000006C650000C4
:10337000647300002E700000726F0000782E000051
:10338000680000005365000074200000686F0000B2
:10339000726900007A6F00006E740000616C0000BA
:1033A00020700000726F0000786900006D690000F5
:1033B00074790000206C0000656400007300000058
:1033C0006C650000647300002E700000726F0000D6
:1033D000782E000076000000536500007420000085
:1033E000766500007274000069630000616C000083
:1033F00020700000726F0000786900006D690000A5
:1034000074790000206C0000656400007300000007
:103410006C650000647300002E7200006300000001
:10342000536500007420000072630000206C0000EF
:1034300065640000006C000065640000732E0000ED
:10344000736F0000756E000064000000536500009B
:1034500074200000736F0000756E0000642000008F
:103460006C650000640000006C650000647300007F
:103470002E740000656D0000706500007261000030
:103480007475000072650000005300006574000050
:10349000206E000074630000206C00006564000072
:1034A000007300006F7500006E6400002E6600005F
:1034B0007265000071000000506C0000617900002E
:1034C000206600007265000071750000656E0000E6
:1034D00063790000004800007A0000006473000077
:1034E000007300006F7500006E6400002E7700000E
:1034F0006176000065000000536500007420000044
:10350000746800006520000070720000696D0000A2
:10351000617200007920000077610000766500008C
:10352000206F000066200000746800006520000025
:10353000746F00006E65000020670000656E00007B
:1035400065720000617400006F7200000077000077
:103550006176000065000000707200006F78000066
:103560002E6300006F6D00006D2E0000656E000080
:10357000616200006C650000004500006E610000A3
:10358000626C0000652000006F7200002064000083
:1035900069730000616200006C6500002074000027
:1035A0006865000020700000726F000078690000FC
:1035B0006D69000074790000206300006F6D0000E9
:1035C0006D7500006E6900006361000074690000A1
:1035D0006F6E0000007300007461000074650000ED
:1035E00000730000642E00006F700000656E000024
:1035F000004F0000706500006E2000006120000098
:10360000666900006C650000206F00006E200000FD
:10361000746800006520000053440000206300002F
:1036200061720000640000006E7500006D620000B1
:103630006572000000730000746100007475000082
:1036400073000000736400002E77000072690000B0
:103650007465000000570000726900007465000086
:10366000206400006174000061200000746F00009D
:103670002074000068650000206F00007065000085
:103680006E65000064200000666900006C65000043
:1036900000640000617400006100000077720000A7
:1036A00069740000746500006E000000736400001F
:1036B0002E72000065610000640000005265000089
:1036C000616400002064000061740000612000005B
:1036D000667200006F6D00002074000068650000D5
:1036E000206F0000706500006E650000642000001F
:1036F000666900006C6500000072000065610000F2
:1037000064000000736400002E7300006565000013
:103710006B00000053650000656B00002074000022
:1037200068650000206F0000706500006E65000095
:1037300064200000666900006C65000000700000F5
:103740006F73000069740000696F00006E00000074
:10375000733000002E7700006176000000730000D7
:10376000322E000077610000760000007333000005
:103770002E7700006176000000730000342E0000F8
:103780007761000076000000733500002E7700009E
:103790006176000000730000362E000077610000A3
:1037A00076000000733700002E770000617600007D
:1037B00000000000480D00000D0000003011000066
:1037C00007000000EC1300000700000000190000D3
:1037D00007000000781E0000070000000000000045
:1037E00000000000781E00000D000000001900001D
:1037F00007000000EC13000007000000301100007B
:1038000007000000480D0000070000000000000055
:10381000000000004C0400000700000098080000B1
:10382000070000000000000000000000E40C0000A1
:1038300007000000301100000D000000C819000052
:103840000700000000000000000000009C270000AE
:1038500002000000AB220000010000009D1C0000DF
:1038600002000000FB180000020000002D320000E2
:1038700001000000322D0000010000004628000079
:1038800002000000E826000001000000BF22000046
:1038900002000000FB18000002000000FF320000E0
:1038A00001000000C620000001000000762F00008B
:1038B000020000002C2E000001000000CE2C0000B1
:1038C00001000000FD3900000200000000000000BF
:1038D00000000000C819000005000000BE0A00003A
:1038E0000400000000000000000000003011000093
:1038F000070000007C150000070000000000000029
:103900000000000030110000070000007C150000DE
:1039100007000000C81900000700000000000000B8
:1039200000000000222A00002B2C00003A3B00007F
:103930003C3D00003E3F00005B5D00007C7F0000DE
:10394000008000009A900000418E0000418F00002E
:10395000804500004545000049490000498E0000AF
:103960008F900000929200004F9900004F55000088
:1039700055590000999A00009B9C00009D9E0000F4
:103980009F410000494F000055A50000A5A600007A
:10399000A7A80000A9AA0000ABAC000021AE00005F
:1039A000AFB00000B1B20000B3B40000B5B6000083
:1039B000B7B80000B9BA0000BBBC0000BDBE000033
:1039C000BFC00000C1C20000C3C40000C5C60000E3
:1039D000C7C80000C9CA0000CBCC0000CDCE000093
:1039E000CFD00000D1D20000D3D40000D5D6000043
:1039F000D7D80000D9DA0000DBDC0000DDDE0000F3
:103A0000DFE00000E1E20000E3E40000E5E60000A2
:103A1000E7E80000E9EA0000EBEC0000EDEE000052
:103A2000EFF00000F1F20000F3F40000F5F6000002
:103A3000F7F80000F9FA0000FBFC0000FDFE0000B2
:103A4000FF0000002E2E00002F2E00002E2F000061
:103A50006D6F00006C6F00006C6500002F69000046
:103A6000326300002F690000326300005F700000C5
:103A700072690000762E0000680000002E2E000003
:103A80002F2E00002E2F00006D6F00006C6F0000C5
:103A90006C6500002F690000326300002F6D00008C
:103AA0006173000074650000725F000070720000B6
:103AB0006F7400006F6300006F6C00002E630000E5
:103AC000000000002E2E00002F2E00002E2F0000E0
:103AD0006D6F00006C6F00006C6500002F690000C6
:103AE000326300002F690000326300005F70000045
:103AF00072690000762E0000680000002E2E000083
:103B00002F2E00002E2F00006D6F00006C6F000044
:103B10006C6500002F690000326300002F6D00000B
:103B20006173000074650000722E000063000000E5
:103B30002E2E00002F2E00002E2F00006D6F000093
:103B40006C6F00006C6500002F690000326300009C
:103B50002F690000326300005F700000726900008E
:103B6000762E0000680000002E2E00002F2E000090
:103B70002E2F00006D6F00006C6F00006C65000060
:103B80002F690000326300002F7300006C61000099
:103B9000766500002E630000000000002E2E00005D
:103BA0002F2E00002E2F00006D6F00006C6F0000A4
:103BB0006C6500002F740000696D000065720000E4
:103BC0002F740000696D0000657200002E63000014
:103BD00000000000010000000000000008000000DC
:103BE0000000000040000000000000000001000094
:103BF000000000005249000046460000000000009E
:103C0000000000005741000056450000666D0000AE
:103C100074200000100000000000000001000000FF
:103C200001000000841E000000000000841E00004F
:103C300000000000010000000800000064610000B6
:103C40007461000000000000000000005F4C0000F4
:103C50004F470000445500004D5000002E23000047
:103C600040210000005F0000544500005354000054
:103C70004D4F0000442E00002340000021000000B2
:103C8000564D0000434F0000444500002E41000007
:103C9000424F0000000000002E2E00002F2E0000DA
:103CA0002E2F00006D6F00006C6F00006C6500002F
:103CB0002F6600006C610000736800002F66000032
:103CC0006C610000736800002E63000000000000BB
:103CD0002E2E00002F2E00002E2F00006D6F0000F2
:103CE0006C6F00006C6500002F69000032630000FB
:103CF0002F690000326300005F70000072690000ED
:103D0000762E0000680000005F7000006F770000F2
:103D1000657200006F66000066000000506F0000D2
:103D200077650000726F000066660000000000000A
:103D30002E2E00002F6D00006D6100003736000050
:103D4000363000002E630000000000005F420000DB
:103D50004C570000484C0000564C00002E44000018
:103D60004154000000000000101100001412000077
:103D7000130000000116000017000000038000007F
:103D80000F0F00000F00000080CD20000102200076
:103D90001088700051CA800061816000A3428000D9
:103DA000830F5100040032000100A20051CA8800B4
:103DB000110020001088700050CA8000620160006D
:103DC000B142800081804000810F51000500320027
:103DD0000010A20050CA88002100200080CD2000E1
:103DE0001088700050CA800064016000C1428000E9
:103DF000C208DD00810F5100050032000020A20042
:103E000050CA88004100200080CD2000108870003A
:103E100050CA800068016000D1428000C308DD0004
:103E2000810F5100050032000030A20050CA880006
:103E30008100200080CD20001088700050CA8000D2
:103E400070016000E1428000C408DD00810F510074
:103E5000050032000040A20050CA88000101200085
:103E600080CD20001088700000000600D0C98000BE
:103E700000000600889FBE008A1F78000004BE0074
:103E800030E702000000000038009000FCDE020075
:103E90000000000042CA8000C80090005800900056
:103EA00098D7020000000000DAC9800040CA8000F4
:103EB0005EA90200000000000A004000D0C988008E
:103EC00041062000810F500001003400D1C9880054
:103ED000C0F92F00D1C98000808F500001003D0043
:103EE000D0C9880042CA8000A80090001800900045
:103EF000A4EE020000000000D0C9800042CA800089
:103F0000E00F50000C003D00F1312000810F510006
:103F100004003A000000E800D0C988000032200008
:103F200018003700810F51000F003E000201E80029
:103F300042CA880014003700E00F50000C00320025
:103F4000E1312000810F510003003A000000E90038
:103F5000D0C98800040037000200E80040CA880089
:103F6000810F5100080036004839EF000600370085
:103F70008200E80041CA8800E1312000810F510031
:103F80000100360040CA8800D5A2A80089804400FC
:103F9000C2932100628078001800400000B17800D0
:103FA00031CA8000FF8F500003003A00890078007A
:103FB0008ADA020000000000E48F54000C003A008E
:103FC0004619EC0030CA880001022000810F500021
:103FD00007003A006CFF07004639EF003C39EF005C
:103FE0003E39EF004039EF004239EF004439EF002D
:103FF0004F0578004F04BE000000060000000000DE
:1040000000000000000000000000000000000000B0
:1040100000000000000000000000000000000000A0
:104020000000000000000000000000000000000090
:104030000000000000000000000000000000000080
:107000000200370031587800030178008201E9005E
:10701000E00F5100FBFF3A000000060002003700BD
:1070200001587800030178008201E900E00F510067
:10703000FBFF3A0000000600889FBE008A9FBE004A
:107040008C9FBE008E1F7800000678000205BE00EF
:107050005C149000EC1490000001EB008A0F5400C7
:107060008B8F5C00380032004C409000E04F5000A5
:1070700024003200EE0220000C07470014C0B300C9
:107080000801BE008E0078001C409000AAA30200F8
:107090000000000012002000E00F50002A003A001B
:1070A000404698005C099000EC0990007C08900034
:1070B0008C1090000200400083804800800F540034
:1070C000818F5C000F003100BC4690000B00370040
:1070D0005C089000EC089000080440008984480097
:1070E00014C0B3000801BE008E0078001C40900060
:1070F000AAA30200000000008D46E900E1CF56007F
:10710000F3FF3E000001EB00E00F5500E08F5D0053
:107110000D003200E10220008C80400014C0B3005A
:107120000A01BE001C40900036A3020000000000CF
:1071300012002000E00F500003003A005A16980099
:107140006B16980000017800020078004F07780065
:107150004F06BE004F05BE004F04BE0000000600F3
:10716000881F780000047800E10220008880400039
:1071700014C0B3001840900036A3020000000000C5
:1071800031C0B300E00F500046003A00D122200089
:1071900088804000914078008181FB00C819DD00A3
:1071A000C122200088804000914078008180FB004F
:1071B0008181710021C0B30052A52A00828F510045
:1071C00038003A0078E39000C833DD000600200064
:1071D00068E190008281FB0002002000020373003E
:1071E0008383730048E190000281FB0003002000CC
:1071F000020373008383730058E190004811DD009F
:107200000300200002037300838373000782FB00E6
:1072100084027800060278000401BE006414240091
:107220004505200080407800840F5100858F59006B
:107230001C00320038439100C833DD0006002000F6
:10724000284091008080FB000000200000037300B4
:1072500081837300084091000080FB000100200042
:107260000003730081837300184091004800DD0023
:107270000100200000037300818373000781FB007D
:1072800082017800060178000200BE000400680058
:1072900085806800010070008000EA0000807000B6
:1072A000CF00DE00014078004F04780000000600A7
:1072B00092002000E00F50000C0032008041EB00F3
:1072C00090CF110009003200B0019000818F510071
:1072D00006003A00104090002AA3020000000000BF
:1072E00061016000010032003200200002007800DD
:1072F00000000600889FBE008A1F78000004780006
:107300006011B800080078004BFF07008004780087
:10731000E08F54005F003A0030C0B300984F100077
:1073200054003A0058409000E04F500051003200A5
:107330006000B8005014980061149800EA02200020
:107340000805450002202000890078000A00780026
:1073500032FF0700C02220000800400052C5B300E1
:1073600002487800D022200008004000A2CAB300E2
:107370000248780022C5B300626C9800726C9800D5
:107380006F4141000274980013C4B3001374980055
:10739000202120000800400024C7B30004487800E2
:1073A00030212000080040000448780040212000DF
:1073B00008004000034878005021200008004000E9
:1073C0000248780078019000880990006021200030
:1073D00008004000024878007121200088804000A9
:1073E0004810DE008048780080212000080040001E
:1073F000401ADE000500200004487800902120009B
:10740000080040004819DE0002487800580190004A
:10741000E8019000A0212000080040000248780008
:10742000B1212000888040004810DE0080487800AC
:10743000C021200008004000401ADE0005002000A6
:1074400004487800D0212000080040004819DE00E0
:107450000248780014C0B30018099000A8099000F1
:107460008A00780018409000AAA3020000000000E3
:10747000594498000001EB008040EB001840900058
:1074800042A40200000000008004EA00808474002E
:10749000CF4CDE00090078004F0578004F04BE0095
:1074A00000000600F6874700889FBE008A9FBE0046
:1074B0008C9FBE008E1F78000244780090017800F7
:1074C0001302FB000403B100E90F520009003E0063
:1074D00093429000A2C3B30082CF520005003A004D
:1074E0000388E800B0002000F0B79F00E00F5200D2
:1074F000E6013A000ECE80008E087800C100200020
:10750000F1B79F00E00F5700E00132000041EB00AF
:107510009E4F11000F0032001E4090002AA302006F
:10752000000000008080FB006180600009003A00DC
:10753000F0B79F00E04F5400D4013200E4806000B7
:10754000A3002000F3B79F00D0013A00F1B79F00DD
:10755000CE0137000040EB00004F78001047980044
:1075600004A20200000000008080FB006180600037
:1075700032002000F2B79F00C4013A00E04F5400EF
:1075800004003200E4806000A3002000F3B79F00F5
:10759000BE013A006011B8000E007800F0FE07004E
:1075A0006066B800E14F50001A003A000EF09300F8
:1075B000D1002000F1B79F00E04F5000B30132002E
:1075C0007EF19300C811DD00020020006EF09300F0
:1075D0008080FB00000020000001710081817100AB
:1075E0004EF093000080FB000100200000017100BC
:1075F000818171005EF093004800DD0001002000F1
:1076000000067100818671000C01BE000E0078003A
:10761000D3FE070012002000F2B79F00E34F500096
:107620009A013200D3002000F3B79F00E04F5000D2
:1076300096013A00AE789000C808DD001E789000F0
:107640000080FB008080700000202000808F5000B0
:107650008E013A005EC590004855DD004EC0900096
:107660000080FB00000575000B002000E00F5500B6
:10767000E08F5D0012003A005ED59000C855DD0035
:107680000A0020004ED090008080FB000000200007
:1076900000057500818575002ED090000080FB00EC
:1076A0000100200000057500818575003ED0900026
:1076B0004800DD000100200000057500818575008F
:1076C0005A0F98006B0F9800EE78900031479800A1
:1076D0000141E900D0002000F0B79F00E14F5100C8
:1076E0006A013E003E799000A2EF9F002247980079
:1076F000E04F510065013200AFE997000381FB00C4
:107700000200E9000201600060013A000EC1900031
:107710004811DD007E7890000080FB0000007100C1
:10772000E0B79F0040079800000178006F006100FB
:1077300056013A002EC190004811DD001EC0900095
:107740000080FB00000171006114B800E00F5400DC
:10775000E08F5C0014003A001ED190000281FB0013
:1077600003002000C813DD00060020000ED19000A9
:107770008281FB00020020000201730083817300FC
:107780006ECC90000884FB00090020000803710003
:10779000898371007EC990004811DD00030020003C
:1077A00002047300838473005E7B90004833DD0025
:1077B0004E7890000080FB0000037300D30020008F
:1077C000F3B79F00310132000182FB000500200069
:1077D0000401BE000A00BE0086BF9F004C040200E8
:1077E0000000000090B79F00A1B79F000FBB97005B
:1077F0006130B800F0AF9F0081B79F00EFB09700F5
:107800004408DE007FA997008FB197000000410077
:10781000E08049001FB19700AFB19700000141001F
:1078200081814900B2B79F00C3B79F00820F540007
:10783000838F5C00150139000203540083835C00D0
:10784000AFE997000382FB00050020000401BE00A1
:107850000600BE002C040200000000000002BE0072
:10786000E00F5000E08F58000801320016C0B3004E
:1078700050FF2000800F5200E08F5A0005003600B4
:1078800036C0B300EB0F4200E08F5A0001003E000B
:1078900026C0B30062044200E0844A00380F98001A
:1078A000490F98003FB19700CFB197000200460002
:1078B00083804E0030179800411798007FA89700EA
:1078C0008FB097000C0140008D814800720F980026
:1078D00003179800E34F53001E003A00D100200028
:1078E000F1B79F006FB19700E00F5100E7003A0039
:1078F0005ED99000C811DD00020020004ED8900033
:107900008080FB0000002000000071008180710079
:107910002ED990000281FB000300200002007000BD
:10792000838070003ED990004811DD0003002000E4
:1079300002007000838070001017980021179800D3
:107940004248DD00CE40DE00810070004240DD0094
:107950001C003700D0002000F0B79F00EFB0970068
:10796000E08F5000C90032001FB09700AFB0970001
:1079700000014100818149001217980023179800E7
:10798000E24F530003003A000800440089804C0095
:107990000C00370032002000030020000800BE0069
:1079A00086BF9F004C040200000000008100D1004F
:1079B0000080D3006104640008004000E0804800BB
:1079C0000FBB9700F01FB0000180B0004709DD0039
:1079D0004900DE0000007100C908DE00D30020006D
:1079E000F3B79F00800F5500818F5D00A70039001D
:1079F0000080EB008080EB0070079800010F98007A
:107A00006000B8005007980061079800E34F5300EA
:107A100093003A000040EB00504798007ED9900058
:107A20004811DD006ED890000080FB00000171005D
:107A300002014600E0814E00120F9800230F9800CB
:107A4000E10220008E80400014C0B3001E40900070
:107A500086BF9F0036A30200000000000FBB970006
:107A6000E00F50007E003A00D02220000E004000BF
:107A7000104078008080FB00C808DD00C022200094
:107A80000E004000104078000080FB0080807000F5
:107A900050A52A00808F500071003A001E7190009E
:107AA000C811DD00020020000E7090008080FB00F5
:107AB0000000200000017100818171006E6890005B
:107AC0000080FB0001002000000171008181710035
:107AD0007E6890004800DD00010020000001710078
:107AE000818171002025250011162400800F51008E
:107AF000818F59005A003A00502120000E004000AA
:107B000010417800C811DD00020020004021200053
:107B10000E004000104078008080FB000000200034
:107B20000001710081817100202120000E004000C1
:107B3000104078000080FB0001002000000171006F
:107B400081817100302120000E004000104078003B
:107B50000080FB004800DD000100200000017100F2
:107B6000818171002027270011142600800F510009
:107B7000818F59003A003A00D02120000E004000C9
:107B800010417800C811DD0002002000C021200053
:107B90000E004000104078008080FB0000002000B4
:107BA0000000710081807100A22120000E014100BF
:107BB000124178000281FB000300200002007000E7
:107BC00083807000B22120000E0141001241780034
:107BD0000281FB004811DD0003002000020070005C
:107BE0008380700050079800610798009021200062
:107BF0000E00400010417800C811DD000200200096
:107C0000802120000E004000104078008080FB00A2
:107C100000002000000071008180710062212000BE
:107C20000E014100124178000281FB000300200098
:107C30000200700083807000722120000E0141005C
:107C4000124178000281FB004811DD000300200092
:107C5000020070008380700070079800010F980088
:107C6000064F7800C219EC0010CE8800300798004B
:107C70006000B80050179800611798000040EB00B2
:107C8000404798000000EB00F0B79F007FB09700DE
:107C90004F0778004F06BE004F05BE004F04BE00E0
:107CA0006F01B1000000060000017800B000200064
:107CB0008001E900E00F50000A0032001240780015
:107CC0000082FB00914278000580FB00000052001A
:107CD00004003A000201E8008100E8000300780097
:107CE000F3FF3700000006008001780021C9290059
:107CF000010037008100E800114178000200FB001C
:107D0000E04F510002003200830F5000F9FF3A00AB
:107D100000000600E8874700889FBE008A9FBE00DB
:107D20008C9FBE008E1F7800E1B79F0091067800FF
:107D3000F4C2B300C3C5B300010037008D06E800EC
:107D40001D417800844F5100FCFF3200834F5100E9
:107D5000FAFF320090057800B200200001022000F6
:107D60000B007800ADFC07000005EB000A07780067
:107D70008C0020008A44780002C2B30011CA290096
:107D80006D447F000E07E800824F54003300360038
:107D9000F0C2B300804F540030003200C0C5B300C1
:107DA000804F54002D003200E0C2B300804F5400D9
:107DB000020032008C0F55000A003900E80F56000F
:107DC00045003A00E0C2B300804F540042003A0040
:107DD00020002000804CDD000C057800BC00200055
:107DE000E7FF3700E04F540004003D003940B30086
:107DF0000884FB000808B10061447C000880FB0097
:107E000081BF9F00F2B79F00B7FF07008FB89700B0
:107E10007FB19700E00F50002F003A00F0CBB30085
:107E200000404400F94F500002003E000914A00039
:107E300007003700F0C9B30000404400F94F50007C
:107E400003003E000904A00000CEB300004444003B
:107E500088757D000A05E800C9FF37006FB09700FC
:107E60000E8846008040EB0000C2B300804F5400F3
:107E700001003E0041C0B30060002000E00F55004B
:107E80001600320050CEB3009B4F100002003A00A3
:107E900050C0B300804D7800E80F560002003A0051
:107EA00020002000804CDD008984FB00638064009A
:107EB000E10F500001003A000144A000EC8464008E
:107EC000E48F540001003A000134A000B14D980045
:107ED0000000EB0001003700600020004F07780031
:107EE0004F06BE004F05BE004F04BE008F00B1001C
:107EF00000000600881F780000047800620051002E
:107F0000E0805900380A9000C80A900062025200CE
:107F1000E0825A006011B800840F5000858F58002D
:107F200009003100284190000281FB00030020007D
:107F30004C0402000000000038119000C8119000AD
:107F400000014100818149000200BE004F04780019
:107F500000000600889FBE008A9FBE008C9FBE0066
:107F60008E1F7800000678000205BE001800200071
:107F700009002000E10F5100E08F59007A0036001F
:107F80003C089000CC089000800F5100818F590070
:107F9000750031001C407800E24F50002F00320085
:107FA000E34F5000450032000084EB008084EB007A
:107FB000E14F50006C003A008206D10082864600F4
:107FC0004969DE007C0890008C109000020140009E
:107FD000E08148000C00780017FC07000084EB00EB
:107FE0008084EB00E00F50005F003A000D00780045
:107FF000F01FB200E002B0006C4778008D06E80088
:108000004969DE007C0890008C109000020140005D
:10801000E08148000C00780007FC0700E00F5000EA
:1080200051003A000E87FB00FD1FB200ED02B000C8
:108030006CC07E004804DD000E047400610565001C
:10804000020032004444DE0002003700FEFF200040
:108050000E04640009002000430037004859DD0089
:108060004850DE0000007100C858DE007C09900016
:108070008C11900000014100818149000C007800C2
:10808000EDFB07000084EB008084EB00E00F500064
:1080900035003A000A054500FA1FB200EA02B000B6
:1080A0006C447D000884FB000A0546001A409000DD
:1080B0004800DD0000047400E6FF37004959DD0088
:1080C0004750DE0000007100C758DE007C099000B8
:1080D0008C11900000014100818149000C00780062
:1080E000D5FB07000084EB008084EB00E00F50001C
:1080F0001D003A004255DD00FA1FB200EA02B0004E
:108100000A004600204190000281FB00030020008D
:10811000C012DD000400200030419000C811DD00D5
:108120000200200002017200838172001040900062
:108130004800DD0001002000000171008181710014
:108140006C407D000080FB000100200000017100F8
:1081500081817100F0FF2000030060008000780042
:10816000020078000004BE000800BE004F0778003F
:108170004F06BE004F05BE004F04BE0000000600C3
:10818000881F7800000478000000EB0020049800AD
:1081900038019000C801900021002000E10F51003B
:1081A000E08F59003D00320018007800300A90003E
:1081B000C00A9000840F5100858F590037003100AC
:1081C000E00F5100E08F590014003A0031C0B300B5
:1081D00090CF100005003A0010119000A0119000FF
:1081E000E00F5100E08F59000C003A006011B80018
:1081F0005204980063049800400190002100200080
:10820000E00F51002500320010119000A0119000E5
:1082100072049800030C980018003700A0409000EA
:10822000E0CF500010003A001800780049FF070026
:108230000001BE00E10F4000E08F48001400320052
:10824000E10F5000E08F580013003600180078004E
:10825000C008900030089000800F5100818F5900B5
:10826000F1FF39000C0037005204980063049800B5
:1082700020FF070070049800010C9800E302200022
:1082800018804100100C98008000EB0003003700BC
:1082900011002000010037002100200001007800BB
:1082A0004F04780000000600889FBE008A9FBE0031
:1082B0008C9FBE008E1F7800000578000204BE006F
:1082C0000406BE0020002000E10F5100E08F59009D
:1082D000960036003A099000CA099000820F5400B7
:1082E000838F5C00910031009A407800E2CF50000B
:1082F00040003200E3CF500052003200E1CF500086
:1083000088003A008805D100888545004959DE007B
:108310007A0890008A10900002014000E081480035
:108320000A00780044FB0700E00F50007D003A008F
:108330000B017800F21FB2006104640008003200F3
:10834000E002200002004000EA407800EFC0600038
:108350000C80FB004400DD0000C07000010037000D
:108360000C40780002014500606998008B05E80028
:1083700010C0B300404598004959DE007A089000CB
:108380008A10900002014000E08148000A00780055
:1083900029FB0700E00F500062003A00FB1FB2000B
:1083A000E00F540005003200CC68DD004466DE00BA
:1083B0000C867000C46EDE000B003700E102200066
:1083C0008B8040006AC1780001CFB300814061001A
:1083D0004869DD004866DE000C067100C86EDE00EC
:1083E0006F4666000CC670008B054500EC6D98006A
:1083F0004C003700484ADD004840DE0000007200B3
:10840000C848DE007A0990008A11900000014100FE
:10841000818149000A00780007FB0700E00F500047
:1084200040003A0008044400F81FB20088004500EC
:10843000EC689800010478004866DE007C6C9800C7
:10844000380037004949DD004740DE000000710078
:10845000C748DE007A0990008A11900000014100AF
:10846000818149000A007800F3FA0700E00F50000C
:108470002C003A004244DD00F81FB200EE0220005A
:10848000080747008E004500E38540008184E8002E
:10849000194178000281FB0003002000C012DD00BA
:1084A000040020001B417800C811DD0002002000FC
:1084B0000201720083817200514278000483FB0044
:1084C0004833DD000700200006027100878271003A
:1084D0006A417F000281FB0003002000020172005C
:1084E0008381720004002F0003016200030020005A
:1084F000C011DD00020020000C0671008D867100A5
:10850000080445006C6C98004861DE0082487800E1
:108510004069DE0003002000824C7800486EDE00D7
:108520008C4D780011C0B300414598004F0778008A
:108530004F06BE004F05BE004F04BE0000000600FF
:10854000889FBE008A9FBE008C9FBE008E1F780051
:10855000000778000204BE00E00F5100E08F5900D0
:108560000B003A005E069000EE069000E00F560009
:10857000E08F5E00120032003E089000CE089000AE
:10858000800F5600818F5E000F0039000C0037000D
:108590000E0078006FFE0700E10F5000E08F5800DA
:1085A0004D0036003E099000CE099000820F500029
:1085B000838F58004E0039000806BE0002003700C5
:1085C0001C0020000D0020000C05BE0061054500C8
:1085D000E0854D003E089000CE089000800F5500C9
:1085E000818F5D0005003900E10F5600E08F5E00CD
:1085F0003C0036002A0020000B0020000A01BE00CB
:108600000E00780053FE0700E00F5000E08F580086
:108610000A003200E10F4000E08F480034003200D1
:10862000E10F5000E08F5800310032008C0F5500F0
:108630008D8F5D00E5FF3A002A003700F4FF2F0020
:10864000F5FF20000A01BE000E00780016FF0700AB
:1086500000017800E00F510018003A00E00F5400CC
:10866000E08F5C00070032000A02BE000801BE0075
:108670000E0078000CFF070000017800E00F5100A9
:108680000E003A005A0798006B0798007E00900091
:108690008E089000E10F4000E08F48001300320088
:1086A00061005000E080580070079800010F9800AA
:1086B00010C0B300504798000C0037001000200095
:1086C00001002000E10F510009003A000080EB009A
:1086D0008080EB0006003700100020000100200021
:1086E000030037006000B800010037000A00BE0038
:1086F0004F0778004F06BE004F05BE004F04BE0076
:1087000000000600E4874700889FBE008A9FBE00E5
:108710008C9FBE008E1F780000057800010678004F
:10872000AA0690008D06E8004B0020007C00320075
:108730007A0090008A089000E00F5000E08F580007
:10874000770032006F8766006C003A0061004000DD
:10875000E080480070059800010D98005A019000D3
:10876000EA0190001A007800E00F5100E08F5900F4
:1087700004003A0040009000808F56005F003900EE
:1087800067003700A04090008180FB008100E90075
:10879000446ADE008480600058003A00EDFD070066
:1087A0000004BE002B002000E10F5000E08F5800B5
:1087B0005B0036001B002000E10F4000E08F480006
:1087C000570032001A00780030099000C00990006C
:1087D000820F5400838F5C00410039004B00200061
:1087E000E00F56004E0032005A019000EA0190005E
:1087F00053FF07000004BE007B002000E00F500084
:10880000E08F5800460032002B002000E10F50009E
:10881000E08F5800420032001B002000E10F4000B2
:10882000E08F48003E0032006011B8001A00780066
:1088300001FA070000067800E00F560038003A0001
:10884000E10220001A804000022020008C00780005
:10885000F2F907001A0278000801BE00040078004F
:1088600084BF9F00A3FD07000FBA97005012980025
:10887000611298000E0037004B4098006011B8005C
:108880001A007800ECF90700E00F500023003A00CE
:108890001A01780052109000E21090006100400030
:1088A000E080480050119800611198000C46E800E3
:1088B0001A007800A0409000814F5600EEFF39006A
:1088C0000C81FB000300200050129000E012900089
:1088D0000201520083815A005210980063109800E0
:1088E00058059800690598000801BE001A00780034
:1088F00080FD070070059800010D98002D05980077
:10890000E10220001A8040004577DD000E0740009C
:108910001E0D98008005EB00010037001B002000B1
:108920000B0078004F0778004F06BE004F05BE00D1
:108930004F04BE004F00B10000000600889FBE003B
:1089400080047800090078000DFE0700000478001C
:10895000E00F540017003A00790190008909900057
:1089600019007800B4F9070000047800E00F540003
:1089700010003A00190890008040EB0090CF1000E2
:108980000B003200B0489000E880600004003A001C
:10899000A9089000C4FC0700E00F50000500320059
:1089A0008000EB000900780056FF0700E7FF370062
:1089B00048002000080078004F04BE0000000600B8
:1089C0000200FA00889FBE0000047800D1BF9F001B
:1089D00011407800F2C2B300824F50000300320011
:1089E000C2C5B300824F500002003A008100E80087
:1089F000D1BF9F006000B800300498004104980087
:108A00005FB89700F1C1B30090CF100005003E00A1
:108A100008007800DAFD07008000EB00110C9800D8
:108A20002B003700F4044400E6805700090078006A
:108A3000B8FC0700E00F500025003A00080078005D
:108A4000BEFF0700A8089000B1489000E00F50005A
:108A500005003200E40F50001D003A00E480600081
:108A60001A0032001A003700E480600018003A0053
:108A700098089000314890007000600013003200A8
:108A8000515190004811DD00415090000080FB00E2
:108A90000001710003002000C011DD000200200071
:108AA000315A90004822DD00A15890008180FB00DF
:108AB000010272000500200004017100858171002F
:108AC0003204980043049800D7FF3700500020007C
:108AD0004F04BE000080FA0000000600889FBE0020
:108AE0008A1F78008004780009007800A4FD070040
:108AF00000047800E00F54001D003A007901900056
:108B000089099000190078004BF9070000047800EB
:108B1000E00F540016003A00190890001040780049
:108B2000FB4F400016003200E04F500014003200AE
:108B30001100200009007800F2FE0700ECFF37006A
:108B4000190D900002022000880078000A007800C9
:108B500032F90700B2002000A90890000A0078004E
:108B600027F907009900780010C0B300C0409800B2
:108B7000080078004F0578004F04BE000000060092
:108B80007901900089099000190078002AF90700FE
:108B900000047800E00F5400F5FF3A00E8FF3700CA
:108BA000889FBE008A9FBE008C9FBE000006780092
:108BB0000204BE0020002000E10F5100E08F5900A8
:108BC0002F0036003C099000CC0990001DC0B30076
:108BD000820F5400838F5C001F003900280037008B
:108BE0000801BE000C007800DAFC07000005BE009A
:108BF000E00F5000E08F58001C003200E10F5000E1
:108C0000E08F58001B003200E10F4000E08F480069
:108C10001A0032006022B8000801BE000C00780083
:108C2000A1FD0700E00F500015003A007C00900005
:108C30008C089000E10F4000E08F480005003200F2
:108C400061004000E080480070069800010E980026
:108C50005D4698000A04BE003C089000CC089000D5
:108C6000800F5400818F5C00DDFF39000000EB00B5
:108C70000300370020002000010037001000200012
:108C80004F06BE004F05BE004F04BE0000000600A8
:108C9000B2002000E04F500009003A0002CE8000F0
:108CA000E00F51000100320000497800E08F5000D1
:108CB000010032008048EB0001CE88000001EB008B
:108CC00002007800000006006F02B000889FBE001E
:108CD0008A9FBE008C9FBE008E1F78000007780020
:108CE00081BF9F00000FEB00FF4661007E416100E5
:108CF000A1FD2F008F80400070805700E9F9070028
:108D0000E1FC2F008F804000F1B79F00E00F500082
:108D100004003A008FB89700A0FD2F000F0040001C
:108D200027FF07006FB69700E00F500003003A00DE
:108D3000E00F560001003A00600020008D80FB002B
:108D40007C81600055003200E00F50000A003200C4
:108D5000E40F500003003A00A0FD2F000F00400078
:108D60005EFF07006FB69700E00F500090003A00DA
:108D70000D34A000070037003C49900071016100EC
:108D8000700020008A003A00E4806000800020002B
:108D900087003A00688066004C00320014AB020085
:108DA00000000000604E98004801DE00724E9800FE
:108DB0004009DE0003002000025698004808DE004B
:108DC000105698008040EB00314E9800415E9800AC
:108DD000515E9800615E9800715E980075004600D3
:108DE00074024600FB0246007A03460010417800F8
:108DF0000284FB004844DD00944178000381FB00BD
:108E00000204740009002000C044DD0008002000B6
:108E1000954378000781FB004811DD0096437800F8
:108E20008781FB000301710003002000020474002D
:108E300083847400014B7800814A7800014A7800ED
:108E4000014878005FA8970011C0B3004140980026
:108E5000E00F5400E08F5C001C00320050159000C1
:108E6000E01590000801BE004DFF0700E00F500024
:108E70004F003A005FA8970061045400E0845C0052
:108E800058009800690098000A01BE006AF80700BF
:108E9000E00F50000D00320045003700E00F500099
:108EA00043003A003C4990000281FB00F001610060
:108EB000400020003E003A00E280600003003200E3
:108EC000610161007000200039003A00688066008E
:108ED000010032000D54A0005FAA970054109000CA
:108EE000E4109000500F9800610F98007C0F9800DC
:108EF0004D479800DC509000C808DD004C509000B1
:108F00000080FB000080700001002000C000DD0038
:108F100000002000BC599000C819DD002C599000B9
:108F20000281FB000281710003002000020070003A
:108F30008380700070079800010F98007C599000A2
:108F4000C811DD00020020006C5890008080FB00FA
:108F50000000200000007100818071004C599000D9
:108F60000281FB000300200002007000838070007B
:108F70005C5990004811DD000300200002007000E1
:108F80008380700050079800610798006000B80067
:108F90003007980041079800300F9800410F980063
:108FA000040F780034029000140798000000EB00D2
:108FB0004F0778004F06BE004F05BE004F04BE00AD
:108FC0006F02B10000000600EA874700889FBE00DC
:108FD0008A9FBE008C9FBE008E1F7800000578001F
:108FE0000104780082057800E3B79F008009EB0058
:108FF0009A0090001A007800ADF80700000778008A
:10900000E00F5700B4003A004A429000E04F52008F
:10901000AE00350061026200AE0032005A029000DC
:10902000EA0290003A019000CA0190000202520048
:1090300083825A00615BB800840F5300858F5B0008
:10904000010036008405780088BF9F0000022000E0
:1090500000004500F0B79F008E007800D1B79F0058
:109060000B077800950037003A019000CA01900084
:10907000F01F20000202600074003A001A0078001D
:10908000C91ADE00C718DD004912DE000482700034
:10909000A04590008B45E90084C5650011003A00A9
:1090A000E00F5100E08F590003003A007A00900071
:1090B0008A089000030037001A099000AA0990005E
:1090C000A4FB0700E10F5000E08F58000D003600B0
:1090D000E10F4000E08F480055003200100D98006D
:1090E000210D98001A0678001A099000AA0990002C
:1090F0000C0078007FFB0700E00F5000E08F580065
:1091000004003A004A4090000074A00040459800D6
:109110006E0037000B84FB000900200000044400AF
:1091200081844C00C976DE00220032002C41900080
:109130008B85FB008B8146000281FB00828F5100F2
:10914000010036008B0651000D4278000801BE0078
:109150008FB897001C40900036A30200000000006A
:109160004A429000E00F500023003A000404B2008D
:109170000E0032003A089000CA0890000800500023
:10918000898058006169B800820F5000838F5800B1
:10919000060031004900DD008FB8970000804000D4
:1091A00002202000FFB0970095F70700496CDD0012
:1091B000360037003A089000CA089000880F500027
:1091C000898F58001F0032004A4190000204B2000B
:1091D0000E00320014C0B3000001BE00FFB09700C3
:1091E0001C409000AAA30200000000004A42900028
:1091F000E00F5000030032000474A00044459800C2
:109200000E0037000464A100444598001A0078005D
:1092100014C0B3000801BE00FFB0970010409000DA
:1092200036A3020000000000E00F500005003200ED
:109230004A4090000074A000404598001E002000A5
:1092400025003700380D9800490D98003A0190002C
:10925000CA01900082017800F31FB20000202000B4
:10926000030150000E047800820F57000100360001
:1092700002047800FFB09700838140000801780065
:10928000830078000FB897005DF707000FB89700CC
:109290000800400080BF9F003A019000CA01900082
:1092A00008014100E081490032059800430598001B
:1092B000EFB097009108440008075700E00F5700EF
:1092C00069FF3A005FB79700030037002E002000C7
:1092D000010037007E0020000E0078004F07780064
:1092E0004F06BE004F05BE004F04BE00AF00B100E8
:1092F00000000600EA874700889FBE008A9FBE00E4
:109300008C9FBE008E1F7800000578000104780055
:1093100082057800E3B79F008009EB009A00900077
:109320001A007800E2F7070000077800E00F570006
:10933000D6003A004A409000E04F50005F003500F0
:1093400062006000D00032005A029000EA029000F1
:109350000B034200E0834A00840F5300858F5B00BB
:10936000010031008E05780088BF9F0000022000B8
:1093700000004500F0B79F008E007800D1B79F0035
:109380000B077800B00037003A019000CA01900046
:10939000F01F2000020260008E003A001A027800DE
:1093A000C91BDE00C718DD004913DE00068370000C
:1093B000A44590008B45E90086C5650021003A0070
:1093C000E00F5100E08F59000B003A007A00900046
:1093D0008A089000E00F5000E08F58000D003A001E
:1093E0000001BE000400780055FC070070059800DD
:1093F000010D9800040037001A099000AA09900096
:10940000040078004EFC0700E00F5000E08F580089
:109410008F0032004A429000E10F5000E08F580068
:1094200003003A000474A00044459800230037006C
:10943000E10F4000E08F480010003200100D98004E
:10944000210D98004A4190000204B2001000320041
:109450001A00780014C0B3003A099000CA099000BD
:10946000FFB0970010409000AAA302000000000087
:109470004A429000E00F5000030032000474A00044
:10948000444598004F0037000464A100444598000B
:109490001A0678001A099000AA0990000C007800BA
:1094A00094FA0700E00F5000E08F580005003A00E2
:1094B0004A4090000074A000404598002E00200013
:1094C000720037000B84FB000900200000044400F8
:1094D00081844C00C976DE00230032002C419000CC
:1094E0008B85FB008B8146000281FB00828F51003F
:1094F000010036008B0651000D4278000801BE00C5
:109500008FB897001C409000AAA302000000000042
:10951000E00F500028003A003A089000CA08900076
:1095200008005000898058006169B800820F50001F
:10953000838F58000A0031004900DD008FB8970082
:109540000080400002202000800078007FB097005B
:10955000ABF607004A4190000264A1004245980022
:10956000496CDD002C0037003A099000CA099000D0
:10957000880F5100898F5900140032003A02900080
:10958000CA0290005A019000EA019000820F520036
:10959000838F5A000D00310014C0B3000801BE00D3
:1095A000FFB097001C40900036A3020000000000AE
:1095B000E00F5000050032004A4090000074A00007
:1095C000404598001E00200030003700380D9800FC
:1095D000490D98003A009000CA009000F01FB200B8
:1095E00001202000008150000E047800820F5700F7
:1095F0000100360002047800FFB0970000804000B0
:10960000080178008FB897007DF607004A41900066
:109610000264A000424598000FB89700080040007F
:1096200080BF9F003A019000CA01900008014100EC
:10963000E08149003205980043059800EFB097009B
:109640009108440008075700E00F57004EFF3A000A
:109650005FB797003A019000CA0190005A0090004D
:10966000EA009000800F5100818F590002003600FF
:109670005205980063059800CA4090000154A0006C
:1096800041459800010037007E0020000E00780060
:109690004F0778004F06BE004F05BE004F04BE00C6
:1096A000AF00B10000000600889FBE0000047800F3
:1096B0009800900018007800FDF60700E00F5000B9
:1096C00042003A00C84090008180FB000101780010
:1096D0000202B2003D0032000104B200100032006C
:1096E00001022000888040001800780014C0B300F8
:1096F00038099000C809900010409000AAA3020009
:10970000000000008000780010002000E08F500072
:109710002E003A00484090000064A10040449800A8
:1097200058099000E80990001800780042F60700F8
:10973000E00F500025003A00F80C90006B804400C8
:109740001054A00028489000C05C98003848900051
:10975000D05C980048489000E05C98005848900021
:10976000F05C980068489000A05C980078489000F1
:10977000B05C980008509000C054980018509000B9
:10978000D054980014AB020000000000E054980090
:109790004801DE00F25498004009DE00030020007A
:1097A000825C98004808DE00905C98004840900079
:1097B0000054A100404498009800780010C0B30005
:1097C000C040980018007800CAF607004F04BE0099
:1097D00000000600881F7800000478000800780068
:1097E000B1FF0700E00F500001003A00000C7800C4
:1097F0004F04780000000600EA874700889FBE00FB
:109800008A9FBE008C9FBE008E1F780000077800E4
:109810000205BE009E0090001E007800A4F607001E
:10982000D0B79F00E00F5000E3003A004E41900097
:10983000E04F5100DE0035005E009000EE00900029
:10984000800F5500818F5D000300360062016100CA
:1098500001003A000005BE003E069000CE069000D2
:109860006000B8003007980041079800E00F5500ED
:10987000E08F5D00940032001E03780026419000C6
:109880000281FB0003002000491CDD00C714DE003C
:10989000890474004914DD00E00F5600E08F5E007B
:1098A0002300320061065600E0865E00610055002C
:1098B000E0805D000801BE0086BF9F002C0402000E
:1098C000000000000002BE000801BE000C00BE0047
:1098D000E4B79F00F5B79F002C04020000000000D1
:1098E0006FB29700FFB297000FBB9700800F520036
:1098F000818F5A000E00390060001400E0801C00C7
:109900000003660001826600840278000602780087
:109910000401BE0032079800430798000205550075
:1099200083855D001E099000AE099000120037008B
:109930007E0190008E099000E00F5100E08F5900E9
:109940000B003A0006007800FDFA07000001BE0097
:10995000E10F5000E08F58004D003200E10F400051
:10996000E08F48007D00320070079800010F9800DA
:10997000120F9800230F9800E00F5100E08F59005C
:109980004E0032002C003700CE409000E280600094
:10999000070032001E007800E9FA07000001BE004F
:1099A000E00F5000E08F580004003A002600370016
:1099B0001E00780067F907000001BE00E10F4100BA
:1099C000E08F490004003A004E4090000074A0006F
:1099D0004047980053003700E10F5100E08F5900D5
:1099E000060036009E007800310A9000C10A9000FF
:1099F000840F5100858F5900050039004E409000BA
:109A00000074A00040479800220020005700370053
:109A1000120F9800230F98003E029000CE02900093
:109A20000402440085824C003407980045079800E2
:109A30000805550089855D00880F5500898F5D00F8
:109A4000D1FF3E00010037000805BE003E02900035
:109A5000CE0290000402450085824D003407980034
:109A6000450798000A027800F41FB20005002000A4
:109A7000E00F5200E08F5A00120032001E00780002
:109A80001CF90700E00F5000E08F580004003A0076
:109A90004E4090000074A0004047980044003700FA
:109AA0004759DD004955DE000A057100C95DDE0039
:109AB0000005450081854D00030037000205BE000A
:109AC000010037000405BE003E009000F01FB20008
:109AD0002A0032003E099000CE099000820F550006
:109AE000838F5D00250032004E4090000004B200DC
:109AF00010003200010220008E8040001E0078001D
:109B000014C0B30010409000AAA30200000000009F
:109B1000CE409000E00F5000040032000174A0001D
:109B20004147980010002000220037000164A10086
:109B300041479800010220008E8040001E007800FE
:109B400014C0B3000A01BE001040900036A302000A
:109B500000000000E00F5000060032004E40900070
:109B60000074A0004047980012002000D2B79F0068
:109B7000110037003A0F98004B0F98003E009000FC
:109B8000CE0090005E019000EE019000820F500028
:109B9000838F58000800360050079800610798002E
:109BA0004E4090000054A00040479800020037004B
:109BB00020002000D0B79F005FB097004F077800CB
:109BC0004F06BE004F05BE004F04BE00AF00B100FF
:109BD00000000600FF4F500002003E008040780069
:109BE000060037008040EB00F2C3B300824F500004
:109BF00002003E0001C4B30080C050000140780064
:109C000000000600889FBE008A1F7800800478004C
:109C1000A058EC00A0F8B70001C6B300814F500077
:109C200001003600A078EF00018A21009140780001
:109C3000814C78000904780000C2B30000C14000E4
:109C4000026C780000C6B300804F5100010036005E
:109C5000004C51000985E8000144B000014D780036
:109C600000C6B30080CF50000100360000CD500088
:109C700019407800D7FF0700804C78001840780022
:109C8000D4FF0700004C78001A407800D1FF07008D
:109C9000004D78004F0578004F04BE00000006001C
:109CA000800078000000EB00E48F500009003200D3
:109CB000E88F50000700320010002000E08F5000B5
:109CC00004003A00A0C480008000EA000080700018
:109CD0004F00DE0000000600889FBE000004BE00AA
:109CE000090444000100370069045400E80F5400DF
:109CF000FDFF3C000100370069044400E00F540000
:109D0000FDFF350008007800E5FF0700E00F500078
:109D1000F3FF3200080078004F04BE000000060088
:109D200001002000E80F5000E08F58002B003E009B
:109D30000060010008003700090037000B00370001
:109D40000E003700110037001300370015003700F0
:109D5000180037001C0037000041EB000C003700F2
:109D60000041EB0001C2B300140037000041EB00DA
:109D700001C2B30001407800110037000041EB0040
:109D80008240780000C2B3000D00370002C2B30069
:109D900082407800F7FF370002C2B3008040EB003A
:109DA000F4FF370002C2B300824078000040EB00AD
:109DB0000300370002C2B3008040EB00024078008D
:109DC000D4BB04000000000052C0B300F1C0B300D7
:109DD00000C2B300D4BB0200000000000000060077
:109DE000881F78000004780008007800CCFF070086
:109DF0006140B800E80F5000E08F58003E003E0080
:109E00000060010008003700090037003700370004
:109E10000D00370035003700170037001F003700EE
:109E200030003700310037000000210030003700DB
:109E300040002000FE6302000000000090AA020023
:109E4000000000002C00370000102000FE6302001C
:109E50000000000040002000FE630200000000003F
:109E60000041EB0082407800F0C0B300D4BB020098
:109E7000000000002000370040002000FE630200C8
:109E80000000000000012000FE630200000000004E
:109E9000600F2000704688001700370060EA290034
:109EA0006AAD02000000000000047800E00F5400DA
:109EB0000E003A0021002000A0962100F8AD02001B
:109EC0000000000021002000C0962100F8AD020033
:109ED00000000000080078006AAD020000000000E9
:109EE000020037009838EF009A38EF004000200059
:109EF000FE630200000000004F047800000006002E
:109F00000400FA00881F7800000478000001EB00CC
:109F10006000B80078BC0200000000008043EB0045
:109F2000074378008742780007427800874178002D
:109F300007417800874078000740780084BB020022
:109F4000000000008040EB0000C1B30090BA0200A6
:109F5000000000008040EB0010C1B30090BA020086
:109F6000000000008040EB0040C1B30090BA020046
:109F7000000000008040EB0050C1B30090BA020026
:109F8000000000008040EB0020C1B30090BA020046
:109F9000000000008040EB0030C1B30090BA020026
:109FA000000000008040EB0060C1B30090BA0200E6
:109FB000000000008040EB0070C1B30090BA0200C6
:109FC000000000008040EB000140780090BA0200E1
:109FD000000000008040EB0010C0B30090BA020007
:109FE000000000006140B800E80F5000E08F58000A
:109FF00056003E00006001000800370009003700ED
:10A00000130037000F0037004D00370014003700F1
:10A0100024003700480037004900370000002100C5
:10A02000480037009AAA020000000000F1F72F0054
:10A0300080CD2000108860009C28EF009E28EF0053
:10A04000030037000010200016640200000000002A
:10A050004000200016640200000000000E003700DF
:10A0600040002000166402000000000000012000F3
:10A0700016640200000000008040EB00E0C1B30065
:10A0800090BA020000000000CE28EF00F1BF2F00C0
:10A0900080CD200010886000AC28EF00AE28EF00D3
:10A0A0002A00370060EA29006AAD020000000000C3
:10A0B000E00F500020003A00D0BF9F00E0BF9F009B
:10A0C0002100200066805700F8AD0200000000006B
:10A0D0002100200064805700F8AD0200000000005D
:10A0E00050CB8000DFB89700808F500004003A000A
:10A0F00060CB8000EFB89700808F50000B003200DB
:10A100006000B800B8AD020000000000210020008F
:10A11000A096210040AE02000000000021002000B7
:10A12000C096210040AE0200000000000000EB00DD
:10A130006AAD020000000000AC28EF00AE28EF007E
:10A140004000200016640200000000004F04780068
:10A150000080FA0000000600AC58EC008040780057
:10A1600001007800ACF8B7000100FB00E0CF500020
:10A170000800340082C2B30082CF50000B003400CC
:10A1800001C8B3008000FD00ACF8B7008000FD00FE
:10A190000000060042002000811F78001100090025
:10A1A0000200D800CF0078000000EA00000006009E
:10A1B0000400FA00889FBE008A9FBE00984380007A
:10A1C0000005EB001000200091032000808040007B
:10A1D0008180400002802000E2807800888F50005B
:10A1E0000200340000057800010478000000E80057
:10A1F000E40F5000F4FF340070CB800062051500BE
:10A2000022002000801F7800110009000200D80001
:10A21000800078004F00780001D5B900C9DA20002D
:10A22000890F54000C00340001FA2000810F540003
:10A2300007003C0088845400809FBE001100090084
:10A240008204D800800478004F00BE00110037005F
:10A250008004EA000F00370071BB2000810F54001A
:10A2600004013C00813EB100810F54000B0034001A
:10A2700089C12F008884440092FF2F00809FBE0078
:10A28000110009008204D800800478004F00BE004D
:10A29000C912B000808F540001003400800478009F
:10A2A0008000EA00818F540001003D0081047800A5
:10A2B000311F2000810F54000A003C00E189210079
:10A2C00091407800E0CF50000300320060458800E4
:10A2D0007045880007003700AC28EF00AE28EF007B
:10A2E000040037000A804400704588000A8054004A
:10A2F000604588009ED8BF004240A9001400340089
:10A300009FD8BF00120032006C8057003DFE07004E
:10A310006FF19700DFF097004FF09700D4BB020079
:10A32000000000005FF19700CFF097006FF09700FA
:10A330000CBC0200000000004FF19700EFF0970006
:10A340005FF09700F0BB020000000000060037003D
:10A3500081FF07000001EB00800078000000EB00A7
:10A3600078BC020000000000E789210097437800D4
:10A37000E0CF5300160032009DD8BF007059B400E2
:10A380009DF8B700FE4F50000200360070F9EF0054
:10A3900004003700E04F500002003A0010C0B30044
:10A3A00070F9B700D5892100954278008580FB00BF
:10A3B0004309DE00C408DE008143780002437800D0
:10A3C00004C2B300854178000040EB00070037006D
:10A3D0000743780005C2B300054278008541780044
:10A3E00007417800874078000740780084BB02006E
:10A3F00000000000D3D7BF000080FB000000EA008F
:10A400004F00DE008000EB00E04F500005003200FE
:10A41000E1922100914078008180FB008100E900F9
:10A42000CF08DE002EF9B700E08F500007003200A1
:10A4300071CB80002103B00071CB8800401F200049
:10A44000808F50000100340070CB8800D0D7BF004F
:10A450000080FB000000EA004F00DE008000EB00FF
:10A46000E04F500005003200D19221009140780069
:10A470008180FB008100E900CF08DE002DF9B700E4
:10A48000E08F50000700320071CB80002103B10043
:10A4900071CB880040ED2F00808F500001003D00FF
:10A4A00070CB880010C0B300411F2000810F540002
:10A4B00003003C000040EB008000EB00050037008B
:10A4C000C1922100914078008180FB008100E90069
:10A4D000CF08DE002CF9B700E08F500003003200F7
:10A4E0006000200052DD020000000000E00F550077
:10A4F0000D003A00E08F540060003A009FD8BF0082
:10A500005E003A00401F2000800F54005B003400C2
:10A5100010C0B3009FF8B7007000200052DD0200A9
:10A5200000000000010037009F78EF0010082000B5
:10A5300041458000808F5000030034005145800069
:10A54000808F500008003C00AC28EF00AE28EF00E0
:10A5500001C2B30080C0B30090BA02000000000046
:10A5600001C2B300050037008040EB0080C0B3009B
:10A5700090BA0200000000008040EB00B0C0B300C1
:10A5800090BA0200000000009ED8BF000200320016
:10A590000040E9009EF8B700D8ECAB003B00320069
:10A5A000F1F72F0080CD2000108860009E78EF002A
:10A5B000724480008E28EF000004EB0010002000A1
:10A5C00071042000808040008181400004802000D0
:10A5D000E4817900828F5100020034000004780089
:10A5E00003017800818040000380200081804100C9
:10A5F0008008EB000000E800E60F5000F0FF340098
:10A6000080BB2000800F510020003400F8448800F7
:10A610009C08ED00E20F50001C003E0010C0B3008B
:10A62000E20F5400030032000040EB008000EB001A
:10A6300005003700B1922100914078008180FB0035
:10A640008100E900CF08DE002BF9B700E08F500051
:10A65000030032007000200052DD02000000000004
:10A66000E20F540009003A0060C0B3009EF8B70042
:10A67000060037008004EB0006FF3700301F200083
:10A68000800F5400A8FF3400A8FF37004F05BE001C
:10A690004F04BE000080FA0000000600EE8747006D
:10A6A000889FBE008A9FBE008C9FBE008E1F7800D0
:10A6B0000E0078000F077800AE01B100030009001A
:10A6C000001FEB0000077800A3FE07000041EB002D
:10A6D00080407800D4BB020000000000A1D8EC004C
:10A6E000A1F8B7008080FB00C508DE0002C2B300FD
:10A6F000FA81570082F178007F4060008101E90013
:10A70000E78161000041510002427800FA8257005F
:10A7100084F279008100E800E78060000041780061
:10A7200082F27800DFEB97004FEB9700BFEA9700CB
:10A730002FEA97009FE997000FE99700FFE0970045
:10A740006FE0970084BB020000000000D3D7BF0079
:10A750000080FB000000EA004F00DE008000EB00FC
:10A76000E04F500005003200019321009140780035
:10A770008180FB008100E900CF08DE0030F9B700DE
:10A78000E08F50000700320091CB80002103B00021
:10A7900091CB8800401F2000808F500001003400C2
:10A7A00090CB8800D0D7BF000080FB000000EA00FB
:10A7B0004F00DE008000EB00E04F5000050032004B
:10A7C000F1922100914078008180FB008100E90036
:10A7D000CF08DE002FF9B700E08F500007003200ED
:10A7E00091CB80002103B10091CB880040ED2F0078
:10A7F000808F500001003D0090CB88009ACB8000F4
:10A80000E00F55005300350098438000A1438000BD
:10A81000C6438000D24380006116B9006142B9008E
:10A820000C0642008D864A00018040006102B9009A
:10A830000C0642008D864A00B04380006302B900D6
:10A84000CFA2DE000C0642008D864A0006004300BF
:10A850006102B9000C0242008D824A00D0FF2F0035
:10A860000088B900CF80DE00C3FF2F0003C4B90009
:10A87000CFC4DE000000440081804C006333B90087
:10A88000CFB3DE000000430081804B004211DD00A9
:10A89000CF91DE0000064100818649000C00420095
:10A8A0008D804A006154B9000801BE00F4B79F00D2
:10A8B00085BF9F004C040200000000000E7D2000B8
:10A8C000811F7800110009004E08D800CF007800E1
:10A8D000800555006B4588007FB297008FBA9700BE
:10A8E0000C0052008D805A000801BE004C0402008A
:10A8F00000000000811F7800110009004E08D800F8
:10A90000CF007800000555007A45880081DA2F00D5
:10A91000818F550001003D0061458800810F550081
:10A9200002003D0080DA2F0070458800802520005D
:10A9300061458000808F5000010034006045880030
:10A940008025200071458000808F50001100340068
:10A950000F003700F24380000A91B90044ED2F0048
:10A96000110009004419D800000178000A014100D3
:10A9700062458800E04380000A80B900811F7800AA
:10A98000110009004408D800CF0078000A004000F8
:10A99000704588001008200041458000808F5000DD
:10A9A0000300340051458000808F500008003C00B7
:10A9B000AC28EF00AE28EF0001C2B30080C0B300A6
:10A9C00090BA02000000000001C2B3000500370089
:10A9D0008040EB0080C0B30090BA0200000000008D
:10A9E0008040EB00B0C0B30090BA0200000000004D
:10A9F0004F0778004F06BE004F05BE004F04BE0053
:10AA0000EF00B10000000600889FBE00A0CB8000D0
:10AA1000800040008080400000468000E00F500031
:10AA200001003D000000EA008080400010468000E8
:10AA3000E00F500001003D000000EA00808040006F
:10AA400020468000E00F500001003D000000EA00B9
:10AA5000008040004200DE00A0CB880018002000EB
:10AA6000ED0F5000010036000004EB0011C0B300F0
:10AA7000EE0F500003003E008040EB000000EB00B2
:10AA80000400370033D9BF000080FB000000E9005C
:10AA90004F00DE008000FD0033F9B7008000FD00AC
:10AAA000E00F5000050032000041EB0082407800CA
:10AAB000F0C0B300D4BB020000000000A0CB8000B7
:10AAC000ED0F500011003E00A218EC0010C58800E8
:10AAD000E50F500007003400EA0F500001003A0073
:10AAE000A238EF000041EB008240780000C2B300C2
:10AAF000030037000041EB008240780002407800FC
:10AB0000D4BB0200000000000500370092FD0700E2
:10AB10000001EB008000EB0078BC020000000000A8
:10AB2000B0468000E00F500004003200D628EF004D
:10AB30005000200052DD020000000000A143800010
:10AB4000803E2000808F500017003400B243800008
:10AB5000800F510014003400C2438000800F510068
:10AB600011003400E2438000800F510003003C00DC
:10AB7000F2438000800F51000B00340020082000B9
:10AB800042458000800F510007003400524580008C
:10AB9000800F510004003400AC28EF00AE28EF0015
:10ABA000180020006600370093438000803E20009C
:10ABB000C2438000808F51000A003C00808F50000B
:10ABC00008003C00B4438000800F520005003C00A8
:10ABD000800F510003003C00D4438000800F5200DE
:10ABE00045003400D04380004500200080037800F9
:10ABF000811F7800110009008500D8008003FD0046
:10AC0000CF0078005400200000037800811F7800F6
:10AC1000110009008401D8000003FD00CF00780076
:10AC200086834300B6438000809FBE001100090068
:10AC30000503D800000378004F00BE008683430060
:10AC400000037800811F7800110009000501D80079
:10AC50000003FD00CF0078008682430000037800E7
:10AC6000811F7800110009000400D8000003FD00D6
:10AC7000CF00780086824200801F78001100090012
:10AC80008400D800800078004F0078006400200025
:10AC9000809FBE00110009008401D8008001780067
:10ACA0004F00BE0083804000A6FF2F00811F780068
:10ACB000110009000600D80000037800CF007800DA
:10ACC00006804000B6FF2F00809FBE0011000900E3
:10ACD0000601D800000378004F00BE0006014000C6
:10ACE000028042000000EA006045880085025100B1
:10ACF0007545880012003700E3438000F14380006F
:10AD0000808F510002003C00808F50000A00340008
:10AD100042002000811F7800110009008201D80044
:10AD2000CF00780060458800110009008200D8003B
:10AD30007045880002003700AC28EF00AE28EF0015
:10AD40001008200041458000808F5000030034002F
:10AD500051458000808F50000B003C00AC28EF0074
:10AD6000AE28EF000041EB008240780000C2B30043
:10AD7000F0BB0200000000000041EB0082407800C0
:10AD800000C2B300080037000041EB0082407800A9
:10AD900002407800F0BB0200000000000041EB0020
:10ADA00082407800024078000CBC020000000000E5
:10ADB00080DA2F0061458000808F500001003D0047
:10ADC0006045880080DA2F0071458000808F500038
:10ADD00001003D007045880080252000614580000D
:10ADE000808F5000010034006045880080252000DD
:10ADF00071458000808F500001003400704588004C
:10AE0000084078008000EB00E04F5400050032005D
:10AE100021932100914078008180FB008100E900AE
:10AE2000CF08DE0032F9B700E08F50000300320097
:10AE30004000200056DD02000000000010C0B300FA
:10AE4000E00F5400030032000040EB008000EB00F4
:10AE50000500370011932100914078008180FB00AC
:10AE60008100E900CF08DE0031F9B700E08F500023
:10AE7000030032000080EB0052DD02000000000001
:10AE80004F04BE00000006000400FA00881F78008E
:10AE900000402000C1668000008060004400320055
:10AEA000F1BF2F0080CD200010886000778A21003C
:10AEB00097437800E0CF53000C003A000700780079
:10AEC000A8F8B70010C0B300A7F8B7000743780090
:10AED0008742780007427800874178000741780070
:10AEE000874078007F40400015003700A8D8BF0099
:10AEF000E1CF530015003A00E24F50002C0034001F
:10AF0000FD4F50002A003C0021C0B3008000FD002E
:10AF1000A7F8B7008000FD000040E800A4F8B700E3
:10AF2000FFC343000043EB008642780006427800EE
:10AF30008641780006417800874078000740780015
:10AF400084BB02000000000019003700E2CF53006C
:10AF500017003A00418A21009140780080CF5000CC
:10AF600013003D0071C2B300814F500010003C003F
:10AF700030C0B300A7F8B700FEC343000743780012
:10AF80008042EB0005427800854178000741780057
:10AF9000874078000740780084BB02000000000072
:10AFA0007000200052DD020000000000A678EF00D3
:10AFB000A8D8BF0031C6B300814F500002003C004A
:10AFC0000040E800A8F8B70020C3B300818A210040
:10AFD0009140780080CF50000B003400A778EF003C
:10AFE0008043EB00074378008742780007427800EF
:10AFF0008741780007417800874078000740780053
:10B0000084BB020000000000A8D8BF00E54F50003C
:10B0100015003A00A5D8BF00E14F500009003A00E2
:10B02000A7D8BF00E14F50000F003A0020C0B30086
:10B03000A5F8B700000520006045880000FB2F0040
:10B0400008003700E24F500007003A00A7D8BF00C1
:10B05000E14F500004003A00A5F8B70000052000B9
:10B060006045880070458800A8D8BF00FE4F50009A
:10B0700012003A00A7D8BF00518A21009140780001
:10B08000E0CF500008003A00E24F500006003A00BE
:10B0900010C0B300A5F8B700000520006045880087
:10B0A0007045880005003700E24F500003003A0069
:10B0B000A578EF00AC28EF00AE28EF0080C2B30007
:10B0C000818A21009140780080CF500009003A0029
:10B0D000A7D8BF00E34F500006003A0010C0B300ED
:10B0E000A5F8B7000105200061458800AE28EF00F3
:10B0F000A6F8B7001008200041458000808F50005E
:10B100000300340051458000808F50000B003C004C
:10B11000AC28EF00AE28EF000041EB008240780041
:10B1200000C2B300F0BB0200000000000041EB00D1
:10B130008240780000C2B300080037000041EB00F5
:10B140008240780002407800F0BB0200000000005E
:10B150000041EB0082407800024078000CBC020005
:10B1600000000000688A210018447800E04F540075
:10B170002200320066805700A2FA07004FF99700BC
:10B18000BFF897002FF89700D4BB02000000000022
:10B190003FF99700AFF897004FF897000CBC0200FA
:10B1A000000000002FF99700CFF897003FF89700B4
:10B1B000F0BB020000000000A658EC00A6F8B700A3
:10B1C000F1C7B300814F500012003A00A678EF009B
:10B1D0000041EB0082407800024078000CBC020085
:10B1E000000000000041EB0082407800024078003F
:10B1F000F0BB02000000000006003700D6FB07008D
:10B20000004178008840780001407800D4BB0200FB
:10B21000000000004F0478000080FA0000000600E3
:10B22000CDFB070000417800804078000040EB0033
:10B23000D4BB020000000000D0D7BF000A003200DB
:10B24000D3D7BF000800320040458000AA08B400F0
:10B2500022002000110009000200D8006009B0009F
:10B2600050CB880010C0B300117D210091407800C0
:10B27000E0CF500012003200417D21009140780063
:10B28000E0CF50000E00320040458000AA08B40014
:10B2900022002000110009000200D80060CB8800C5
:10B2A00051092000810F500002003E00800C200058
:10B2B00060CB8800A0F62F006C39B4000200370084
:10B2C000E04F50000D0032008043EB000743780050
:10B2D000874278000742780087417800074178006C
:10B2E000874078000740780084BB0200000000001F
:10B2F000AC28EF00AE28EF000000060043458000B8
:10B3000052CB8000828F510001003100AAF8B700B3
:10B3100061CB8000818F51000200360010C0B30065
:10B32000AAF8B70050458000820F5000010031009C
:10B33000AB78EF00810F50000200360010C0B30060
:10B34000ABF8B700AAD8BF00B18A210091407800BD
:10B3500006003A00E0CF500008003A008000FD00EF
:10B36000A9F8B7008000FD0015003700E14F50003C
:10B3700002003A00E0CF500010003200E1CF500050
:10B3800004003A00E04F500002003A00A9F8EF0034
:10B390000B003700A9D8BF004240A90002003400CA
:10B3A00020C0B30005003700E04F5000020032001B
:10B3B000E0CFB30001003700A0C0B300A9F8B70088
:10B3C000978A210097437800E0CF53000B003A00A2
:10B3D000C01220006045880070458800074378004F
:10B3E0008742780004C2B3008741780007417800A3
:10B3F000874078000440780036003700E1CF5300E2
:10B400000B003A00C012200060458800AE28EF0013
:10B410008043EB00074378008742780007427800BA
:10B4200003C2B3000741780083407800280037004A
:10B43000E1CF43000A003A00AC28EF00C012200020
:10B440007045880007C2B3000043EB0087427800D4
:10B450000642780086417800064178001B003700DC
:10B46000E2CF43000D003A0040ED2F006045880018
:10B47000C0122000704588008043EB0006C2B30074
:10B4800087427800074278008741780007417800BA
:10B4900087407800074078000E003700E2CF530065
:10B4A0000E003A00C01220006045880040ED2F00D9
:10B4B000704588008043EB0007437800874278009E
:10B4C000074278008741780002C2B30086407800C6
:10B4D0000640780084BB040000000000EACF53005F
:10B4E00004003A00C01220006045880040ED2F00A3
:10B4F000704588000000060017FB07000041780037
:10B500008040EB00D4BB020000000000D1D7BF0098
:10B510000080FB000000EA004F00DE008000EB002E
:10B52000E04F5000050032009193210091407800D7
:10B530008180FB008100E900CF08DE0039F9B70007
:10B54000E08F500002003200A0F62F00D0C4880027
:10B55000D4D7BF000080FB000000EA004F00DE00EF
:10B560008000EB00E04F5000050032008193210085
:10B57000914078008180FB008100E900CF08DE0067
:10B5800038F9B700E08F5000020032006009200057
:10B59000D0C48800D0D7BF000080FB000000EA00C4
:10B5A0004F00DE008000EB00E04F5000050032004D
:10B5B00071932100914078008180FB008100E900B7
:10B5C000CF08DE0037F9B700E08F500007003200E7
:10B5D000D0C48000E00F5000020032009A38EF0023
:10B5E00002003700A0F62F009838B400D3D7BF0070
:10B5F0000080FB000000EA004F00DE008000EB004E
:10B60000E04F500005003200619321009140780026
:10B610008180FB008100E900CF08DE0036F9B70029
:10B62000E08F500007003200D0C48000E00F5000CF
:10B63000020032009A38EF00020037006009200053
:10B640009838B4000000EB00017D210091407800A3
:10B65000E0CF500004003200D3D7BF000080FB00D1
:10B660000000EA004F00DE008000EB00E04F5000D9
:10B670000500320051932100914078008180FB0049
:10B680008100E900CF08DE0035F9B700E08F5000F7
:10B69000010032009838EF000000EB00417D2100EE
:10B6A00091407800E0CF500004003200D1D7BF00B5
:10B6B0000080FB000000EA004F00DE008000EB008D
:10B6C000E04F500005003200419321009140780086
:10B6D0008180FB008100E900CF08DE0034F9B7006B
:10B6E000E08F5000010032009A38EF005046800091
:10B6F000E00F50004800320001022000810F50008E
:10B700003000320014003C00E60F50003C003200D4
:10B7100006003C00E40F50002F0032003B003C00CC
:10B72000E20F50003B003A0026003700ED0F5000BA
:10B730003600320003003C00E80F500035003A00AC
:10B7400027003700F00F50002D003200F10F50009D
:10B7500030003A002000370001052000810F500022
:10B760001800320008003C00E3805000810F5000B8
:10B77000190032008100E800810F500020003200E3
:10B78000110220000500370051052000810F5000F4
:10B790001100320004003C00E4805000810F500092
:10B7A0001C003A000E00370061052000810F500098
:10B7B000130032008100E800810F500015003A00AC
:10B7C00012003700D0C48000E00F500007003A009C
:10B7D0006009200008003700A0F62F00090037009C
:10B7E000D0C48000E00F5000020032009A38EF0011
:10B7F00008003700A0F62F009838B4000500370085
:10B8000060092000D0C48800020037009A38EF0099
:10B810009838EF00CA28EF0080252000C1C48000BE
:10B82000808F500001003400C0C4880080DA2F00EF
:10B83000C1C48000808F500001003D00C0C488005A
:10B8400080252000D1C48000808F5000010034008A
:10B85000D0C4880080DA2F00D1C48000808F5000CF
:10B8600001003D00D0C48800C1C48000D0C4800065
:10B87000010140006245880000805000704588004A
:10B880000000060000102000FE630200000000001F
:10B8900000202000FE6302000000000000012000E4
:10B8A000FE6302000000000040002000FE63020072
:10B8B0000000000010002000FE63020000000000F5
:10B8C00000012000FE630400000000009C58EC0012
:10B8D0009CF8B70041C6B300814F500022003600EB
:10B8E00050C6B3009CF8B700D2D7BF000080FB0061
:10B8F0000000EA004F00DE008000EB00E04F500047
:10B9000005003200A1922100914078008180FB0067
:10B910008100E900CF08DE002AF9B700E08F50006F
:10B920001100320090C4800075F90700B0C4800097
:10B93000E00F500002003A000040210015003700DF
:10B9400091C48000810F500004003A000000EB0019
:10B9500023F907009238EF000300370020F90700B1
:10B960009618F8009218F90086EC0200000000001A
:10B97000E00F500004003A0076BE02000000000014
:10B98000700060000600320090C480005CF907007F
:10B99000004020001664020000000000B9FF3700DC
:10B9A00090C4800001002000E70F5000E08F580095
:10B9B0005D003E00006001000700370054003700C2
:10B9C0005400370054003700570037005300370049
:10B9D0005300370053003700D0D7BF000080FB0072
:10B9E0000000EA004F00DE008000EB00E04F500056
:10B9F0000500320091922100914078008180FB0087
:10BA00008100E900CF08DE0029F9B700E08F50007F
:10BA1000040032008080EB00B0C48000AEF8070064
:10BA2000B0C48800D1D7BF000080FB000000EA004E
:10BA30004F00DE008000EB00E04F500005003200B8
:10BA400081922100914078008180FB008100E90013
:10BA5000CF08DE0028F9B700E08F50000400320064
:10BA60008080EB00B0C480009BF80700B0C4880061
:10BA7000D3D7BF000080FB000000EA004F00DE00CB
:10BA80008000EB00E04F5000050032007192210071
:10BA9000914078008180FB008100E900CF08DE0042
:10BAA00027F9B700E08F5000040032001100200099
:10BAB000B0C4800088F80700B0C48800D4D7BF00A5
:10BAC0000080FB000000EA004F00DE008000EB0079
:10BAD000E04F500005003200619221009140780053
:10BAE0008180FB008100E900CF08DE0026F9B70065
:10BAF000E08F50000400320011002000B0C480002C
:10BB000075F80700B0C48800B0C4800084F837001E
:10BB1000A7F93700E1FA3700BBFB3700DAFC370042
:10BB2000BFFD370074FE070000000600A0C48800B7
:10BB30000000EB00AAF80700A0C48000E00F50004E
:10BB4000020032009638EF0003003700100020009A
:10BB5000B0C4880072F80700B0462000FE630400FD
:10BB600000000000004020000E6402000000000001
:10BB7000800078000080EB00E08F50000100320070
:10BB800090C480000000060071C58000E08F500066
:10BB900013003200B4D8EC00B4F8B700FF4F5000E7
:10BBA00004003400E380600071C5880000CEB3005B
:10BBB000B4F8B70070C58000E00F500008003200F4
:10BBC000418B2100914078008100FB0001003B0087
:10BBD0008100EA00E0C0B30090BA0200000000005B
:10BBE00010C0B30071C58000E08F50000300320028
:10BBF0000040EB008000EB0005003700418721008A
:10BC0000914078008180FB008100E900CF08DE00D0
:10BC100074F8B700E08F5000040032008040EB0061
:10BC2000E0C0B30090BA020000000000000006006F
:10BC3000889FBE000000EB0002C2B300017D21001E
:10BC4000E1417800818B2100E0CF510007003200F4
:10BC5000E1417800E3C141008370780082CF510058
:10BC6000030036008270780001003700837078008E
:10BC70000000E800E40F5000F0FF3400BAD8BF0025
:10BC80000B0032000802200039022000A18B2100A5
:10BC9000914078000840780090BA0200000000004F
:10BCA0000804E800890F5400F8FF34001C00370036
:10BCB000818B210091407800E0CF500003003200DA
:10BCC00010C2B30090BA020000000000918B210066
:10BCD00091407800E0CF50000300320020C2B30052
:10BCE00090BA020000000000B18B21009140780062
:10BCF000E0CF50000300320000C2B30090BA02004F
:10BD000000000000C18B210091407800E0CF50007E
:10BD10000300320030C2B30090BA020000000000FD
:10BD20000000EB00818B210091407800E0CF5000B3
:10BD300004003A00BAD8BF000080FB000000E90010
:10BD40004F00DE008000EB00E04F500005003200A5
:10BD5000C1872100914078008180FB008100E900CB
:10BD6000CF08DE007CF8B700E08F500004003200FE
:10BD70008040EB0010C2B30090BA02000000000047
:10BD80000000EB00918B210091407800E0CF500043
:10BD900004003A00BAD8BF000080FB000000E900B0
:10BDA0004F00DE008000EB00E04F50000500320045
:10BDB000B1872100914078008180FB008100E9007B
:10BDC000CF08DE007BF8B700E08F5000040032009F
:10BDD0008040EB0020C2B30090BA020000000000D7
:10BDE0000000EB00B18B210091407800E0CF5000C3
:10BDF00004003A00BAD8BF000080FB000000E90050
:10BE00004F00DE008000EB00E04F500005003200E4
:10BE1000A1872100914078008180FB008100E9002A
:10BE2000CF08DE007AF8B700E08F5000040032003F
:10BE30008040EB0000C2B30090BA02000000000096
:10BE40000000EB00C18B210091407800E0CF500052
:10BE500004003A00BAD8BF000080FB000000E900EF
:10BE60004F00DE008000EB00E04F50000500320084
:10BE700091872100914078008180FB008100E900DA
:10BE8000CF08DE0079F8B700E08F500004003200E0
:10BE90008040EB0030C2B30090BA02000000000006
:10BEA0004F04BE00000006004CD9BF000080FB001C
:10BEB0000000E9004F00DE008000EB00E04F500082
:10BEC0000500320021882100914078008180FB002C
:10BED0008100E900CF08DE0082F8B700E08F500053
:10BEE000040032008040EB00D0C1B30090BA0200E1
:10BEF000000000004CD9BF00050032004C79EF0073
:10BF000001C2B300D0C1B30090BA0200000000002B
:10BF100000000600881F7800C058EC00C0F8B70089
:10BF2000EA4F500023003A00C078EF00314680000D
:10BF300050092000808F500006003C008040EB003C
:10BF400060C2B30090BA02000000000001C2B3005A
:10BF50001500370080112000808F5000060034004B
:10BF600001C2B3006E40400090BA02000000000021
:10BF70008040EB000C0037006109B100C508DD000E
:10BF800022082000110009008200D80080007800FB
:10BF90000144780060C2B30090BA020000000000C3
:10BFA00001C2B30088C0500070C2B30090BA020052
:10BFB000000000004F04780000000600889FBE00CB
:10BFC00029248000E884640041003200688B21004D
:10BFD00018447800E04F54000E003A008840780082
:10BFE00050C0B30090BA0200000000008840780002
:10BFF00060C0B30090BA02000000000088407800E2
:10C0000070C0B30090BA02000000000010C0B3007E
:10C01000B6F8B700B7D8BF00120020000100320008
:10C020000001FB0071C0B300EA0F510007003C00A3
:10C0300023002000801F7800110009000301D800B0
:10C04000800078004F0078008140E80000C0400088
:10C05000B7F8B70041C6B300814F50001500340057
:10C06000B558EC00B5F8B70011C0B3008000FD0072
:10C07000B7F8B7008000FD00E34F500001003A0020
:10C08000B578EF00588B210018447800E04F540039
:10C0900008003A008840780070C0B30090BA0200EF
:10C0A000000000008840780060C0B30090BA020031
:10C0B00000000000B5D8BF0065404000718B210032
:10C0C0009140780090BA020000000000B0003700F4
:10C0D00080458000B208B400883E20000880B90086
:10C0E000A8F82000809FBE00110009004888D800F1
:10C0F000000478004F00BE00B6D8BF002700320011
:10C1000009007800B6F8B70050182000800F5400DE
:10C110000A00360001C2B30050C0B30090BA02005A
:10C120000000000001C2B30060C0B30090BA02007A
:10C130000000000001C2B300150037008016200087
:10C14000800F54000600360001C2B30050C0B30097
:10C1500090BA02000000000001C2B30008003700DE
:10C1600040152000800F54000C00360001C2B300BF
:10C1700050C0B30090BA020000000000894078006F
:10C1800060C0B30090BA020000000000894078004F
:10C1900070C0B30090BA02000000000010C0B300ED
:10C1A00051182000810F540003003E000040EB00B6
:10C1B0008000EB0005003700818721009140780066
:10C1C0008180FB008100E900CF08DE0078F8B7002D
:10C1D000E08F50000C00320001C2B30050C0B30029
:10C1E00090BA02000000000001C2B30060C0B300BA
:10C1F00090BA02000000000001C2B30070C0B3009A
:10C2000090BA02000000000071E92F008880400011
:10C2100010C0B300F78F5000030036000040EB0061
:10C220008000EB0005003700718721009140780005
:10C230008180FB008100E900CF08DE0077F8B700BD
:10C24000E08F50000C00320001C2B30050C0B300B8
:10C2500090BA02000000000001C2B30060C0B30049
:10C2600090BA0200000000008040EB0070C0B300F4
:10C2700090BA020000000000B1EA2F008880400060
:10C2800010C0B300EE8F5000030036000040EB00FA
:10C290008000EB00050037006187210091407800A5
:10C2A0008180FB008100E900CF08DE0076F8B7004E
:10C2B000E08F50000C00320001C2B30050C0B30048
:10C2C00090BA0200000000008040EB0060C0B300A4
:10C2D00090BA0200000000008040EB0070C0B30084
:10C2E00090BA02000000000010C0B3004115200009
:10C2F000810F5400030036000040EB008000EB008B
:10C300000500370051872100914078008180FB00B3
:10C310008100E900CF08DE0075F8B700E08F50001B
:10C32000080032008040EB0060C0B30090BA020009
:10C33000000000008040EB0070C0B30090BA020023
:10C340000000000040152000800F540010003E0047
:10C35000B758EC00B7F8B700E34F500004003A00BC
:10C3600001C2B30050C0B30090BA02000000000048
:10C37000B7D8BF00E54F5000050034008040EB0007
:10C3800050C0B30090BA020000000000B778EF0080
:10C390004F04BE0000000600D0D7BF000080FB00A5
:10C3A0000000EA004F00DE008000EB00E04F50008C
:10C3B0000500320011882100914078008180FB0047
:10C3C0008100E900CF08DE0081F8B700E08F50005F
:10C3D000030032002000200052DD020000000000B7
:10C3E000D1D7BF000080FB000000EA004F00DE0054
:10C3F0008000EB00E04F5000050032000188210072
:10C40000914078008180FB008100E900CF08DE00C8
:10C4100080F8B700E08F50000300320020002000B9
:10C4200052DD020000000000D2D7BF000080FB00F8
:10C430000000EA004F00DE008000EB00E04F5000FB
:10C4400005003200F1872100914078008180FB00D7
:10C450008100E900CF08DE007FF8B700E08F5000D0
:10C46000030032003000200052DD02000000000016
:10C47000D3D7BF000080FB000000EA004F00DE00C1
:10C480008000EB00E04F500005003200E187210002
:10C49000914078008180FB008100E900CF08DE0038
:10C4A0007EF8B700E08F500003003200200020002B
:10C4B00052DD020000000000D4D7BF000080FB0066
:10C4C0000000EA004F00DE008000EB00E04F50006B
:10C4D00005003200D1872100914078008180FB0067
:10C4E0008100E900CF08DE007DF8B700E08F500042
:10C4F000030032002000200052DD02000000000096
:10C5000000000600889FBE008A9FBE008C1F780036
:10C510000000EB002386210002852100910320000A
:10C52000808040008180400004802000E48078000A
:10C5300000024000E3027A00818F520001003D00BA
:10C5400081317A00E08F5000050032000002400087
:10C55000E2027A00818F52000100340001317A003A
:10C560000000E800E60F5000ECFF3400404580007A
:10C5700081C38000808F500001003D0080C388008F
:10C580005045800091C38000808F500001003D0025
:10C5900090C388000004EB000C0220004BEB290044
:10C5A0000801440000852100E0007900900320008C
:10C5B0000800400000004000038020006300780075
:10C5C0002386210063057900010555000100500014
:10C5D00001003B000000EB000C80B900809FBE0012
:10C5E000110009004A08D800000578004F00BE007D
:10C5F000EB447C008A4078000940780090BA020041
:10C6000000000000E20F540005003A008944E800F1
:10C610008A4078000940780090BA020000000000CB
:10C620000804E800E60F5400DDFF340082C38000F8
:10C6300040458000E00F500001003D000000EB008D
:10C64000080220000880B900811F7800110009004D
:10C650004208D800CF0078008040780060C1B30065
:10C6600090BA02000000000093C380005245800091
:10C6700008007800E00F510001003D000001EB00D0
:10C680000090B900811F7800110009004308D8000C
:10C69000CF0078008040780070C1B30090BA0200EB
:10C6A000000000004F0678004F05BE004F04BE009A
:10C6B00000000600889FBE0020468000F40F500056
:10C6C0003D003C001146800000468000507502008D
:10C6D0000000000022002000110009000200D80024
:10C6E000037D200003014000F1F92000C801200073
:10C6F000810F51001C003600027721000202400029
:10C70000B8012000810F520017003600047122008A
:10C7100004024000A8012000810F520012003600E0
:10C72000046B23000402400098012000810F520096
:10C730000D00360088012000F5D52600850F520037
:10C7400009003E00830150006C044400818F5100B9
:10C750000500360002005000F8012000810F500053
:10C7600001003E006604440029468000E08F54002A
:10C7700001003D008904EA00F48414008984440027
:10C7800001003B008004EB00F0C58000E00F50008A
:10C79000030035008040EB0090BA0200000000006A
:10C7A000894078000840780090BA0200000000003C
:10C7B000F8C5880007003700F0C58000E00F500082
:10C7C000030035008040EB0090BA0200000000003A
:10C7D000BEB8EF004F04BE00000006006700600016
:10C7E000C800DD00F2058000F08F2F00000061001E
:10C7F00001007000F00588000000060091C580006F
:10C80000E08F500002003A008AC0A9009AC0A80038
:10C810000100700090C5880000000600B218B60044
:10C82000000006008AC0A800000006000080EA00A0
:10C83000B218B60090C5880001003A009AC0A9005D
:10C84000000006001000FA00889FBE008A9FBE000C
:10C85000C6D8BF00E14F500055023A0086EC0200F6
:10C8600000000000E00F500004003A0076BE020015
:10C8700000000000F00060002500320000002100F0
:10C88000EAFF07000001EB006000B80078BC02007E
:10C89000000000008043EB000743780087427800E7
:10C8A0000742780087417800074178008740780088
:10C8B0000740780084BB0200000000008043EB00CA
:10C8C0000743780087427800074278008741780064
:10C8D00007417800874078000740780028BC0200B4
:10C8E00000000000AC28EF00AE28EF0076BE02008A
:10C8F000000000000002B20002003200A2BF0200ED
:10C9000000000000425C020000000000410237000D
:10C91000438C210093417800E1CF510008003200A0
:10C92000E2CF510009003200E0CF51000B003A0085
:10C9300001017800F100200000022000050037000E
:10C9400001017800010220000100370002022000EE
:10C95000F000200078BC020000000000C5D8BF0035
:10C96000E14F40001F003A00C158EC00C1F8B70089
:10C97000FC4F50000A003A0007C2B300074378009A
:10C9800087427800074278008741780007417800A5
:10C99000874078000740780028BC020000000000B3
:10C9A00080C3B300118C21009140780080CF5000EB
:10C9B0003B003600C178EF008043EB00074378006E
:10C9C0008742780007427800874178000741780065
:10C9D000874078000740780028BC02000000000073
:10C9E0002F003700AC50020000000000AC500200E5
:10C9F00000000000AC5002000000000000047800BD
:10CA0000884378000843780088427800084278001C
:10CA10008841780008417800884078000840780014
:10CA200028BC020000000000438C210093417800E4
:10CA3000E1CF51000A003200E2CF51000E00320077
:10CA4000E0CF510011003A00C545DD00C55DDE00B4
:10CA50006F44B9004545DE00834478000B00370081
:10CA60006F40B900C505DE004544DD004545DE00E8
:10CA70008044EB00050037006F40B900C505DE00BB
:10CA80004544DD00C544DE000045EB000981FB00A4
:10CA90008A80FB000B80FB0078BC020000000000D5
:10CAA000C5D8BF000000FB00CF80DE006100400061
:10CAB000E0804800E30F5000E08F5800B9013E00CD
:10CAC00000600100030037006B003700D100370021
:10CAD00093013700D0D7BF000080FB000000EA00C0
:10CAE0004F00DE008000EB00E04F500005003200F8
:10CAF00001892100914078008180FB008100E900DC
:10CB0000CF08DE0090F8B700E08F5000010032003F
:10CB1000C478ED00D3D7BF000080FB000000EA001E
:10CB20004F00DE008000EB00E04F500005003200B7
:10CB3000F1882100914078008180FB008100E900AC
:10CB4000CF08DE008FF8B700E08F50000100320000
:10CB5000C478EC00D1D7BF000080FB000000EA00E1
:10CB60004F00DE008000EB00E04F50000500320077
:10CB7000E1882100914078008180FB008100E9007C
:10CB8000CF08DE008EF8B700E08F500001003200C1
:10CB9000C478EC00D4D7BF000080FB000000EA009E
:10CBA0004F00DE008000EB00E04F50000500320037
:10CBB000D1882100914078008180FB008100E9004C
:10CBC000CF08DE008DF8B700E08F50000100320082
:10CBD000C478ED00C4D8BF0009003B0076BE020057
:10CBE00000000000610060000200320020C0B300BD
:10CBF0000100370010C0B300C4F8B7000A003700C6
:10CC0000E14F50000400340076BE02000000000036
:10CC100061006000F8FF3200C4D8BF00E24F50004E
:10CC200001003400C478EF00D2D7BF000080FB00C1
:10CC30000000EA004F00DE008000EB00E04F5000F3
:10CC400005003200C1882100914078008180FB00FE
:10CC50008100E900CF08DE008CF8B700E08F5000BB
:10CC600050013200C4D8BF00C5F8B70010C0B300EF
:10CC7000C7F8B7004B013700D0D7BF000080FB00DA
:10CC80000000EA004F00DE008000EB00E04F5000A3
:10CC900005003200B1882100914078008180FB00BE
:10CCA0008100E900CF08DE008BF8B700E08F50006C
:10CCB00003003200C378EC0050B202000000000014
:10CCC000D3D7BF000080FB000000EA004F00DE0069
:10CCD0008000EB00E04F500005003200A1882100E9
:10CCE000914078008180FB008100E900CF08DE00E0
:10CCF0008AF8B700E08F500003003200C378ED00DF
:10CD000050B2020000000000C3D8BF0002003B0088
:10CD1000C378EF0004003700E84F500002003400F1
:10CD200080C0B300C3F8B700318C21009140780077
:10CD30008100FB0091AA88000040EB006182100096
:10CD40008080FB0081014200C219DD00818040002B
:10CD5000F88257000181420003097800E08F5100FA
:10CD600001003D000009EB000040E800E74F5000E3
:10CD7000F3FF36008FEB97002FEB9700CFEA970079
:10CD80006FEA97008FF197002FF19700CFF097008F
:10CD90006FF0970084BB0200000000000000EB0071
:10CDA000217D210091407800E0CF50000400320046
:10CDB000C7D8BF000080FB000000E9004F00DE0084
:10CDC0008000EB00E04F5000050032009188210008
:10CDD000914078008180FB008100E900CF08DE00EF
:10CDE00089F8B700E08F5000EE003200C5F8EF0080
:10CDF0008043EB00074378008742780007427800C1
:10CE00008741780007417800874078000740780024
:10CE1000BD00370060458000E00F50006700320021
:10CE2000D4D7BF000080FB000000EA004F00DE0006
:10CE30008000EB00E04F50000500320081882100A7
:10CE4000914078008180FB008100E900CF08DE007E
:10CE500088F8B700E08F500003003200C278EC0081
:10CE600050B2020000000000D1D7BF000080FB00DC
:10CE70000000EA004F00DE008000EB00E04F5000B1
:10CE80000500320071882100914078008180FB000C
:10CE90008100E900CF08DE0087F8B700E08F50007E
:10CEA00003003200C278ED0050B202000000000022
:10CEB000218C210091407800E0CF5000190035000E
:10CEC000FFCF5000100034007FC150008043EB00C2
:10CED000074378008742780007427800874178004E
:10CEE000F1C1B3000740780084BB020000000000DD
:10CEF00020C3B300218C21009140780080CF5000E6
:10CF000026003400190037008043EB000743780007
:10CF1000874278000742780087417800074178000F
:10CF20001B003700FFCF400012003D00F7C1B300E7
:10CF300016CEB300014353008042EB000542780057
:10CF400085417800054178008540780005407800EB
:10CF500084BB020000000000E0CCB300218C210063
:10CF60009140780080CF50000C003D00C2F8B7001F
:10CF70000A0037008143EA000043EB008642780054
:10CF800006427800864178000641780086407800A5
:10CF90000640780084BB020000000000C2D8BF0039
:10CFA0000000FB00011020008080400011AB8800D1
:10CFB000011020000080500020AB8800D0D7BF00B7
:10CFC0000080FB000000EA004F00DE008000EB0064
:10CFD000E04F500005003200618821009140780048
:10CFE0008180FB008100E900CF08DE0086F8B700F1
:10CFF000E08F50000B003200614580000108B10055
:10D000006145880000F82F00AE28B40010E82F001A
:10D01000808F500003003D000000E900604588005B
:10D0200070458800D3D7BF000080FB000000EA00F5
:10D030004F00DE008000EB00E04F500005003200A2
:10D0400051882100914078008180FB008100E90037
:10D05000CF08DE0085F8B700E08F50000B003200EB
:10D06000614580000108B00061458800000820008B
:10D07000AE28B400F0172000808F50000300340069
:10D080000000E80060458800704588000000EB0063
:10D09000217D210091407800E0CF50000400320053
:10D0A000C7D8BF000080FB000000E9004F00DE0091
:10D0B0008000EB00E04F5000050032004188210065
:10D0C000914078008180FB008100E900CF08DE00FC
:10D0D00084F8B700E08F50003200320060458000D5
:10D0E000E00F50000B003A00C5F8EF0080437800D5
:10D0F0000043780080427800004278008041780048
:10D10000004178008040780084BB020000000000ED
:10D1100024003700AC28EF00AE28EF0021003700D4
:10D1200076BE0200000000000002B20002003A00D9
:10D130009ABF0200000000000000EB00217D2100EA
:10D1400091407800E0CF500004003200C7D8BF0003
:10D150000080FB000000E9004F00DE008000EB00D3
:10D16000E04F5000050032003188210091407800E6
:10D170008180FB008100E900CF08DE0083F8B70062
:10D18000E08F50000700320076BE02000000000071
:10D190000002B20002003200A2BF02000000000044
:10D1A000C5F8EF00D2D7BF001A003A0016003700CA
:10D1B000D1D7BF0016003200D4D7BF001400320010
:10D1C000C758EC00C7F8B70041C6B300814F500004
:10D1D000100036008140E800814F500009003A00FD
:10D1E00010C0B300C6F8B700004020008FFD070054
:10D1F000C5F8EF0052D5BF00C3F8B70062D5BF0035
:10D20000C2F8B70060C6B300C7F8B7000100370026
:10D21000C778EF004F05BE004F04BE000080FA0043
:10D22000000006003600F800809FBE00829FBE000E
:10D23000849FBE00869FBE003400F80000002000DE
:10D24000A00188008AC0A900B278AB0001003200BA
:10D250004DFA0700B2B8AB000100320057FB0700DF
:10D26000B238AB000100320071FA0700B218AB000F
:10D270000100320048FC0700B258AB000100320048
:10D28000A0FC0700B2D8AB000100320006FB07008B
:10D29000B318AB000100320006FD0700B338AB0045
:10D2A000010032001BFB07000040200091C58000F8
:10D2B0000080600002003200665C02000000000096
:10D2C0000080200091C580000080600002003200D4
:10D2D000A8980200000000000000210091C5800015
:10D2E000008060000100320056FD07003400F900A4
:10D2F0004F03BE004F02BE004F01BE004F00BE00F4
:10D300003600F90000400600028B2100124178002F
:10D31000B298AB001800320071468000E08F5000D8
:10D320000B0032000080FB00810F5000030034002E
:10D330004300DE00804F510003003900E04F5100F0
:10D34000060032000240E900B0F8B70003003700E1
:10D350008000FD00B0F8B7008000FD00018B2100C7
:10D3600091407800814F510003003200E0C1B300CA
:10D3700090BA02000000000000000600E18A2100CF
:10D38000E00F500003003D0067006000910870004E
:10D39000000006000080EA0091086000000006001E
:10D3A0000200FA00F0BF9F0001017800CF80DE008C
:10D3B000E40F5000E08F580010003E0000600100B4
:10D3C000040037000500370006003700070037006B
:10D3D00008003700120888000E0037006208880035
:10D3E0000C003700720888000A003700D208880055
:10D3F00008003700E2088800060037008F81E90046
:10D4000042102000014D2000E0DC290008EF02005E
:10D41000000000000080FA00000006000200FA0090
:10D42000F0BF9F00EA0F500019003E0012002000DC
:10D430000010DD0082412000020160000D003A0072
:10D44000000178006220B20003003A006100600031
:10D4500015003A000E003700E1806000C308DD00CF
:10D46000800880000030A100010070008008880062
:10D470000D003700E1806000C308DD00F008800087
:10D480000030A10001007000F0088800060037009D
:10D490008F81E90042102000A1462000E0DC290035
:10D4A00008EF0200000000000080FA000000060003
:10D4B0000200FA00F0BF9F0001017800CF80DE007B
:10D4C000EA0F5000E08F580034003E000060010079
:10D4D0000A00370011003700180037001F0037001E
:10D4E000260037002D0037002C0037002B003700B6
:10D4F0002A00370009003700180037006301610077
:10D500004410DD0022088000F1FC2F0001016100C1
:10D5100000017100220888002600370063016100C5
:10D520004410DD0082088000F1FC2F000101610041
:10D5300000017100820888001E003700630161004D
:10D540004410DD0092088000F1FC2F000101610011
:10D550000001710092088800160037006301610025
:10D560004410DD00F2088000F1FC2F000101610091
:10D5700000017100F20888000E00370063016100AD
:10D580004410DD0002098000F1FC2F000101610060
:10D590000001710002098800060037008F81E90050
:10D5A00042102000214A2000E0DC290008EF0200A0
:10D5B000000000000080FA00000006000200FA00EF
:10D5C000F0BF9F00401ADE0005002000E90F500068
:10D5D00003003200EA0F500007003A000300370052
:10D5E000620888007408880009003700D2088800A3
:10D5F000E4088800060037008F81E900421020000F
:10D60000A14F2000E0DC290008EF0200000000002C
:10D610000080FA0000000600E80F5000020034000D
:10D620000000D0007100500000000600800078006B
:10D6300010002000E88F500001003C000000EB00CB
:10D64000000006000200FA00889FBE008A1F7800D2
:10D65000C0BF9F0000047800EC0F540006003600A5
:10D66000E881570042102000E1152000E0DC29008D
:10D6700008EF02000000000008007800E6FF070045
:10D6800000057800E98221004250DD00008044005E
:10D69000900078000110A1000100A00001087800AE
:10D6A00008007800E1FF0700E00F5000040032009E
:10D6B0000A00E8004200DD00008044001000A000E5
:10D6C0004F0578004F04BE000080FA0000000600FD
:10D6D000D1FF07004200DD000080E800C182210088
:10D6E0006100780061006000000006000200FA009E
:10D6F000889FBE00D0BF9F0001047800800478009E
:10D70000EC8F540004003600E681570042102000E0
:10D71000E11920000C00370009007800BEFF070067
:10D720004200DD000080E800C18221006100780035
:10D730000000D1006140600006003A00E681570019
:10D7400032102000211A2000E0DC290008EF02003E
:10D75000000000006148B900EA0F5000E08F580057
:10D760002A003E00006001000A0037000F00370069
:10D7700014003700190037001E003700230037005F
:10D780002200370021003700200037000700370053
:10D79000120037004F44DD002008800000F0A10097
:10D7A00008007000200888001C0037004F44DD008E
:10D7B0008008800000F0A100080070008008880048
:10D7C000160037004F44DD009008800000F0A100F3
:10D7D0000800700090088800100037004F44DD00FA
:10D7E000F008800000F0A10008007000F008880038
:10D7F0000A0037004F44DD000009800000F0A1005E
:10D80000080070000009880004003700E681570016
:10D8100042102000511C2000CBFF37004F04BE00F7
:10D820000080FA00000006008000EB00AFFF370028
:10D8300011002000ADFF37000200FA00F0BF9F008A
:10D84000CF80DE00EA0F5000E08F580018003E0045
:10D85000006001000A0037000C0037000D0037009F
:10D860000F0037001000370011003700100037009C
:10D870000F0037000E0037000300370007003700A5
:10D88000020888001000370043088800320888002A
:10D890000D003700520888000B003700B3088800DD
:10D8A000A208880008003700C20888000600370078
:10D8B0008F81E90042102000D11E2000E0DC290009
:10D8C00008EF0200000000000080FA0000000600DF
:10D8D0002F04B000889FBE008A9FBE008C9FBE00B0
:10D8E0008E1F7800D0A79F00E2A79F00F3A79F009C
:10D8F00081AF9F006000B8006011B800909F9F004A
:10D90000A19F9F00B29F9F00C39F9F000E007800C1
:10D910000F0778006E04B100A1DE2900070009009E
:10D92000311F7800000778005FA69700EC0F5600C3
:10D9300005003600A3FC2F008F814100421020001B
:10D94000211020000E0037000C00780032FF070085
:10D9500080007800C208DD008180E800C2822100DA
:10D96000E28078008100D100E1C0600007003A0049
:10D97000A3FC2F008F814100321020006110200095
:10D98000E0DC290008EF0200000000008FA89700EB
:10D99000E08F500013003200E38F5000110032007E
:10D9A000E68F50000F003200E98F50000D0032006A
:10D9B000E18F400025003200E28F4000230032005A
:10D9C000E38F400021003200E48F40001F0032004E
:10D9D00003FD2F008F81410052102000B110200064
:10D9E000E7FF37006FA19700FFA19700929F9F006C
:10D9F000A39F9F000001EB00B29F9F00C29F9F006A
:10DA000082067800698710000E003700A40020000D
:10DA1000050020006033B8001F989700AF9897006A
:10DA20003F999700CF99970058040200000000002A
:10DA3000909F9F00A19F9F00B29F9F00C39F9F0048
:10DA40008D06E8008E8F5600F0FF3500E80F560077
:10DA5000A1003C008040EB000C0078006FFE070046
:10DA60000FA99700E00F5100880035001F9C970018
:10DA7000AF9C97003F9D9700CF9D970048EE020016
:10DA80000000000090B79F00A1B79F008003EB004B
:10DA9000B7B79F000000EB00C0B79F001FB2970010
:10DAA000AFB297003FB39700CFB397000440E100B7
:10DAB00005C8E10006D0E10007D8E1001F003900E9
:10DAC0001F989700AF9897003F999700CF999700BC
:10DAD000D0AF9F00E1AF9F00F2AF9F0083B79F00E0
:10DAE00048EE0200000000000004BE004FB59700A1
:10DAF0008A05780004F02F00F50F20006033B8008D
:10DB00000800BE000A01BE00580402000000000028
:10DB10005FAA9700EFAA97007FAB97008FB397009B
:10DB20000020E10001A8E10002B0E10003B8E1003B
:10DB300002003E004FB697000600370023FB2F007F
:10DB40008F81410012102000D11120008CFF37007E
:10DB50000C06E8001F989700AF9897003F99970030
:10DB6000CF99970090B79F00A1B79F00B2B79F00D1
:10DB7000C3B79F0048EE0200000000004261DD00D4
:10DB8000A3FB2F008F814100028141001202BE00E1
:10DB9000D4B79F00E5B79F008002EB00F5B79F0068
:10DBA0000003EB0086BF9F000004BE000A002000B7
:10DBB0000B002000F4FF2F00050020006033B800A8
:10DBC0000800BE000A01BE00580402000000000068
:10DBD0005FB29700EFB297007FB397008FBB9700BB
:10DBE00058040200000000001FB29700AFB2970077
:10DBF0003FB39700CFB397000020E10001A8E100F8
:10DC000002B0E10003B8E100D1FF3E001F98970089
:10DC1000AF9897003F999700CF99970090B79F00D2
:10DC2000A1B79F00B2B79F00C3B79F0048EE0200A4
:10DC3000000000000004BE000FBD97008A057800B8
:10DC40005FB29700EFB297007FB397008FBB97004A
:10DC50000800BE000A01BE005804020000000000D7
:10DC60000203BE000002BE001FB09700AFB09700D5
:10DC70003FB19700CFB197007A0502000000000085
:10DC80000205BE000004BE000C0037006FA0970024
:10DC9000FFA09700E10F4000E08F5800050036001C
:10DCA000C3FC2F008F814100121020007112200050
:10DCB00033FF37000286EA000004BE008C007800C3
:10DCC0005FA09700FAFD0700880078005FA097002A
:10DCD000B3FD07008C00370011C0B3000C007800C2
:10DCE000CEFD07008FA89700E08F50007D00350023
:10DCF0001F9C9700AF9C97003F9D9700CF9D97007A
:10DD000048EE020000000000D0B79F00E1B79F007E
:10DD10008003EB00F7B79F000000EB0080BF9F007F
:10DD20005FB29700EFB297007FB397008FBB970069
:10DD30000440E10005C8E10006D0E10007D8E10099
:10DD4000200039001F989700AF9897003F999700DF
:10DD5000CF999700D0AF9F00E1AF9F00F2AF9F0037
:10DD600083B79F0048EE0200000000000004BE00E0
:10DD70000FBD97008A05780004F02F00F5FF2F00F3
:10DD8000F60F2000070020000800BE000A01BE00B8
:10DD900058040200000000005FAA9700EFAA970055
:10DDA0007FAB97008FB397000020E10001A8E1004E
:10DDB00002B0E10003B8E10002003E000FBF97008F
:10DDC0000600370023FB2F008F8141001210200036
:10DDD000A1132000EAFE37000E07E8001F98970005
:10DDE000AF9897003F999700CF999700D0B79F00C1
:10DDF000E1B79F00F2B79F0083BF9F0048EE02008B
:10DE0000000000000001BE004270DD00A1FB2F00F9
:10DE10008F804000008040001006BE000C00BE0055
:10DE20004C040200000000000004BE000005EB00EE
:10DE30008A0578000802BE000A03BE005FB09700A2
:10DE4000EFB097007FB197008FB997007A05020075
:10DE500000000000F4FF2F00F5FF2F006033B80032
:10DE60000400E1000588E1000690E1000798E10068
:10DE7000D9FF3E000800BE000A01BE0090B79F0017
:10DE8000A1B79F00B2B79F00C3B79F001F9C970028
:10DE9000AF9C97003F9D9700CF9D970048EE0200F2
:10DEA000000000000002BE004FB397008603780018
:10DEB0000800BE000A01BE007A0502000000000052
:10DEC0000C02BE004FB49700080378008803780066
:10DED0007A050200000000000205BE000004BE003A
:10DEE000030037000187EA006FA49700FFA49700A2
:10DEF0008E0078005FA097006DFD07000801BE004E
:10DF00005FA09700ADFD07006011B8005FA097000B
:10DF100049FE07004F0778004F06BE004F05BE00C0
:10DF20004F04BE002F04B100000006000200FA00FA
:10DF3000F0BF9F00CF80DE00EA0F5000E08F580056
:10DF40001F003E00006001000A0037000B00370090
:10DF50001000370011003700170037001800370095
:10DF6000170037001600370015003700060037008D
:10DF70000C003700000880000100370030088000E6
:10DF800001002000140037003208800040088000A3
:10DF90000600370050088000F9FF3700A008800015
:10DFA000F7FF3700A2088000B008800080007800EA
:10DFB0000200780008003700C0088000F0FF37003A
:10DFC0008F81E9004210200051212000E0DC29006F
:10DFD00008EF0200000000000080FA0000000600C8
:10DFE0000400FA00E0BF9F00F1BF9F00010178002C
:10DFF000E10F5100040036008F81E900621020001B
:10E00000912220003E0037006FB89700CF80DE00DD
:10E01000EA0F5000E08F580036003E00006001001B
:10E020000A003700120037001900370021003700BE
:10E03000280037002F0037002E0037002D00370052
:10E040002C0037000900370019003700610161001A
:10E0500002014100200880000010A10002007000B1
:10E060002008880005A1A9002800370013A1A900F5
:10E070006101610002014100800880000010A100E0
:10E08000020070008008880011A1A9001F0037005D
:10E090006101610002014100900880000010A100B0
:10E0A000020070009008880013A1A9001700370033
:10E0B00021A1A9006101610002014100F008800076
:10E0C0000010A10002007000F00888001FA1A90044
:10E0D0000E0037006101610002014100000980006B
:10E0E0000010A100020070000009880021A1A90011
:10E0F00006003700E481570042102000112620005E
:10E10000E0DC290008EF0200000000000080FA00B7
:10E11000000006000200FA00F0BF9F000101780035
:10E12000CF80DE00EA0F5000E08F58002F003E0045
:10E13000006001000A0037001000370016003700A9
:10E140001C00370022003700280037002700370066
:10E15000260037002500370008003700150037007B
:10E16000610161004611DD00200880000060A1000F
:10E170000200700020088800220037006101610061
:10E180004611DD00800880000060A10002007000E0
:10E19000800888001B003700610161004611DD0026
:10E1A000900880000060A1000200700090088800C4
:10E1B00014003700610161004611DD00F0088000A5
:10E1C0000060A10002007000F00888000D00370018
:10E1D000610161004611DD00000980000060A100BE
:10E1E0000200700000098800060037008F81E900F6
:10E1F0004210200041292000E0DC290008EF020045
:10E20000000000000080FA00000006000400FA0090
:10E21000889FBE008A1F7800B0BF9F00010578006C
:10E22000C2BF9F0080047800EC8F540004003600C9
:10E23000EA81570042102000812A200007003700A1
:10E240004FBC97000800E900E60F500006003600BA
:10E25000E881570022002000912A2000E0DC2900FC
:10E2600008EF02000000000009007800EAFC070047
:10E270004200DD00C28221000A3178006148B90005
:10E28000EA0F5000E08F58003C003E0000600100A3
:10E290000A003700130037001C0037002400370045
:10E2A0002D003700350037003400370033003700C9
:10E2B000320037001500370027003700670464007C
:10E2C0004C40DD0028058000F1FF280001046400B7
:10E2D00000047400280588008460A9009460A800E8
:10E2E0002A003700670464004C40DD0038058000D8
:10E2F000F1FF280001046400000474003805880060
:10E3000084E0A90094E0A8002000370067046400BE
:10E310004105800080FF2F0000806000080470002D
:10E32000480588008500A9009500A800170037005F
:10E33000670464004C40DD0088058000F1FF280080
:10E340000104640000047400880588008760A90047
:10E350009760A8000D0037006704640091058000F5
:10E3600080FF2F000080600008047000980588007E
:10E370008780A9009780A80004003700EA81570031
:10E3800042102000D12E2000B4FF37004F05780046
:10E390004F04BE000080FA00000006000200FA00F0
:10E3A000F0BF9F00CF80DE00EA0F5000E08F5800E2
:10E3B0002A003E00006001000A0037000F0037000D
:10E3C00014003700190037001E0037002300370003
:10E3D0002200370021003700200037000D003700F1
:10E3E00018003700A00480004300DE0061006000D8
:10E3F0009460A8008460A8001E003700A00480007C
:10E400004700DE006100600094E0A80084E0A800FE
:10E4100018003700A00480004800DE0061006000A2
:10E420009500A8008500A80012003700B004800005
:10E430004B00DE00610060009760A8008760A800C4
:10E440000C003700B00480004C00DE00610060006A
:10E450009780A8008780A800060037008F81E90018
:10E4600042102000F1332000E0DC290008EF020018
:10E47000000000000080FA00000006000200FA0020
:10E48000F0BF9F00CF80DE00EA0F5000E08F580001
:10E490001E003E00006001000A0037000C0037003B
:10E4A0000E00370010003700120037001700370049
:10E4B000160037001500370014003700070037003A
:10E4C0000C003700200480004300DE000B00370002
:10E4D000200480004700DE00080037002004800090
:10E4E0004800DE0005003700300480004B00DE00ED
:10E4F00002003700300480004C00DE006100600044
:10E500000080FA0000000600060037008F81E90055
:10E510004210200011372000E0DC290008EF020043
:10E52000000000000200FA00F0BF9F000101780027
:10E53000CF80DE00EA0F5000E08F580038003E0028
:10E54000006001000A003700110037001A00370090
:10E550002100370028003700310037003000370035
:10E560002F0037002E00370013003700220037003D
:10E57000200480004300DE00610060006101610052
:10E580004311DD00210480000130A10007003700A5
:10E59000200480004700DE0061006000610161002E
:10E5A0004711DD00210480000170A100828070000D
:10E5B0002104880020003700200480004800DE008D
:10E5C00061006000610161004811DD0021048000EC
:10E5D0000180A100F5FF3700300480004B00DE0011
:10E5E00061006000610161004B11DD0031048000B9
:10E5F00001B0A10007003700300480004C00DE00AD
:10E6000061006000610161004C11DD003104800097
:10E6100001C0A1008280700031048800060037002C
:10E620008F81E90042102000613B2000E0DC2900DE
:10E6300008EF0200000000000080FA000000060061
:10E640000200FA00F0BF9F00CF80DE00EA0F50000A
:10E65000E08F58001B003E00006001000A003700F8
:10E660000C0037000E003700100037001200370092
:10E670001400370013003700120037001100370074
:10E68000070037000C0037009460A9008460A900DF
:10E690001200370094E0A90084E0A9000F003700C1
:10E6A0009500A9008500A9000C0037009760A9001B
:10E6B0008760A900090037009780A9008780A9001A
:10E6C000060037008F81E90042102000913F2000B2
:10E6D000E0DC290008EF0200000000000080FA00E2
:10E6E000000006000600FA00889FBE008A9FBE0058
:10E6F0008C9FBE00F0B79F0081067800000578006F
:10E70000EC0F550004003600F28157004210200043
:10E71000210C2000100037000A00780082BF9F0003
:10E7200093BF9F00BCFB0700000678004264DD0039
:10E730000880E800C1822100610278006142620025
:10E740000FB997009FB9970006003A00F281570071
:10E7500022102000610C2000E0DC290008EF0200FC
:10E7600000000000EB822100088445009804780036
:10E770000910A0000900A100090C78000A00780027
:10E7800082BF9F0093BF9F00A8FB07000FB99700AF
:10E790009FB99700E00F5000060032000C00E8001F
:10E7A0004200DD00008045001000A1001820A000FC
:10E7B000020037000920A100090C78007FB0970003
:10E7C00082BF9F0093BF9F009DFF07008D007800D0
:10E7D0000FB997009FB997007FB097003CFC0700E6
:10E7E0008000EB007FB09700FDFD07008000EB008C
:10E7F0007FB0970047FE07004F06BE004F05BE00E2
:10E800004F04BE000080FA00000006000200FA007B
:10E81000F0BF9F00CF80DE00EA0F5000E08F58006D
:10E820001B003E00006001000A0037000B003700AB
:10E830000C0037000D0037000E00370014003700C1
:10E8400013003700120037001100370003003700B3
:10E85000060037002108800007003700810880008B
:10E86000050037009108800003003700F1088000A0
:10E870000100370001098000C408DE00E380600069
:10E8800000042000E28F500007003A000D0037001E
:10E890008F81E9004210200091422000E0DC290035
:10E8A00008EF02000000000000102000E38F50007D
:10E8B0000400320080002000E18F5000010032008F
:10E8C000100020000080FA00000006003600F8006A
:10E8D000809FBE00829FBE00849FBE00869FBE00B8
:10E8E0003400F80000002000A00188000000EB00C8
:10E8F00061C18000010001008460A9003400F900BA
:10E900004F03BE004F02BE004F01BE004F00BE00CD
:10E910003600F900004006003600F800809FBE0077
:10E92000829FBE00849FBE00869FBE003400F80018
:10E9300000002000A001880084E0A9001000200051
:10E9400081C18000010001003400F9004F03BE00C6
:10E950004F02BE004F01BE004F00BE003600F9005E
:10E96000004006003600F800809FBE00829FBE0077
:10E97000849FBE00869FBE003400F8000000200087
:10E98000A00188008500A90090C180006600600099
:10E99000E60F500003003A009000200081C1800083
:10E9A0000200370020002000A1C18000010001000A
:10E9B0003400F9004F03BE004F02BE004F01BE00FD
:10E9C0004F00BE003600F900004006003600F80097
:10E9D000809FBE00829FBE00849FBE00869FBE00B7
:10E9E0003400F80000002000A00188008760A90022
:10E9F00030002000C1C18000010001003400F90096
:10EA00004F03BE004F02BE004F01BE004F00BE00CC
:10EA10003600F900004006003600F800809FBE0076
:10EA2000829FBE00849FBE00869FBE003400F80017
:10EA300000002000A00188008780A900D0C18000CC
:10EA400066006000E60F500003003A00A0002000BE
:10EA5000C1C180000200370040002000E1C18000F9
:10EA6000010001003400F9004F03BE004F02BE0058
:10EA70004F01BE004F00BE003600F9000040060006
:10EA800090089000E001900001814000630179004E
:10EA90008100E900110898000200780000000600DB
:10EAA0000200FA00889FBE0080047800010478000C
:10EAB000E08F540003003A000000280000006400CA
:10EAC0005C00370000002400E00F540056003200C4
:10EAD0000802780001003D000802EA000900780001
:10EAE000E08F540001003D000900EA00CF80DE0005
:10EAF00066815700811F7800110009004488D80002
:10EB000001097800CF0078005FB99700030020006A
:10EB1000C011DD0002002000809FBE00110009002E
:10EB20004499D800000178004F00BE0080007800B2
:10EB3000020078000181CF00E00F51000300320095
:10EB40000402200002025200040037000082CF00BD
:10EB5000E00F52000100320070021200EC0252007D
:10EB600009003B00C2282000030020004C040200E2
:10EB700000000000440BDD004C00DE0000007300CC
:10EB8000CC88DE00240037001200200003002000A3
:10EB9000040378000603E90003003300020141008A
:10EBA00083814900FBFF370002005000838058003A
:10EBB000680252000402E900030033008180D100A2
:10EBC0000080D300FBFF3700FF0060004580DE00BF
:10EBD000C32ADD000501400002004100C6F92800FB
:10EBE0006600780003022000018251000482B9000F
:10EBF0000201E80002014100660079000180B900CD
:10EC00000000420081804A00811F78001100090045
:10EC10004308D800CF007800E00F540002003D0008
:10EC20000100280000805000E08F540001003C00EB
:10EC30000000EA004F04BE000080FA000000060059
:10EC4000889FBE008A9FBE008C1F7800000178005C
:10EC5000E00F51000C003D0001002C00810F51001D
:10EC600003003D00000028000000410004003700C0
:10EC700010002800810F51002C0032000200EA0031
:10EC80001A0020000B00370001002400810F510002
:10EC90000300340000002800020050000400370088
:10ECA000F0FF2700810F51002000320002007800A1
:10ECB0000005EB00C780DE0000017800F207B2001B
:10ECC00081814000A0E92800E08579000C0820003F
:10ECD000020656008100E8008180400060807800D4
:10ECE000CF80DE00CF91DE004C0402000000000067
:10ECF0000004BE006162B9006159B9000400BE00A1
:10ED00004C04020000000000080040008980480018
:10ED10004909DD004700DE0000007100C788DE0001
:10ED2000E00F5500010032000000EA004F067800B5
:10ED30004F05BE004F04BE00000006000100240085
:10ED400001004000BEFF3700010024000100370031
:10ED5000C288DE00808F5000FDFF3C00000178007B
:10ED60000000EB0007003700808140000080D100E8
:10ED7000830F5100020035000301510001004000E3
:10ED8000C288DE00E08F5000F7FF3A000000060066
:10ED9000889FBE008A9FBE00800278000100780034
:10EDA0008001EB004A0020005900200018003700C5
:10EDB0000A01B800811F7800110009004999D800A4
:10EDC000CF0078000001EB00820178000D003700D1
:10EDD0008203410087834200170378000402420047
:10EDE0000482420014047800880553004240A900C0
:10EDF00003003400880B7800060A78001300200016
:10EE00000201E80000024100810F5200F0FF3900CA
:10EE1000E10F5000E6FF3E00E08F5100E9FF3A00AD
:10EE20004F05BE004F04BE0000000600889FBE00D4
:10EE30008A1F7800000478000800780010FF07009F
:10EE400000057800080078000DFF070080047800B6
:10EE5000080078000AFF07008000EB000700370079
:10EE6000C80190000A0145000982440064B179009C
:10EE70000A05E8008904E8008100E800808F50005E
:10EE8000F7FF39004F0578004F04BE000000060070
:10EE9000889FBE008A1F7800000478000800780070
:10EEA000F7FE07008004780008007800F4FE0700F1
:10EEB0000005780008007800F1FE07008000EB00F4
:10EEC0000A05450005003700C8019000098144008B
:10EED0006AB179008904E8008100E800808F500061
:10EEE000F9FF39004F0578004F04BE00000006000E
:10EEF000889FBE008A9FBE0000047800080078004A
:10EF0000DFFE07000005780008007800DCFE07003F
:10EF10008004780008007800D9FE0700800578009A
:10EF200008007800D6FE0700C80090008B854500D9
:10EF300061817D008000EB0009003700C80290006D
:10EF40008A01450083814200098244000482420014
:10EF5000940941000A05E8008904E8008100E800FE
:10EF6000808F5000F5FF39004F05BE004F04BE00F2
:10EF700000000600889FBE008A9FBE000004780043
:10EF800008007800BEFE07008005780008007800C1
:10EF9000BBFE07000005780008007800B8FE0700F7
:10EFA0008004780008007800B5FE07008000EB00C0
:10EFB0000D003700480190008B814500830141001E
:10EFC00009824400040241008A0245000501410013
:10EFD00014027800920942008B05E8000A05E80057
:10EFE0008904E8008100E800808F5000F1FF3900BB
:10EFF0004F05BE004F04BE0000000600889FBE0003
:10F000008A9FBE0000047800080078009CFE07007C
:10F01000800578000800780099FE07000005780058
:10F020000800780096FE0700800478000800780049
:10F0300093FE07008000EB000D00370048019000B0
:10F040008B814500830141000A0245000402410012
:10F05000898244000501410014027800920952009F
:10F060008B05E8000A05E8008904E8008100E80053
:10F07000808F5000F1FF39004F05BE004F04BE00E5
:10F0800000000600889FBE008A9FBE000004780032
:10F09000080078007AFE07008005780008007800F4
:10F0A00077FE0700000578000800780074FE07006E
:10F0B000800478000800780071FE07008000EB00F3
:10F0C0000C003700480290008B8245008981440083
:10F0D0000A014500E4817900640179000299B900D0
:10F0E00002B27A008B05E8000A05E8008904E8000E
:10F0F0008100E800808F5000F2FF39004F05BE000C
:10F100004F04BE0000000600889FBE008A9FBE001C
:10F110008C9FBE008E1F78000004780008007800E5
:10F1200057FE0700800578000800780054FE0700AD
:10F13000000578000800780051FE07008004780080
:10F14000080078004EFE0700800678000006EB00FD
:10F150001C003700C80090000A00450061007800DC
:10F160000981440061017900CF91DE00E00F510078
:10F17000E08F59000B0032000A05E8008904E8001E
:10F180000B8745000E874000CF80DE007A06020024
:10F1900000000000000F78008B05E8000C06E80076
:10F1A0000800370023002000730498007001440019
:10F1B000710029000800780060CE02000000000005
:10F1C000020037008D0F5600E2FF39004F0778002C
:10F1D0004F06BE004F05BE004F04BE0000000600F3
:10F1E000889FBE008A9FBE00000478000800780057
:10F1F00023FE0700800578000800780020FE070045
:10F2000000057800080078001DFE070080047800E3
:10F21000080078001AFE07008000EB000F0037009E
:10F22000480190008A014500E28179000A05E80062
:10F23000898244008904E8000B82450004024100F1
:10F2400062817A00830F51000100340003017800CD
:10F25000020A78008B05E8008100E800808F5000EA
:10F26000EFFF39004F05BE004F04BE00000006004E
:10F27000889FBE008A9FBE000004780008007800C6
:10F28000FFFD07008005780008007800FCFD0700FE
:10F290000005780008007800F9FD07008004780078
:10F2A00008007800F6FD07008000EB000F00370033
:10F2B000480190008A014500E28179000A05E800D2
:10F2C000898244008904E8000B8245000402410061
:10F2D00062817A00830F510001003D000301780034
:10F2E000020A78008B05E8008100E800808F50005A
:10F2F000EFFF39004F05BE004F04BE0000000600BE
:10F30000889FBE008A9FBE008C1F78000004780092
:10F3100008007800DAFD0700000678000800780091
:10F32000D7FD07008005780008007800D4FD0700AD
:10F330000005780008007800D1FD070080047800FF
:10F3400008007800CEFD07008001EB0014003700B4
:10F35000C80090000B814500610279008B05E80030
:10F360000A014500E10279000A05E800098144002C
:10F37000610179008904E800820F520004003C001A
:10F3800005017800840F510001003D000401780060
:10F390000C02460082307A000C06E8008301E80087
:10F3A000808F5100EAFF39004F0678004F05BE00FC
:10F3B0004F04BE0000000600889FBE008A9FBE006A
:10F3C0008C9FBE000004780008007800ACFD0700A8
:10F3D0008004780008007800A9FD07008006780006
:10F3E00008007800A6FD0700000678004805900098
:10F3F00008007800A2FD070000017800020141002A
:10F40000EA057900080078009DFD070000057800F6
:10F4100000022000808F550005003C000D0378009D
:10F420008C0078008003EB006011B8000F003700FB
:10F43000480090008984440089044000800CEB005F
:10F440001400370001804000650278008100E80068
:10F4500006004300650078000603E8000482B90056
:10F460000201420083814A008703E800C80290003D
:10F470008A8F5300F3FF3900898444008B05E9002B
:10F48000030033008381D1000281D300FBFF3700EA
:10F4900082B27C004F06BE004F05BE004F04BE0086
:10F4A00000000600889FBE008A9FBE008C1F780067
:10F4B000000478000800780071FD070080047800DF
:10F4C000080078006EFD070000067800080078004C
:10F4D0006BFD0700800578000800780068FD0700D4
:10F4E000000578000800780065FD0700000178003D
:10F4F000E00F5100250032004802900009804400CE
:10F50000E40178000903E8006118B9000C06460020
:10F5100003327E008B8445004802900003B27C00D9
:10F52000170020001000370086014300E4817900B5
:10F530000603E8000C024200948F510001003D00D8
:10F54000030A78004802900009024200948F51009B
:10F5500001003400030A7800611AB900000042007B
:10F5600081804A008703E80048029000828F5300A0
:10F57000EDFF39000A0545000A054200030020009E
:10F580007A06020000000000000D78004F067800A7
:10F590004F05BE004F04BE0000000600889FBE005D
:10F5A0008A9FBE00000478000800780034FD070040
:10F5B000800578000800780031FD0700000578001C
:10F5C000080078002EFD070080047800080078000D
:10F5D0002BFD070000027800E00F520016003200F9
:10F5E0000B0178008000EB0005002800F0FF2700E9
:10F5F0000A054500898444004803900082014100C7
:10F60000E68179000201E800808F510002003D0090
:10F6100001337D0003007800858F51000300340022
:10F62000C802900081B27C00830278008100E8006B
:10F63000848F5000F0FF39004F05BE004F04BE001C
:10F6400000000600889FBE000004780008007800D3
:10F650000BFD0700800478000800780008FD070013
:10F660008000780089844400480090000900400030
:10F67000C7FD07004F04BE0000000600E8874700F2
:10F68000889FBE008A9FBE008C9FBE008E1F7800A0
:10F69000000578000A007800F9FC070000077800F0
:10F6A0000A007800F6FC0700800678000A0078005F
:10F6B000F3FC0700000678000A007800F0FC070061
:10F6C000800578000A007800EDFC070080037800D0
:10F6D0000003EB002A003700CA0090000D804600AE
:10F6E000610278000C004600610078000B81450043
:10F6F00061047900CFC4DE00E00F5400E08F5C00AD
:10F70000170032008D06E8000C06E8008B05E800C3
:10F710000E01470002814000E2B79F00CF80DE006B
:10F72000CFA2DE000401BE00F6B79F0087BF9F0096
:10F730004C040200000000000801BE007A0602002E
:10F74000000000006FB19700000978000E07E80084
:10F750007FB397000603E8008FBB970008003700CF
:10F7600023002000730598007001450071002900F6
:10F770000A00780060CE020000000000020037009E
:10F78000870F5300D4FF39004F0778004F06BE00A3
:10F790004F05BE004F04BE008F00B1000000060000
:10F7A000889FBE008A9FBE008C9FBE008E1F78007F
:10F7B0000004780008007800B1FC0700800578009C
:10F7C00008007800AEFC070000057800080078000B
:10F7D000ABFC07008004780008007800A8FC070054
:10F7E000000778000006EB000C003700C806900008
:10F7F0000A0045006D0078000A05E8008980440091
:10F80000ED8078008904E800A5FC07008B804500A6
:10F8100080B678008B05E8000C06E8008E0F5600D5
:10F82000F2FF39004F0778004F06BE004F05BE00BB
:10F830004F04BE0000000600889FBE008A9FBE00E5
:10F840008C9FBE0000047800080078008CFC070044
:10F85000000578000800780089FC07008004780023
:10F860000800780086FC0700000678008005EB00A1
:10F8700009003700C8069000098044006D00780038
:10F880008904E800EEFC07008A00450080B6780095
:10F890000A05E8008B05E8008C8F5500F5FF39005C
:10F8A0004F06BE004F05BE004F04BE00000006001C
:10F8B000889FBE008A9FBE008C9FBE000004780017
:10F8C000080078006EFC070000057800080078004A
:10F8D0006BFC0700800478000800780068FC0700D3
:10F8E000000678008005EB0009003700C80690008C
:10F8F000098044006D0078008904E8000FFD0700CE
:10F900008A00450080B678000A05E8008B05E8000B
:10F910008C8F5500F5FF39004F06BE004F05BE0025
:10F920004F04BE0000000600EE874700889FBE001F
:10F930008A9FBE008C9FBE008E1F78000007780053
:10F940000E0078004EFC0700E0B79F000E00780024
:10F950004BFC0700000478000E00780048FC07000C
:10F96000CE04900088004400698678000804E8000E
:10F970000804440069037C0000004000690478002A
:10F980000800780086BF9F00ECFC070000057800A7
:10F9900008007800AAFC070000047800EFB0970088
:10F9A0000180400000804400D0B79F00CFE6DE0019
:10F9B000CFD5DE000A01BE000C00BE004C040200E0
:10F9C00000000000B0B79F00C1B79F000FBB9700B9
:10F9D000CFB3DE00CFC4DE000801BE000600BE00CB
:10F9E00086BF9F00F7B79F004C0402000000000094
:10F9F0000002BE003FB09700CFB097000402500055
:10FA000085825800C128DD004F22DE00048270008C
:10FA1000CFAADE005FB1970004097800EFB197002C
:10FA20000300E8004E079000000040000007470078
:10FA30000A01BE000FBB9700FFB397000600BE008F
:10FA40004C040200000000000005BE000801BE00DA
:10FA50000C00BE004C040200000000000A00400040
:10FA60008B8048004109DD004F00DE00000071007E
:10FA7000CF88DE00000F78004F0778004F06BE00E9
:10FA80004F05BE004F04BE00EF00B10000000600AD
:10FA9000889FBE008A9FBE008C9FBE000004780035
:10FAA00008007800F6FB07000005780008007800E1
:10FAB000F3FB07008004780008007800F0FB0700E3
:10FAC000000678008005EB0009003700C8069000AA
:10FAD000098044006D0078008904E8009AFC070062
:10FAE0008A00450080B678000A05E8008B05E8002A
:10FAF0008C8F5500F5FF39004F06BE004F05BE0044
:10FB00004F04BE0000000600889FBE008A9FBE0012
:10FB10008004780009007800D9FB07000004780011
:10FB200009007800D6FB070000057800090078007E
:10FB3000D3FB07008005780009007800D0FB0700A0
:10FB400080017800490190008B854500E2837D00AB
:10FB50008000EB00070037008100E800838F500031
:10FB60000400360008044400080141000009EB00CD
:10FB70004F0037000A80400000004000620078001B
:10FB8000E00F5000F4FF3A00010078000B0037004E
:10FB90008100E800838F500008003600080444000C
:10FBA000E00F50003A0032000000E900870F5000DB
:10FBB000370039000000D1003C0037000A824000C5
:10FBC0000402420062027A00E00F5200F0FF3200AD
:10FBD0000003EB000600780006027800840278003B
:10FBE000030037008502E800838F52000B003100CC
:10FBF00081844200809FBE00110009008384D800E8
:10FC0000810478004F00BE008A8444008984440047
:10FC1000E2847C00E08F5400F2FF3A0084845200BA
:10FC2000808F540003003400048242000483D1001A
:10FC300009007800838F5200050039001100370059
:10FC40000402E800830F5200020039000D00370063
:10FC50000502780081024200809FBE001100090069
:10FC60008382D800810278004F00BE008A82420061
:10FC700085824200E2827A00E08F5200D7FF3A008C
:10FC8000EFFF370008044400870F500003003D00D9
:10FC900008044100008CEB000500370081004300A0
:10FCA000110009008380D8008000FD0000317C0035
:10FCB0004F05BE004F04BE000000060040CE880085
:10FCC000000006005025260041CE80000088B900C3
:10FCD000926123000000410040CE88000000060031
:10FCE000889FBE008A9FBE008C1F780000047800A9
:10FCF0000800780062FB07008004780008007800A4
:10FD00005FFB0700800578000005EB000700370067
:10FD1000098044004806900000064600E9FF0700FD
:10FD2000000E78008904E8000A05E8008B0F5500F2
:10FD3000F7FF39004F0678004F05BE004F04BE00A4
:10FD400000000600AA24AB000D00320032828000C1
:10FD50009240900000C8B30080CF500007003A00E6
:10FD6000808280009040900040C8B30080CF500057
:10FD700002003A006840400010419800AA24A900FF
:10FD80000008200050248800000006000103210024
:10FD90009140780000C8B30080CF50002F003A0097
:10FDA00000CCB3005CF0B70033D0BF00E24F50008E
:10FDB00008003200E34F500017003200E14F5000BE
:10FDC00025003A0000122100D08288002001200086
:10FDD0001D00370032D0BF000080FB000000400053
:10FDE000E11B2100E1007800D1828800D0828000F0
:10FDF000801F7800204090005EF0B7004F00780030
:10FE0000D0828000801F7800304090005FF0B70003
:10FE10004F0078000000060032D0BF00E24F5000D3
:10FE20000B003E0032D0BF000080FB00000040000D
:10FE3000011C2100E1007800D1828800D08280007E
:10FE4000104078000080FB00F0828800000006006F
:10FE50005C70EF00000006005C70EF000000060020
:10FE60003870EF003970EF0030D0BF007F006000C5
:10FE7000E10F50000B003200E20F50000B00320087
:10FE8000E00F50001B003A005CF0A8003810A800FA
:10FE900010848000E10F500016003A003830A800AE
:10FEA000140037005CF0A800120037005CF0A800D6
:10FEB00034D0BF000500330034D0BF006F006000B5
:10FEC00000004000A10421000400370034D0BF002E
:10FED0006F00600000004000010521006100780013
:10FEE00010409000640060000200320010C0B300B7
:10FEF00038F0B7005CF0AB00050032008003210051
:10FF0000D08288005C10A80020C0B3005EF0B7006B
:10FF100000000600F082800081C0B300E70F5000AF
:10FF20000A003E00F182800056D0BF0002003A0075
:10FF300010C0B3000400370056D0BF00E14F50009E
:10FF400002003A0020C0B30056F0B7000180FB0069
:10FF50005E30B50080828000014878008003210077
:10FF6000408388005C10AB00070032000F003700B0
:10FF7000D08280004283800030597800428388001C
:10FF8000D08288008140E900E0CF5000F8FF3A00BD
:10FF900000000600D0828000428380003059780043
:10FFA00042838800D08288008140E900E0CF500081
:10FFB000F8FF3A0000000600881F78008082800069
:10FFC000100478004E44DE00614464005050AA00E2
:10FFD00000828000E80F50000A003A0032D0BF00D3
:10FFE0000080FB00B0248800B0248000E00F5000A7
:10FFF0000200320000012000010037004000200014
:020000040001F9
:100000000082880058D0BF00E14F500011003A0034
:10001000800321008182800090009800BDFF0700CE
:10002000610521009140780080828000E2CF50007D
:1000300002003A0041C8B3000400370081CCB3008D
:10004000E04F54000100320081C8B3001140980015
:100050001200370062D0BF000F003B0065D0BF0028
:100060000080FB006106210091407800C808DD0097
:10007000008070000700320065D0BF000080FB00E8
:100080006106210091407800C808DD000080700002
:100090000000010062F0A9005870EF004F047800E2
:1000A000000006000080FB000181FB000000400012
:1000B000000141004311DD00030021000301410064
:1000C00012F0A100E0CF500002003A00A10421008C
:1000D00001003700010521008230780012E0A10004
:1000E0006401410012E0A000000006000001EB00E6
:1000F00022848800820078004007200008ED02007A
:10010000000000008284A900000120000024880073
:10011000000006008284A80000012000502488000E
:1001200010002000208488000001EB008000EB001C
:100130005007200008ED0400000000000200FA0053
:10014000881F780032D0BF00E14F50000B003A000A
:1001500030D0BF007F40600008003A005CF0A8008B
:1001600031D0BF00E34F500003003A0010002000E0
:1001700010848800010037008230EF0032D0BF00C9
:100180008E003A0030D0BF007F406000E24F500048
:100190008A003A0034D0BF006F4060008700320010
:1001A00034D0BF006F006000E20F500083003C00BD
:1001B0000182800000022000808F50007F003A0002
:1001C0005CF0A80034D0BF000A00330034D0BF0078
:1001D0006F00600000004000A1042100E1007800F1
:1001E000E1BF9F0034D0BF006F00600021072100F5
:1001F0000900370034D0BF006F00600000004000ED
:1002000001052100E1007800E1BF9F0034D0BF006C
:100210006F006000E10621006144780061406400E5
:1002200004003A004FF897000024A100C0FF9F008F
:1002300003003700CFF897000124A000C1FF9F0002
:1002400034D0BF000500330034D0BF006F00600021
:1002500000004000A10421000400370034D0BF009A
:100260006F00600000004000010521006FB9970099
:100270008230780031D0BF00E34F500018003A00C0
:100280006FB897008000EB00908F10000E003D00CB
:1002900034D0BF00050033004103210091407800B5
:1002A000EF80600022072100040037004103210095
:1002B00091407800EF806000E206210062C0780083
:1002C0000014A00000F17800EFB8970011419000F1
:1002D00040C8B300004071009040980037003700DC
:1002E0004FF997000224A200C2FF9F00EFB89700C9
:1002F000114090000001EB00910F110008003D003B
:100300000074A1000064A00090409800220020002A
:100310005000200008ED020000000000020037003D
:100320000064A000904098004FF897000024A200BD
:10033000C0FF9F006244640006003A006FB8970057
:10034000024028001001610001002800810F5100C7
:1003500017003A0034D0BF000500330041032100EC
:1003600091407800EF8060002207210004003700F0
:100370004103210091407800EF806000E2062100F7
:1003800062C078000014A10000F17800EFB8970077
:1003900011409000B043B20090409800220020002D
:1003A0005000200008ED02000000000003003700AC
:1003B00090409000B143B200114098004F04780083
:1003C0000080FA00000006005CF0A800AC24EF00FA
:1003D000AE24EF000040EB00020021008081FB0012
:1003E00001002100C219DD00830141008009EB00FA
:1003F000B31178000040E800EB4F5000F7FF3600E3
:100400009424A8004470EF009424A9006880400060
:1004100080828800318288004182880032D0BF000B
:1004200042F0B70042D0BF0002003A0000012000B5
:1004300006003700120020002104210010002000D7
:1004400008ED020000000000000220000082880089
:100450000000060030D0BF000046B20035003A0070
:1004600031D0BF000080FB0001002000EB0F5000E6
:10047000E08F58002F003E0000600100130037009D
:10048000130037002B003700110037002900370018
:100490000600370009003700210037000900370047
:1004A000070037000B003700140037005CF0A8008D
:1004B00080002000008288000000060033FE370024
:1004C000C1FF3700200421000600370064FE37001A
:1004D0001AFF370034D0BF000080FB004104210028
:1004E00001004000D08288005C10A80010C0B3005A
:1004F0005EF0B7005CF0A800000006005CF0A80009
:1005000034D0BF000080FB0041042100821F78002E
:1005100022032100927078004F017800000006004D
:100520000001EB008000EB002000200008ED02003D
:1005300000000000000006009EC0A9008EA4EF008D
:100540008AA4EF00AA24EF00AC24EF00AE24EF0051
:100550002000200030258800A824EF008644A90050
:10056000F009200080248800602488008804A80006
:10057000010021004808DE00C02488000040EB0094
:100580000081FB004211DD00028140000009EB0008
:10059000321178000040E800EB4F5000F8FF3600C1
:1005A0009424A8009624EF0094A4A9009424A90000
:1005B0008000200009003700502488005C70EF00A4
:1005C0006270EF0031062100914078006370EF0007
:1005D00041062100914078006470EF0051248000B2
:1005E000E8806000F4FF3A0010002000C08388001B
:1005F000D0838800E1838800F1838800218488000B
:100600000140780005052100A40421000081FB00C1
:100610008201410003834200000BEB008301420092
:100620008009EB00E3062100817179002307210096
:10063000817179000040E800E24F5000F3FF36007E
:100640008000210080828800D00020005025880092
:10065000000321001080880080C0B30000F0B700C4
:1006600040C8B30001F0B7004270EF004030EF0027
:1006700000000600C0838000E00F500024003A0014
:1006800011002000C1838800D0838000E00F50005B
:100690001F003A00D18388008205210012417800B2
:1006A000E24F510006003A008182800080487800C5
:1006B00080CCB3008182800090409800000006004A
:1006C0008205210012417800E14F510010003A00EC
:1006D0000084880080C0B300328280000049780026
:1006E00034828000030321001302980042C8B30043
:1006F000124298000184880041828000804878007E
:10070000418280009300980000C8B3009040980098
:1007100000000600308280009040780063D0BF0067
:100720000080FB0042062100124178004811DD00E4
:10073000000071000181FB00800F510003003600B2
:10074000310621009140780064D0BF0063D0BF0023
:100750000080FB0042062100124178004811DD00B4
:10076000000071008181FB0003005000320621006F
:100770001241780063F0B7004800DE004206210015
:100780001241780064F0B7000040EB00160037001B
:1007900002062100124178000281FB0013062100AD
:1007A00093417800C819DD000082FB0002817100CE
:1007B0008303210063597A000306210093417800E6
:1007C0000001FD0060F0B7000001FD004811DE00EF
:1007D00013062100934178000001FD0061F0B7008D
:1007E0000001FD000040E800814F5000E8FF3900A3
:1007F00063D0BF000080FB004106210091407800DB
:10080000C808DD0000807000418280000E003200C8
:1008100080C0B300804878004082800081032100BE
:100820001100980001002400328280009280600054
:1008300002003A0081CCB3000100370081C8B30048
:10084000114098000000060080C0B3008048780086
:1008500041828000000321009000980040C8B3004E
:100860009040980065D0BF000080FB006106210029
:1008700091407800C808DD00008070000700320059
:1008800065D0BF000080FB00610621009140780028
:10089000C808DD00008070000000010062F0A900BF
:1008A000B0838000E00F500001003A0071FF0700A4
:1008B0000000060058D0BF00E24F500001003A008F
:1008C00094FF37005870EF0000848000E00F500064
:1008D00009003A0080C0B30041828000804878005F
:1008E000418280000003210090009800C0C8B3003E
:1008F00090409800000006008030EF0000000600E5
:100900007C30EF007E30EF0058D0BF00E24F500047
:1009100005003A0080C0B300418280008048780022
:10092000418280001200370036D0BF000080FB00FB
:100930007103210091407800C808DD00008070003C
:10094000F2828000820F50000700310036D0BF00D5
:100950000080FB007103210091407800C808DD0091
:1009600000807000F08288006AFD070081828000AC
:10097000800321009000980080CCB3009040980044
:100980000000060094A4A9005CF0AB0017003A0038
:1009900062D0BF0009003B0020C0B30058F0B70090
:1009A000F0838000E00F500001003A00D4FF070000
:1009B0007A30EF007830EF000000060080C0B3000E
:1009C000418280008048780041828000000321003D
:1009D00090009800C0C8B300904098006840500054
:1009E00081828000904098000000060030D0BF0057
:1009F0000C003B0010C0B30058F0B700E08380004B
:100A0000E00F500001003A00BDFF07007A30EF0010
:100A10007830EF00B0838000E00F500011003A0002
:100A200014FF370020C0B30058F0B70080C0B300F7
:100A300041828000804878004182800000032100CC
:100A40009000980040C8B300904098007A30EF00C2
:100A50007830EF00B0838000E00F500001003A00D2
:100A600004FF070000000600881F78005670EF00A2
:100A70000004EB00B8838800E8838800F8838800CE
:100A8000088488000800780058F0B7008182800050
:100A9000114090000074A1009040980001052100D1
:100AA0001124A20082828000124090000074A100F4
:100AB000104198001124A200418280001140900052
:100AC0000074A10090409800080078005CF0B70026
:100AD000F88288000800780062F0B70063D0BF0099
:100AE0000800780063F0B70064D0BF000004FD0088
:100AF00064F0B7000004FD0056FE0700080178000E
:100B0000820078003000200008ED020000000000A4
:100B10009CFF07004F04780000000600D0C2B3001D
:100B200086F0B7006CD0BF00B00FB20020003A00D2
:100B3000C1062100914078008181FB00C219DE00CE
:100B40004219DD0004002100840041003182880048
:100B5000418288004850AA006402790002C0230044
:100B60000202620002402300820F52000F003A008E
:100B7000910290000082FB00020321009542780060
:100B800005717A00110290000402E80094009800B8
:100B90000040E800E74F5000F5FF3600C219DD00C5
:100BA0002000210002B07900AFFF370041FF37007D
:100BB0006CD0BF00B00FB200E80F500001003A0047
:100BC000FDFC070000000600889FBE008A1F780019
:100BD00000447800814478000985FB0068006500C6
:100BE000030032008040EB00084078002DFD070034
:100BF000640565000300320011C0B30008407800AE
:100C000028FD07000884FB0008044400A04A2000D7
:100C100009707C004F0578004F04BE0000000600FC
:100C2000E04F50000C003A0080C0B30041828000C9
:100C300080487800418280000003210090009800E5
:100C4000C0C8B30090409800684050008182800086
:100C500090409800000006008180FB000080FB00AF
:100C600000004000008040004300DD00040021003F
:100C7000040140009241900041C8B30081C171005D
:100C800013419800640040000400400010419000AF
:100C900081407100114098000000060080427800F9
:100CA0000582FB00E0CF5000030032000402420046
:100CB000000521000200370004024200A0042100C8
:100CC00060007A00E00F500015003200120098001A
:100CD00003487800104190000244B200124098008E
:100CE0009041900082C8B30002C171001240980088
:100CF0000581FB00E0CF50000500320002014100F9
:100D000001052100010141001224A200000006009B
:100D100002014100A1042100010141001224A200AE
:100D20000000060094A4AB00180032000080FB0015
:100D30000000400001052100E10278001501BE001D
:100D4000040420000201620003002000828ABE0029
:100D5000E10278000204200003002000951A6900D7
:100D600095926900010140001224A200E10178007F
:100D7000134190000244B20092419800E1007800D3
:100D80001140900004406800904098000000060068
:100D90000000EB00A0248800602488000082880006
:100DA0000000060000828000E00F500010003A00B2
:100DB000A0248800602488002100200031258800BC
:100DC000402588008644A900F0092000802488007E
:100DD000602488009EC0A800010037009404A80089
:100DE0009404AB00FDFF3200100020000082880058
:100DF00000000600627E2400F10F200012C860008F
:100E00001241900012409800827E2400928160007E
:100E1000234098001241900032409800A27E2400A6
:100E2000928060004140980012419000524098002A
:100E3000917F24009140780061409800A17F2400B8
:100E40009140780071409800B17F24009140780073
:100E500001489800C17F2400914078001148980013
:100E6000C17E24009140780021489800D17E240062
:100E70009140780031489800E17E2400914078004C
:100E800041489800F17E2400914078005148980034
:100E9000017F24009140780061489800117F240070
:100EA0009140780071489800417F2400914078007B
:100EB00001509800517F2400914078001150980013
:100EC000317F24009140780021509800717F2400E8
:100ED0009140780031509800817F24009140780043
:100EE0004150980000000600889FBE008A9FBE0007
:100EF0008C9FBE000004BE000C4020000D002000AE
:100F00000006460081864E00FAFF2F00FB0F2000EE
:100F1000080037000800BE0064C6020000000000A0
:100F20008A0F50008B8F580007003A00620444007B
:100F3000E0844C008C0F54008D8F5C00F5FF39006D
:100F40000000EB0001003700100020004F06BE003B
:100F50004F05BE004F04BE00000006000001EB007C
:100F60001102210000012000DAED02000000000063
:100F700081012000607E2400E6ED020000000000F8
:100F800022EE020000000000800078001000200027
:100F9000E27F2400928F5000010032000000EB003D
:100FA000000006002E00FA0023FD2F008F81410073
:100FB000D2022000AEC60200000000001000200097
:100FC0009FA89700E38F5000010032000000EB0063
:100FD0000080FA00000006001600FA00889FBE009C
:100FE0008A9FBE007E044000E08448000A40200042
:100FF0000B0020000005450081854D000A003700E8
:10100000FE815700520120000800BE00AEC602005B
:10101000000000000FE897006100600006003A0041
:101020006E044400E0844C008A0F54008B8F5C00F7
:10103000F3FF39006044B8000800BE004F05BE0051
:101040004F04BE000080FA00000006001600FA00FF
:10105000889FBE008A9FBE008C1F78000006780023
:101060000205BE008C017800D20220000A00BE00FA
:10107000AEC60200000000000C6890000040E800CE
:10108000006E98007E044500E0844D000040200082
:10109000010020000A0540008B854800CA00370087
:1010A00003FE2F008F814100520120000800BE0086
:1010B000AEC6020000000000CC6090006FE0970018
:1010C00000C0700040669800DC6090007FE09700F0
:1010D00000C0700050669800EC6090000FE8970028
:1010E00000C0700060669800FC6090001FE89700E8
:1010F00000C0700070669800CFF097008180FB0000
:101100002C6190000281FB003C6090004800DD00F3
:101110000200700000804000206698004800DE0059
:1011200030669800BFF097008180FB000C61900052
:101130000281FB001C6090004800DD00020070008E
:1011400000804000006698004800DE0010669800AD
:10115000AFF097008180FB006C5990000281FB008A
:101160007C5890004800DD000200700000804000C4
:10117000605E98004800DE00705E98009FF0970067
:101180008180FB004C5990000281FB005C5890006C
:101190004800DD000200700000804000405E9800C2
:1011A0004800DE00505E98008FF097008180FB00C1
:1011B0002C5990000281FB003C5890004800DD0053
:1011C0000200700000804000205E98004800DE00B1
:1011D000305E9800FFE897008180FB000C5990007A
:1011E0000281FB001C5890004800DD0002007000E6
:1011F00000804000005E98004800DE00105E98000D
:10120000EFE897008180FB006C5190000281FB00A9
:101210007C5090004800DD0002007000008040001B
:10122000605698004800DE0070569800DFE897008E
:101230008180FB004C5190000281FB005C509000CB
:101240004800DD0002007000008040004056980019
:101250004800DE0050569800CFE897008180FB00E0
:101260002C5190000281FB003C5090004800DD00B2
:101270000200700000804000205698004800DE0008
:1012800030569800BFE897008180FB000C51900019
:101290000281FB001C5090004800DD00020070003D
:1012A00000804000005698004800DE00105698006C
:1012B0004C4990000281FB00DC499000C819DD0018
:1012C000028071006C4990000281FB00FC49900093
:1012D000C819DD00828071002FB197000200400024
:1012E000E0804800404E98004801DE00524E9800D1
:1012F000614E98004808DE00704E98000C4990003E
:101300000281FB009C499000C819DD000280710039
:101310002C4990000281FB00BC499000C819DD00F7
:10132000828071001FB1970002004000E0804800F9
:10133000004E98004801DE00124E9800214E9800A1
:101340004808DE00304E98004C4190000281FB00BE
:10135000DC419000C819DD00028071006C419000F2
:101360000281FB00FC419000C819DD008280710001
:101370000FB1970002004000E0804800404698000E
:101380004801DE0052469800614698004808DE0099
:1013900070469800AFE897008180FB002C419000D8
:1013A0000281FB003C4090004800DD00020070001C
:1013B00000804000204698004800DE00304698003B
:1013C0006E044400E0844C008A0F54008B8F5C0054
:1013D00033FF39004F0678004F05BE004F04BE00B2
:1013E0000080FA00000006003200FA00889FBE006C
:1013F0008A9FBE008C1F78000004BE00E00F5100E1
:10140000E08F590008003A000E0078000F077800BE
:101410008E03B10015000900001FEB00005FEB0018
:10142000000778000300370080FC2F000F00400009
:1014300006FF070030002000C0A79F000800BE0084
:10144000A9FE0700E00F5000030032000800BE00B4
:101450000CC70200000000000005EB00CC022000D9
:1014600051FC2F008F8040008105E80010003700FC
:1014700081FC2F008F8040000A804000B04078003F
:10148000C1C79F00B0407800D1C79F00904D780041
:101490002FA19700BFA197000800BE0048C7020017
:1014A0000000000062044400E0844C006305450035
:1014B0008C0F5500EEFF36004F0678004F05BE003A
:1014C0004F04BE000080FA000000060000C02300A8
:1014D00011002000B3FE0700E00F500014003A0096
:1014E0000000240011002000AEFE07006011B800CB
:1014F000E00F50000800320000002400110020001E
:10150000B5FE0700E00F5000E08F580028003A00B9
:10151000020024001300200000C02300110020005E
:10152000B1FF0700E0C12300110020000000060009
:1015300000C0230011002000A7FE0700E00F5000AC
:10154000E08F58001A003A0000002400110020002B
:1015500094FE0700E00F500008003A0002C023008C
:101560001300200000002400110020009EFF07004F
:10157000E00124001100200000000600000024000B
:101580001100200094FE0700E00F5000E08F58008B
:1015900007003A00020024001300200000C02300CE
:1015A0001100200090FF0700E0C12300110020007F
:1015B000000006001A00FA00889FBE008A9FBE0045
:1015C0008C1F78000005EB00F0282000814580008A
:1015D000808F50002E003400BCFF07000004BE00C6
:1015E0000BFE2F008F8545000B00780001FE0700E1
:1015F000D0FD2F000F0040000006E8000E0037006D
:101600008A80450031407800C0DF9F00314078007B
:10161000D0DF9F00114E78006FA99700FFA99700B7
:101620000800BE0048C70200000000006204440039
:10163000E0844C0063054500F40F5500F0FF3600D0
:101640000200240013002000820F5400838F5C00EE
:1016500006003A0002C02300130020000800BE006C
:1016600061FF07001A002000090037001A0020005F
:101670000440240015002000840F5400858F5C0076
:1016800003003A0000C023001100200056FF0700AD
:101690000A0078004F0678004F05BE004F04BE00D8
:1016A0000080FA0000000600303F8200E10F400099
:1016B00002003200617E24008008E800B25D020072
:1016C00000000000E00F500006003D00717F240084
:1016D00011407800E14F40000A0032008048E800E5
:1016E00008003700E8004000627E2400E2C0780075
:1016F000E1CF4000030032008140E8006801410072
:10170000017178008464AB000F00320086EC0200A7
:1017100000000000E00F500006003200403F820051
:10172000E10F400008003200817E24008008E800BC
:1017300000000600503F8200E10F4000020032002E
:10174000A17E24008008E800000006000080FB0065
:10175000C300DE00927F240002814000C308DD0048
:1017600001005000110020000008DD001249700047
:101770000000060061052000810F50000B003900B9
:101780008100E800810F500004003600F080400026
:10179000810F500005003A000200370070C0B3000E
:1017A000EAFF370000C1B300E8FF070000000600B1
:1017B00021062000810F500011003E008180E900C9
:1017C000810F50001D003100F1032000810F5000F7
:1017D00007003E00E6805000810F500015003100E8
:1017E000A002B100E40F50001C003E000F003700C3
:1017F0000005B100E50F500018003E000D00370055
:1018000051062000810F500004003E008100E900D5
:10181000810F50000D0031000A00370061062000E2
:10182000810F50000D003A000A003700F0C0B300ED
:101830000700370080C0B30005003700E0C0B300E8
:101840000300370090C0B3000100370010C1B3009F
:10185000BEFF370000C1B300BCFF07000000060058
:10186000010020007B005000E0805800EF0F500086
:10187000E08F58001F003E00006001000F0037009D
:101880000E0037000D0037000E0037000F00370044
:101890000E0037000D003700080037000D0037003C
:1018A0000E0037000D0037000E0037000D00370026
:1018B0000C0037000F0037000C003700A0C0B30049
:1018C00009003700D0C0B30007003700C0C0B30024
:1018D0000500370020C1B30003003700B0C0B300DB
:1018E0000100370030C1B30098FF370070C1B3006A
:1018F00096FF07000000060042CD800053CD800017
:1019000061004100E080490040CD880051CD880051
:1019100002302A0023002000820F5000838F5800DD
:1019200007003A00A839EF00AA39EF00817F2400B0
:1019300011407800E14F4000010032008048E8008B
:10194000000006000001EB00110221000001200050
:10195000DAED02000000000081012000607E24001A
:10196000E6ED02000000000022EE02000000000090
:10197000F03F8A000000060020C0B30073FF37006C
:10198000A619EC0030CD880001A62E00810F500072
:1019900002003A00A639EF0043FF070000000600EE
:1019A000889FBE008A1F7800607780007177800072
:1019B0008004EB0018002000EAFF2F00910F1000B8
:1019C00033003600740037008800440001004000F6
:1019D0001000550001002000F00F5000E08F58006B
:1019E00022003E0000600100100037000F003700A9
:1019F0000E0037000D0037000C0037000B003700D9
:101A00000C003700190037000C0037000B003700BE
:101A10000C00370015003700100037000B003700AE
:101A20000C0037000F0037000E003700F0C0B30085
:101A30000D00370080C0B3000B003700E0C0B300DA
:101A40000900370000C1B3000700370010C1B30020
:101A50000500370070C0B3000300370040C1B30079
:101A60000100370050C1B30038FF07008800E800CC
:101A700001007800EE0EB40000017800628078006A
:101A8000808F540001003100800478000884E80051
:101A900070778000900F5400CBFF39003A00370078
:101AA0007177800008004400610078004C01DE007E
:101AB00003002000ED0F5100E08F590030003E0080
:101AC000026001000D0037002D00370019003700BB
:101AD0000D0037000F0037001100370013003700EA
:101AE00027003700260037001400370011003700A8
:101AF00016003700200037001A003700890F540005
:101B00001F003900240037000A00600028FF07008A
:101B10001B0037000A00600016FF0700180037009E
:101B20000A00600022FF0700020037000A00600080
:101B300010FF07000884E800140037004400DD00AF
:101B40004480DE0008004000070037000800E8007D
:101B5000000040006100780015FF070063044400A6
:101B60000A0037000A006000808F54000400310032
:101B700080047800020037000A00600038FF070088
:101B80000804E80001003700FAFF200060778000B9
:101B9000800F5400C2FF39004F0578004F04BE008B
:101BA00000000600D17E240011407800E14F400083
:101BB000010032008048E80079FF3700E7FC0700A9
:101BC000E00F500003003A00607E24000C00090082
:101BD0000018EB004027AB000300320010C0B30038
:101BE000DAFE07004027A900807F24008040EB0038
:101BF00090CF100004003A00313F8200005A2000CC
:101C0000808F5000060036006AFE0700E00F50008B
:101C100003003200607E24000C0009000018EB0075
:101C2000C17E240011407800E14F400001003200E5
:101C30008048E800000006001C00FA00889FBE00F3
:101C40008A9FBE008C1F7800000678005C0190001F
:101C5000EC0190000C007800FC4B0200000000003A
:101C600008C0230019002000FA3F24001B002000B8
:101C70000800BE0064C6020000000000E0AF9F0044
:101C8000F1AF9F00A3FD2F008F81410032002000A3
:101C9000C1FD2F008F8040000C0078007A490200BF
:101CA000000000005FA89700E30F500025003A00F5
:101CB00062044400E0844C008A0F54008B8F5C0067
:101CC000EBFF360000FE2F000F00400049FC07002C
:101CD000A3FD2F008F8141005201200001FE2F0043
:101CE0008F8040000C0078007A490200000000005C
:101CF000607E24000C0009000018EB0000C02300E7
:101D00001100200078FC0700E00F500004003200B2
:101D100000C02300110020000CC7020000000000DA
:101D200000002400110020006FFC0700E00F5000AD
:101D30000400320000002400110020000CC7020043
:101D4000000000004F0678004F05BE004F04BE00A3
:101D50000080FA0000000600881F78000004780068
:101D6000611BB8000002EB00F10F5300E08F5B0035
:101D700066003E00066001001100370012003700C7
:101D80001300370014003700150037001600370025
:101D90001C003700320037003300370034003700B2
:101DA00035003700380037003C0037003F0037006F
:101DB0004200370045003700490037004C0037002B
:101DC000020ADD0051003700028ADE004F003700B2
:101DD000010241004D003700028250004B003700E5
:101DE0000192B90049003700E00F510007003200AE
:101DF00000027800110009008200D8000002FD00F6
:101E000042003700E00F51000F003A00C0CB28001D
:101E1000E00F5000040032008200780008007800D3
:101E2000BC8C020000000000230020007304980016
:101E300070014400710029000800780060CE0200A3
:101E40000000000024003700801F78001100090006
:101E50008200D800010278004F0078002B00370084
:101E600001027100290037000102690027003700D4
:101E7000010261002500370014002000828F50000D
:101E800015003A0021003700028168000202EA00D2
:101E9000020172004F12DE001C0037001400200007
:101EA000828F500019003C000B0037001400200006
:101EB000828F500015003D000700370014002000FD
:101EC000828F5000110035000300370014002000FD
:101ED000828F50000D0034000002EB000B00370031
:101EE00014002000E08F500003003200070037008C
:101EF000E08F5000040032000202EA000202720089
:101F00004F22DE0001003700010278000400780053
:101F10004F04780000000600E18F500004003200FA
:101F200005003900E28F500007003A000400370036
:101F3000E00F500005003D000000EA000000060030
:101F40000080EA00000006000000EB000000060030
:101F50008000EB000108980071009800211898009B
:101F60002001900001097800300190000201410039
:101F700040009000FC0604000000000020019000DA
:101F80009201780010002000090037000002400094
:101F900062027A00810F520004003A000000E8005B
:101FA0000000400062007800000006000080E800A9
:101FB000830F5000F5FF3900000005000600FA000D
:101FC000889FBE008A1F780000047800A800900057
:101FD0000808900000014000E10479004C49DE004F
:101FE00003002000EE0F5100E08F5900F1003E0089
:101FF000026001000E0037001100370019003700A1
:10200000220037002D003700380037004B00370022
:10201000750037007E0037008E00370091003700D2
:10202000B7003700C8003700D0003700DA003700AB
:10203000780090000000A10070049800DD003700D7
:10204000E8009000180890000000E800100C9800CC
:1020500000004000C44CDD00C4CCDE0089307800B4
:10206000BE003700E8019000180990000201E80066
:10207000120C9800020141000000E800000040003E
:1020800061007800803179005400370068019000C9
:10209000180890000000E800100C980000004000B4
:1020A000F1FF200081846400C8009000898444000E
:1020B000E1847C0009317800A800370018089000FE
:1020C000F1FF20008184640048019000898444006D
:1020D000E801900080004000E380780001B17C00BE
:1020E0000000E900100C98009C0037000001E80097
:1020F00002014100E101790018099000020141004C
:10210000E80090000281400092007800838F500028
:1021100003003900A0BF9F00B3BF9F001500370028
:10212000F0FF200080846400898040004800900017
:102130008180400060897800280037000001E800B5
:102140000201410061017900680290009808900046
:102150008101E90083814100E481790081804000B0
:10216000E4807800828F500013003900A0BF9F00E8
:10217000B2BF9F00C1BF9F002000200070049800E4
:10218000630020006C81570061002900080078007E
:1021900060CE020000000000C0CB2800E00F50001D
:1021A000840032008000EB0008007800BC8C020044
:1021B000000000007F003700F0FF200080846400F2
:1021C00089804000480090008180400003B0780082
:1021D000180890000080E900100C98000808900092
:1021E0000080E8005F003700180D90000A054500E8
:1021F000680090000A05400089007800F10FB200E5
:102200001A00780044FF0700000D780053003700E3
:10221000E800900018089000000140000000E9006C
:10222000000040008981FB0061017900E100780035
:1022300008007800C8FE0700980890008100E900B7
:10224000110C9800680190008180400000B1780076
:1022500042003700C44CDD00C4CCDE0000804400E6
:1022600040003700E800900018089000000140008E
:102270000000E900000040008981FB006101790055
:10228000E100780008007800B3FE0700980890008D
:102290008180E900110C980088089000E00F500040
:1022A000050032000930B200220020000330200077
:1022B000838F540006003A00A80190000101E80055
:1022C0000201410063017900E00F50000500320077
:1022D0008180400028009000810040001190A00003
:1022E0000300370081804000818041001190A100EF
:1022F0000808900002014000020C98002D003700F1
:102300000081E80002014100E10179000000E800DD
:102310000000400061017800020141004800900087
:1023200002014000F1FF20008180640083814100B0
:102330000800780060CE020000000000080890004D
:102340006300400007003700F1FF20008180640037
:102350000800780002B002000000000008089000A9
:102360000000E800000C980012003700680190009F
:10237000980890008100E800110C980081804000CE
:10238000810041008008E800F0FF200080846400A4
:10239000090C9800070037001808900068019000A9
:1023A00080004000E2807800010C98000000E90005
:1023B000100C98004F0578004F04BE000080FA0012
:1023C000000006000000FA00889FBE008A9FBE0041
:1023D0008C9FBE0080047800810578000F0678008D
:1023E0000B0078000C0702000000000000047800D9
:1023F000E3064400650044000000A1008087470018
:102400000C057800C0CB2800E00F5000040032001B
:102410008B00780009007800BC8C020000000000EE
:1024200020002000F004980009089000000D7800BA
:102430002845980063004500080178008B0078006B
:10244000EC060200000000008D0178000A0178000F
:10245000910029000900780060CE02000000000011
:102460008C0778004F06BE004F05BE004F04BE002B
:102470000080FA00000006008000EB000B0037002F
:102480006A814000020141006001790080099000EA
:10249000830F510004003A00F00090000110A000EA
:1024A00071009800100005008100E80020199000DC
:1024B000828F5000F2FF390000000500889FBE00A7
:1024C0000004BE00780090000020A0007004980076
:1024D000E08F54000D003200030037000800780040
:1024E000B6FE07008904E9007800900065006000EE
:1024F000E50F500009003A00E08F5400F7FF3A0062
:102500000600370008007800ACFE07007800900055
:1025100065006000E50F5000FAFF3200780090007F
:102520000020A100700498004F04BE0000000600C7
:10253000A01990000041EB00EF8F510006003E0013
:102540006A81410002014100013079008301E80005
:102550002318980012C0B300024078000000060063
:10256000010178008000EB00120037006A82400011
:102570000402420060027A00820F52000C003A000E
:102580000301E9002218980006003700EA814000A4
:1025900003824100EB814000838141006332780077
:1025A0008100E800828F5000F8FF3900100005001C
:1025B0008100E800A0199000838F5000EBFF3900E4
:1025C000000005008000EB002118980000000600C4
:1025D0000400FA0080089000E1BF9F00F000900026
:1025E000F1BF9F004300200064815700A100290033
:1025F00060CE0200000000000080FA00000006002B
:10260000889FBE000004BE00780090000020A0005B
:1026100070049800E08F54001B0032000700370060
:102620000800780094FF0700E00F50000E003A0009
:102630000800780061FE07008904E9007800900036
:1026400065006000E50F500013003A00E08F540071
:10265000F3FF3A00100037000800780086FF0700FB
:10266000E00F500006003200780090000010A0003B
:102670007004980008007800D5FF070009003700B3
:10268000080078004DFE07007800900065006000AB
:10269000E50F5000F0FF3200780090000020A1000C
:1026A000700498004F04BE0000000600F001900086
:1026B000618161000B003200E28161000001EB00EA
:1026C000828F510007003A0020199000E00F51005E
:1026D00002003200CAFF07000100370077FF070041
:1026E000120020000200780000000600889FBE0053
:1026F000000478000800780020FE070080047800BD
:10270000E08F5400130032007800900061006000F8
:1027100006003200700144002300200081002900DF
:102720000800780060CE020000000000090C98004C
:102730000080EB00100C9800F80090000100A00051
:1027400071049800E2806000020032000800780006
:102750009FFF0700090078004F04BE00000006003C
:102760000400FA00881F78000004780000002A00A6
:10277000808F500004003A0008007800DACE020092
:10278000000000007E00370012007800980F500013
:102790007B003A000280E8000302E900F2FF250016
:1027A000F3FF2F0001014100E0814900EE0F5100CD
:1027B000E08F590072003E00026001000E003700F9
:1027C0001A003700210037002C0037003100370095
:1027D000360037002C003700360037004200370043
:1027E00045003700470037004C00370059003700DC
:1027F0005C0037005F003700900178000402E900B8
:102800008000EB0007003700038140000201410017
:10281000280390008100E80081824000E0827A0075
:1028200005337900848F5000F7FF39002000200025
:10283000700498008080EB0008007800ABFF070070
:10284000E00F50004E003A000F0037007800900073
:102850000010A10070049800080078005CFF0700D9
:1028600020DD2800E00F500045003200080078000D
:10287000D28D020000000000410037007800900077
:102880000010A000700498000800780050FF0700B6
:102890003B00370078009000610060003800320093
:1028A00008007800C5FD0700F7FF37002000200072
:1028B000F4FF370090007800D1BF9F000800780037
:1028C0001BFF07000080FB00E0BF9F0043002000CB
:1028D00066815700B10029000800780060CE020030
:1028E0000000000026003700900078000800780003
:1028F0001BFF0700220037000800780031FF0700A7
:102900001F00370010019000900078000800780048
:102910008ECE020000000000190037009001780000
:102920000402E9008000EB0007003700038140004B
:1029300002014100480390008100E80081824000CC
:10294000E0827A0005337900848F5000F7FF390068
:102950000B0037000800780012B0020000000000F1
:102960000700370008007800D6AF02000000000022
:102970000300370008007800F6AF020000000000F6
:102980004F0478000080FA000000060092007800F2
:10299000E08F50000600350078FD0700130020008E
:1029A000E00F50000F0032008001EB000D003700F7
:1029B00013002000F4FF2900848F50000900360026
:1029C000120190008001EB000402E800848F5000A7
:1029D00004003200900169000300EA0083017000E6
:1029E000CF19DE000300780000000600889FBE00BB
:1029F0000004EB00890E2000803E20008EEE0200D5
:102A0000000000000804E800890F5400FAFF3600B7
:102A10004F04BE000000060001C2B30080C0B30036
:102A200090BA020000000000F0FF07008040EB00B9
:102A300080C0B30090BA02000000000001C2B300E1
:102A400090C0B30090BA020000000000E7FF07004A
:102A50008040EB0090C0B30090BA0200000000007C
:102A600001C2B300A0C0B30090BA02000000000091
:102A7000DEFF07008040EB00A0C0B30090BA020068
:102A80000000000001C2B300B0C0B30090BA020061
:102A900000000000D5FF07008040EB00B0C0B3008D
:102AA00090BA02000000000001C2B300C0C0B30031
:102AB00090BA020000000000CCFF07008040EB004D
:102AC000C0C0B30090BA02000000000001C2B30011
:102AD000D0C0B30090BA020000000000C3FF07009E
:102AE0008040EB00D0C0B30090BA020000000000AC
:102AF00001C2B30020C0B30090BA02000000000081
:102B0000BAFF07008040EB0020C0B30090BA02007B
:102B10000000000001C2B30030C0B30090BA020050
:102B200000000000B1FF07008040EB0030C0B300A0
:102B300090BA02000000000001C2B30040C0B30020
:102B400090BA020000000000A8FF07008040EB00E0
:102B500040C0B30090BA04000000000001C2B300FE
:102B600020C2B30090BA0200000000009FFF0700DF
:102B70008040EB0020C2B30090BA020000000000C9
:102B800001C2B3000140780090BA020000000000CA
:102B900096FF07008040EB0000C2B30090BA02002D
:102BA0000000000001C2B30030C2B30090BA0200BE
:102BB000000000008DFF07008040EB0030C2B30032
:102BC00090BA02000000000001C2B30010C2B300BE
:102BD00090BA02000000000084FF07008040EB0074
:102BE00010C2B30090BA04000000000001C2B3009C
:102BF000C0C1B30090BA0200000000007BFF0700D4
:102C00008040EB00C0C1B30090BA02000000000099
:102C100001C2B30040C2B30090BA0200000000003D
:102C200072FF07008040EB0040C2B30090BA020080
:102C30000000000001C2B30050C2B30090BA02000D
:102C40000000000069FF07008040EB0050C2B300A5
:102C500090BA02000000000001C2B300F0C1B3004E
:102C600090BA02000000000060FF07008040EB0007
:102C7000F0C1B30090BA02000000000001C2B3002E
:102C800080C1B30090BA02000000000057FF0700A7
:102C90008040EB0080C1B30090BA02000000000049
:102CA00001C2B30090C1B30090BA0200000000005E
:102CB0004EFF07008040EB0090C1B30090BA0200C5
:102CC0000000000001C2B300A0C1B30090BA02002E
:102CD0000000000045FF07008040EB00A0C1B300EA
:102CE00090BA02000000000001C2B300B0C1B300FE
:102CF00090BA0200000000003CFF07008040EB009B
:102D0000B0C1B30090BA04000000000001C2B300DB
:102D100000C1B30090BA02000000000033FF0700BA
:102D20008040EB0000C1B30090BA02000000000038
:102D300001C2B30010C1B30090BA0200000000004D
:102D40002AFF07008040EB0010C1B30090BA0200D8
:102D50000000000001C2B30040C1B30090BA0200FD
:102D60000000000021FF07008040EB0040C1B300DD
:102D700090BA02000000000001C2B30050C1B300CD
:102D800090BA02000000000018FF07008040EB002E
:102D900050C1B30090BA02000000000001C2B300AD
:102DA00020C1B30090BA0200000000000FFF07002E
:102DB0008040EB0020C1B30090BA02000000000088
:102DC00001C2B30030C1B30090BA0200000000009D
:102DD00006FF07008040EB0030C1B30090BA04004A
:102DE000000000008040EB0050C0B30090BA020029
:102DF00000000000C5FF070001C2B300D0C1B3004E
:102E000090BA020000000000F8FE07008040EB00CE
:102E1000D0C1B30090BA02000000000001C2B300AC
:102E2000E0C1B30090BA020000000000EFFE07000E
:102E30008040EB00E0C1B30090BA02000000000047
:102E400001C2B30050C0B30090BA020000000000FD
:102E5000E6FE07008040EB0050C0B30090BA0200CD
:102E60000000000001C2B30060C0B30090BA0200CD
:102E700000000000DDFE07008040EB0060C0B300F2
:102E800090BA02000000000001C2B30070C0B3009D
:102E900090BA020000000000D4FE07008040EB0062
:102EA00070C0B30090BA0200000000004FFF07009E
:102EB0002AFF070001C2B30060C2B30090BA02004B
:102EC00000000000C9FE07008040EB0060C2B300B4
:102ED00090BA02000000000001C2B30070C2B3004B
:102EE00090BA020000000000C0FE07008040EB0026
:102EF00070C2B30090BA02000000000001C2B3002B
:102F00000040EB0090BA020000000000B7FE07008E
:102F10008040EB000140780090BA02000000000001
:102F200001C2B300E0C0B30090BA0200000000008C
:102F3000AEFE07008040EB00E0C0B30090BA020094
:102F40000000000001C2B30010C0B30090BA02003C
:102F500000000000A5FE07008040EB0010C0B30099
:102F600090BA02000000000001C2B30060C1B300CB
:102F700090BA0200000000009CFE07008040EB00B9
:102F800060C1B30090BA02000000000001C2B300AB
:102F900070C1B30090BA02000000000093FE070069
:102FA0008040EB0070C1B30090BA02000000000046
:102FB00099FE37008BFF070001C2B30020C0B300A9
:102FC00090BA02000000000001C2B30000C1B300CB
:102FD00090BA02000000000001C2B30010C1B300AB
:102FE00090BA02000000000001C2B30040C1B3006B
:102FF00090BA02000000000001C2B30020C1B3007B
:1030000090BA02000000000001C2B30030C1B3005A
:1030100090BA02000000000001C2B3000040EB00C3
:1030200090BA02000000000001C2B30010C0B3005B
:1030300090BA02000000000001C2B300E0C1B3007A
:1030400090BA02000000000001C2B30070C2B300D9
:1030500090BA02000000000001C2B30080C1B300BA
:1030600090BA02000000000001C2B30090C1B3009A
:1030700090BA02000000000001C2B300A0C1B3007A
:1030800090BA02000000000001C2B300B0C1B3005A
:1030900090BA02000000000001C2B300C0C1B3003A
:1030A00090BA02000000000001C2B30040C2B300A9
:1030B00090BA02000000000001C2B30050C2B30089
:1030C00090BA02000000000001C2B300F0C1B300DA
:1030D00090BA02000000000001C2B300D0C1B300EA
:1030E00090BA02000000000001C2B30060C1B3004A
:1030F00090BA02000000000001C2B30070C1B3002A
:1031000090BA02000000000001C2B30080C0B3000A
:1031100090BA02000000000001C2B300D0C0B300AA
:1031200090BA02000000000001C2B300E0C0B3008A
:1031300090BA02000000000000802000FE63020040
:1031400000000000100020007ADE040000000000F3
:1031500031468000910CB100A0122000808F5000F9
:1031600005003E00AC19A8008040EB006340500011
:1031700090BA02000000000080458000B208B40050
:10318000813E20000180B900A2F82000811F780054
:10319000110009004288D800CF007800C018B100A3
:1031A00011022000810F500005003E008040EB001E
:1031B000D0C0B30090BA020000000000AC39A800F3
:1031C000914380005138B100A0C12000808F500091
:1031D00005003E008040EB0000C1B30090BA020041
:1031E00000000000AC59A800A14380005138B10094
:1031F000A0C12000808F500005003E008040EB0001
:1032000010C1B30090BA020000000000AC79A80021
:10321000B14380005138B100A0C12000808F500020
:1032200005003E008040EB0040C1B30090BA0200B0
:1032300000000000AC99A800C14380005138B100E3
:10324000A0C12000808F500005003E008040EB00B0
:1032500020C1B30090BA020000000000ACB9A80081
:10326000D14380005138B100A0C12000808F5000B0
:1032700005003E008040EB0030C1B30090BA020070
:1032800000000000ACD9A800E14380005138B10033
:10329000A0C12000808F500005003E008040EB0060
:1032A0000140780090BA020000000000ACF9A800CC
:1032B000F14380005138B100A0C12000808F500040
:1032C00005003E008040EB0010C0B30090BA020041
:1032D00000000000AD19A800414580005106B10072
:1032E000E0312000808F500005003E008040EB0060
:1032F00060C1B30090BA020000000000AD39A80020
:10330000514580005106B100E0312000808F50000F
:1033100005003E008040EB0070C1B30090BA02008F
:1033200000000000AD59A80050468000E00F50009A
:1033300003003A0040468000E00F500005003200D4
:103340008040EB00D0C1B30090BA02000000000042
:10335000AD79A8008002200061468000808F500077
:103360000C00340080468000810C2000810F50004A
:1033700008003400B1122000810F500005003C000D
:10338000AD99A8008040EB00E0C1B30090BA020004
:1033900000000000ADB9A8008040EB00C0C1B30040
:1033A00090BA020000000000ADD9A8008040EB00F8
:1033B00050C2B30090BA020000000000C04280007A
:1033C000E00F5000110032008040EB0090C1B300CC
:1033D00090BA0200000000008040EB00B0C1B300D2
:1033E00090BA0200000000008040EB0040C2B30031
:1033F00090BA0200000000008040EB00F0C1B30072
:1034000090BA020000000000ADF9A800D042800090
:10341000E00F5000050032008040EB0080C1B30097
:1034200090BA020000000000AE19A800E04280003F
:10343000E00F5000050032008040EB00A0C1B30057
:1034400090BA020000000000AE39A80078EC02003B
:1034500000000000E00F5000050032008040EB004B
:10346000E0C0B30090BA020000000000AE59A8000E
:10347000C008EC00E20F50000B003E00C208EC0058
:10348000E20F500008003E0020468000F40F50007C
:10349000050034008040EB0080C0B30090BA020009
:1034A00000000000AE79A800F0FF2F00F10020001E
:1034B00062CD800073CD8000800F5100818F590054
:1034C00008003A008040EB0020C0B30090BA020030
:1034D0000000000001C2B30030C0B30090BA020087
:1034E00000000000B019EC0080CD8800710C2000B5
:1034F000810F500002003E008100E8006145880015
:1035000072F32F0000014100610C2000810F510077
:1035100002003E0081F32F0061458800F2E62F0093
:1035200000014100610C2000810F510003003E00AA
:10353000AC28EF008180E8007145880072DA2F0026
:1035400000014100610C2000810F510002003E008B
:1035500081F32F0071458800F2CD2F00000141005A
:10356000E1182000810F510002003E00AE28EF005C
:1035700000000600014B2000810F500001003A00BE
:10358000B039EF000000060090089000E0019000C4
:1035900001814000630179008100E9001108980071
:1035A00002007800000006000002EB000271220019
:1035B000A5002000811F7800110009000280D800BA
:1035C0008001780001007800CF007800E08F510082
:1035D00004003A00E00F520002003A00E10F5100EF
:1035E00003003A0004C3B30084D841001400200053
:1035F000809FBE00110009000581D80000017800FD
:103600004F00BE00E00F5100EAFF3A0001007800D1
:1036100000000600E4FF0700E1C2B30001487800A3
:1036200071C7B30001687800F6C0500001687800E7
:10363000F5C04000016878008040EB001140980020
:1036400000000600889FBE008A1F780000047800F2
:10365000C804900008007800CBFF0700000040007D
:10366000E90478004805900008007800C6FF0700CC
:1036700000004000EA007800EF8F5400080032009C
:10368000E08F54000600350070022000808F540047
:1036900003003C000940780090BA020000000000DE
:1036A0004F0578004F04BE00000006000E00FA002F
:1036B000881F78008E0078000F0778000E01B10097
:1036C00005000900001FEB00005FEB000107780018
:1036D00001C7B30081F79F0040049000AAFF0700D4
:1036E000000040006804780010002000166402000A
:1036F000000000009EDC0200000000000000EB0063
:10370000E10F440004003200EF8057000800780009
:10371000C0FF07007080570038DD02000000000085
:103720004F0478000080FA00000006000E00FA0046
:10373000881F78008E0078000F0778000E01B10016
:1037400005000900001FEB00005FEB000107780097
:1037500021C7B30081F79F00400490008AFF070053
:103760000000400068047800E10F440003003A00C4
:1037700074AC0200000000000900370010002000B7
:103780001664020000000000EF8057000800780077
:10379000A0FF07007080570014AC0200000000007A
:1037A0004F0478000080FA00000006000E00FA00C6
:1037B000881F78008E0078000F0778000E01B10096
:1037C00005000900001FEB00005FEB000107780017
:1037D00021C7B30081F79F00400490006AFF0700F3
:1037E0000000400068047800100020001664020009
:1037F000000000009EDC0200000000000000EB0062
:10380000E10F440004003200EF8057000800780008
:1038100080FF07007080570038DD020000000000C4
:103820004F0478000080FA00000006000E00FA0045
:10383000881F78008E0078000F0778000E01B10015
:1038400005000900001FEB00005FEB000107780096
:1038500031C7B30081F79F00400490004AFF070082
:103860000000400068047800100020001664020088
:10387000000000009EDC020000000000080078004C
:1038800052DD02000000000080007800E08F500050
:1038900006003200EF805700080078005DFF070047
:1038A0007080570038DD0200000000004F047800EF
:1038B0000080FA0000000600E6874700889FBE00EF
:1038C0008A9FBE008C9FBE008E1F78000004780087
:1038D000C8049000080078002BFF0700000040009B
:1038E000E9047800480590000800780026FF0700EA
:1038F000000040006A057800C805900008007800C4
:1039000021FF070000004000EB057800480690000A
:10391000080078001CFF0700000040006C067800DB
:10392000C80690000800780017FF0700000040005C
:10393000ED067800480790000800780012FF0700A5
:10394000000040006E077800C80090000800780072
:10395000F1B79F000CFF070000004000FFB0970088
:1039600061037800C800900008007800F1B79F005C
:1039700086BF9F0004FF070000004000FFB09700D3
:1039800061047800001020001664020000000000AE
:10399000884378000FBB97008E4278000D42780074
:1039A0008C4178000B4178008A407800094078000B
:1039B00084BB0200000000004F0778004F06BE00E5
:1039C0004F05BE004F04BE006F00B10000000600AE
:1039D000889FBE008A9FBE0000047800C804900043
:1039E00008007800E8FE070000004000E9047800C5
:1039F0004805900008007800E3FE07000000400042
:103A00006A057800C805900008007800DEFE07000F
:103A1000000040006B0178008A407800094078007F
:103A2000D4BB0200000000004F05BE004F04BE00E2
:103A300000000600889FBE008A9FBE000004780038
:103A4000C804900008007800CFFE07000000400086
:103A5000E90478004805900008007800CAFE0700D5
:103A6000000040006A057800C80590000800780052
:103A7000C5FE0700000040006B0178008A40780016
:103A800009407800F0BB0200000000004F05BE00B6
:103A90004F04BE0000000600889FBE008A9FBE0043
:103AA00000047800C804900008007800B6FE070003
:103AB00000004000E9047800480590000800780004
:103AC000B1FE0700000040006A057800C8059000BC
:103AD00008007800ACFE0700000040006B01780091
:103AE0008A407800094078000CBC02000000000009
:103AF0004F05BE004F04BE0000000600889FBE00B8
:103B00008A9FBE008C1F780000047800C8049000D3
:103B1000080078009CFE070000004000E9057800DE
:103B2000C80490000800780097FE070000004000DD
:103B300069057800C80490000800780092FE07002C
:103B400000004000E9047800480690000800780072
:103B50008DFE0700000040006C047800200020006B
:103B600016640200000000008B40780000C2B30021
:103B700090BA0200000000008A40780030C2B30012
:103B800090BA0200000000008940780010C2B30023
:103B900090BA0200000000008840780020C2B30004
:103BA00090BA0200000000004F0678004F05BE00EA
:103BB0004F04BE0000000600E6874700889FBE0055
:103BC0008A9FBE008C9FBE008E1F78000004780084
:103BD000C8049000080078006BFE07000000400059
:103BE000E9047800480590000800780066FE0700A8
:103BF000000040006A057800C805900008007800C1
:103C000061FE070000004000EB05780048069000C8
:103C1000080078005CFE0700000040006C06780099
:103C2000C80690000800780057FE0700000040001A
:103C3000ED067800480790000800780052FE070063
:103C4000000040006E077800C8009000080078006F
:103C5000F1B79F004CFE070000004000FFB0970046
:103C600061037800C800900008007800F1B79F0059
:103C700086BF9F0044FE070000004000FFB0970091
:103C8000610478004000200016640200000000007B
:103C9000884378000FBB97008E4278000D42780071
:103CA0008C4178000B4178008A4078000940780008
:103CB00028BC0200000000004F0778004F06BE003D
:103CC0004F05BE004F04BE006F00B10000000600AB
:103CD000889FBE008A1F780000047800C804900006
:103CE0000800780028FE070000004000E904780082
:103CF000480590000800780023FE070000004000FF
:103D00006A047800400020001664020000000000F1
:103D10008940780060C1B30090BA02000000000042
:103D20008840780070C1B30090BA02000000000023
:103D30004F0578004F04BE0000000600881F780081
:103D40004004900010FE0700000040006804780066
:103D50000004200016640200000000008840780083
:103D6000D0C1B30090BA0200000000004F047800F8
:103D700000000600881F78004004900002FE070043
:103D80000000400068047800000120001664020072
:103D90000000000088407800E0C1B30090BA020043
:103DA000000000004F04780000000600889FBE005D
:103DB0008A1F780000047800C8049000080078008A
:103DC000F1FD070000004000E9047800480590007C
:103DD00008007800ECFD0700000040006A0478004D
:103DE00000202000166402000000000089407800D6
:103DF00060C2B30090BA0200000000008840780062
:103E000070C2B30090BA0200000000004F057800B5
:103E10004F04BE0000000600889FBE008A1F780085
:103E200000047800C804900008007800D6FD070060
:103E300000004000E9047800480590000800780080
:103E4000D1FD0700000040006A0478001000200047
:103E500016640200000000009EDC0200000000006A
:103E6000880078000900780074DD0200000000007E
:103E70004F0578004F04BE0000000600889FBE007A
:103E800000047800C804900008007800BEFD070018
:103E900000004000008044008000EB00F30F200091
:103EA000D2082000018240000402400005082000E2
:103EB00014824200830F520005003600217F290042
:103EC00008007800E29102000000000005003700C1
:103ED0008100E800828F5000F2FF34005CEC0200A9
:103EE000000000004F04BE0000000600881F78009C
:103EF00040049000A4FD0700000040006800780026
:103F0000E00F50000300320090AA02000000000001
:103F1000020037009AAA0200000000004F04780057
:103F2000000006000E00FA00889FBE008A1F78007D
:103F300000047800C80490000800780092FD070093
:103F40000000400069057800080078008EFD070039
:103F5000800478000E0078000F0778004E01B10051
:103F600005000900001FEB00005FEB000007780070
:103F700051C7B300C1EF9F00E10F450008003A00B0
:103F80000000EB006AAD0200000000004800900055
:103F90008984440089044000800CEB001400370041
:103FA000F38057000A0078007FFD0700E1C2B300EC
:103FB0000148780041C6B30001687800E3C05000B2
:103FC00001687800F3C04000016878008040EB0091
:103FD0001140980089844400480090008904400002
:103FE000748057006AAD020000000000800C780069
:103FF0004F0578004F04BE000080FA000000060064
:10400000889FBE008A9FBE0000047800C80590000B
:10401000080078005CFD0700800478000800780044
:1040200059FD0700000578000800780056FD0700DC
:10403000800078000A054500480090000A0540000D
:1040400081804000898444000980450040AE020020
:1040500000000000000DD1004F05BE004F04BE005F
:1040600000000600889FBE008A9FBE000004780002
:10407000C80590000800780043FD07008004780020
:104080000800780040FD070000057800080078006F
:104090003DFD0700800078000A05450048009000BB
:1040A0000A05400081804000898444000980450061
:1040B000F8AD020000000000000DD1004F05BE0069
:1040C0004F04BE0000000600889FBE000004780078
:1040D000C8049000080078002BFD07000000400095
:1040E000E90478000800780027FD070080007800C8
:1040F0008180400048049000010444006148B900F8
:104100000000400081804800B8AD020000000000BF
:10411000000C78004F04BE00000006000080FB0089
:10412000401388006002AB00FEFF320040138000A5
:1041300000000600401F2000A0CD880000C0EB005A
:10414000F6FF070000C0EB00F4FF0700E14F40005E
:1041500003003200A1CD8000E08F5000F9FF3A004B
:1041600000000600CDC2A80000C0EB00EBFF370046
:10417000CDC2A900EFFF070011002000E14F400071
:1041800002003200F7FF07008000EB00010078001A
:1041900000000600CDC2A800C9C2A900B0132000CB
:1041A000101388006422EF0061E2A80000000600FE
:1041B000EFFF0700EBFF0700C9C2A80061E2A900FA
:1041C000D019A80000000600889FBE008004780077
:1041D000010478004006200090CD880000C0EB006C
:1041E000CEFF070080417800E1CF410004003A0093
:1041F00092CD8000E00F5100F8FF3A002200370016
:104200000001EB00E2CF41001F003A00F20F200056
:10421000421388006002AB00FEFF320041138000B1
:104220000900780001587800421388006002AB0052
:10423000FEFF3200411380000158780042138800CD
:104240006002AB00FEFF320041138000015878008D
:10425000421388006002AB00FEFF32004113800071
:104260000148780064045400020032008004E80031
:10427000E7FF370000C0EB00A8FF070000C0EB001D
:10428000A6FF070012002000020078004F04BE00C5
:1042900000000600889FBE008A1F78008004780016
:1042A00001447800A3FF07000001EB00E14F40004C
:1042B00019003A000840780098FF0700120020001B
:1042C000E34F440014003200082020000905E800F4
:1042D0001940780091FF07008984E8001A407800AF
:1042E0008EFF07000884E900F8FF3A0000C0EB00E9
:1042F0008AFF070000C0EB0088FF070000C0EB004A
:1043000086FF07007F00600012002000E50F5000CC
:104310000100320008017800020078004F057800A3
:104320004F04BE0000000600889FBE008A1F780070
:10433000004578000204BE00E04F550006003D0035
:104340006011B80070C3B300F7FF0700E14F5000E1
:104350002A003E000A74A10082FF070084FF0700C4
:104360008000780000C0EB00E08F50002300320096
:104370000A4078000064A00068FF07004848DE009B
:104380000100200065FF07004048DE00010020001A
:1043900062FF07004849DD004840DE000000710070
:1043A000C848DE005DFF0700084078005BFF07009B
:1043B00050C9B300E04F5500040032006E40500079
:1043C000E84F55000100320010C0B30053FF070052
:1043D000EC4F550002003A0000C0EB004FFF070011
:1043E000A8C0B30000C0EB004CFF0700E04F500036
:1043F00002003D000844E900FAFF3A004F0578004A
:104400004F04BE00000006000400FA00889FBE00B2
:104410008A1F78008040780010C0B300E0CF5000C1
:1044200088003A00511680000000240000806000DF
:104430008300320057FF070061E2A90011138000DA
:1044400030FE2F00008060004001B3001013880090
:1044500011138000C0FF2F00008060000000A0004A
:104460001013880061E2A800A9C0B30000C0EB00EF
:104470002AFF07008944E900FCFF3A006011B800F8
:1044800009407800A8FF070000457800094478003B
:10449000E14F550059003A00803E200090CD880041
:1044A000A21A20000300200080C0B3009EFF070076
:1044B000E14F500033003A0000C0EB0017FF070047
:1044C0008880FB00804178006A81570003F1780002
:1044D0000844E800E34F5400F7FF36000044EB00C7
:1044E0000FF89700E14F500044003A00A0CAB30013
:1044F0009FF8970080CF500040003A0090CD800098
:10450000E00F5000060032000200200003002400EB
:1045100090CAB30084FF0700E04F5000F7FF3A0055
:1045200098CD8000E00F5400340032006011B800D4
:10453000A0C3B3007CFF07000044EB00884F50008D
:104540002E003A0000C0EB00F4FE07008980FB005B
:10455000804178006A81570003F178008944E800BF
:10456000E3CF5400F7FF3600EFF097000180FB0027
:104570000004B20048C0B30020003200C8C0B3003D
:104580001E0037006011B80090CAB30066FF070034
:1045900028C0B30099CAB300E14F500002003600B2
:1045A0000A4478008844780090CD8000E00F5000E5
:1045B000050032006011B800094078005AFF07007A
:1045C000E04F5000F8FF3A0090CD8000E00F50001F
:1045D00007003200022020000300200000C1B300C9
:1045E00051FF0700E04F500003003A00030037007E
:1045F00000447800010037000044EB000880FB0015
:10460000B0CD8800D7FE0700E04F54000B00320009
:10461000D019A90061E2A9001113800030FE2F001B
:10462000008060008001B30010138800300020007B
:104630006222B70061E2A80001003700DCFE07003B
:10464000D0D9BF004F0578004F04BE000080FA00AB
:10465000000006008040780010C0B300E0CF50009A
:1046600001003A00D0D9BF0000000600889FBE00BC
:104670008A1F7800810478000444780044002000F8
:10468000E04F50002F003A00E04F54002D00320060
:10469000D0D9BF00610060003400200029003A003A
:1046A000B679AB0004003A004918DD00C711DE00FE
:1046B000830170004911DD00E14F54000B003A0006
:1046C00010C1B30018FF070000457800E04F550007
:1046D00018003A000120200009007800BAFE070007
:1046E000E00F500012003A001200370020C1B30062
:1046F0000DFF0700E04F50000E003A00012020009F
:1047000009007800B0FE0700E00F500004003200FE
:104710000844E900020032000920B000F7FF37002A
:104720006011B800C0C0B300FFFE070001003700F1
:104730000A4478008BFE07000882FB000402EA00AE
:104740004F22DE00040078004F0578004F04BE00C1
:1047500000000600889FBE008A9FBE008105780089
:104760000204BE000445780042002000E04F5000E3
:1047700040003A00E04F55003E003200D0D9BF0063
:1047800061006000320020003A003A00D0D9BF003A
:10479000640060002200200036003A00B0CD8000A6
:1047A000E800600004003A00C948DD00C744DE00AC
:1047B000898470004944DD00E14F55000C003A0047
:1047C0000801BE0080C1B300D7FE07000044780096
:1047D000E04F540023003A00E1CFB3000B00780013
:1047E000ACFE0700E00F50001B003A001D00370030
:1047F00066006000040032000A81FB000300200014
:1048000070C9B300C8FE07000801BE0090C1B30024
:10481000C5FE0700E04F500012003A00C1CFB300C0
:104820000B0078009BFE0700E00F500004003200F0
:104830000A45E900020032000B20B000F7FF370004
:10484000D1CFB3000000EB0092FE0700E00F500054
:1048500003003200030037000845780001003700EC
:104860001AC0B3003FFE07000A81FB000201EA0004
:104870004F11DE00020078004F05BE004F04BE005D
:10488000000006001000FA00889FBE008A9FBE004C
:1048900080417800014078008204780048002000C0
:1048A000E0CF5100D4003A00019D210091407800F2
:1048B000E180600038002000CF003A000080FB005B
:1048C00001002000EE0F5000E08F5800C8003E00AD
:1048D000006001000E003700130037004800370069
:1048E0004A003700C2003700C1003700C00037005F
:1048F000BF003700BE003700BD0037008E00370014
:1049000091003700930037009A003700A800370065
:1049100017FE070018002000E00F5000B50032001D
:1049200010FE0700860037006011B80090C0B30089
:104930007DFE070018002000E04F5000AD003A0057
:1049400001012000788057001FFE0700E00F500093
:10495000A80032000FE897008080FB00C608DE0048
:104960000FF09700E1CF50000B003A001FF19700C5
:104970000281FB00080141004800DD000001410008
:10498000030020004A18DD00C610DE008100700020
:104990004A10DD003C0037000080FB004600DE00CE
:1049A000FFE897008180FB00C208DD0001004000A5
:1049B0000000E800EFE89700E3806000CA08DD002F
:1049C00001004000010020005FEA97006F42620092
:1049D000AFF197008381FB00C719DE0083414200DD
:1049E00083C1E8001FF1970063416100024141006B
:1049F00002C141000281FB00690151001D00370026
:104A000000202000800C78004D003700BBCD8000D6
:104A1000648565001E0032006011B800D0C8B30084
:104A200041FE070018002000E04F500071003A00DE
:104A300000C0EB00B9FD070001012000788057009D
:104A4000E1FD0700E00F50006A00320008C3B30028
:104A500000C0EB00B1FD07000844E900FCFF3A008C
:104A60002FF197000281FB004411DE0000012000BD
:104A7000010020000201E9000300330000004000B3
:104A800081804800FBFF3700808CBE002C0037007F
:104A90006011B80090C0B30023FE0700180020008A
:104AA000E04F500053003A00010120007880570089
:104AB000C5FD0700E00F50004E0032006284650023
:104AC0002FF19700BFF097000F0032000180FB002C
:104AD0004700DE000000E800F203B20002014100DE
:104AE00002004000DFF197008381FB00C619DE0061
:104AF0008301E9000300DD0001002000808CBE007E
:104B00000A0478003B0037008180FB004508DE0086
:104B10000000E800E3806000C308DD000100400001
:104B2000C207B2004291DE000201E8000280B90033
:104B3000808CBE002F003700689B2100984C7800C5
:104B40000004EB002B0037006011B80090C0B300E8
:104B5000020037006011B800A0C0B300F2FD0700EA
:104B60001800200001012000E04F500021003A0011
:104B7000180037006011B800A0C3B300EAFD0700B9
:104B800018002000E04F50001A003A00004478005E
:104B900000C0EB0061FD07008880FB0080F4780016
:104BA0000844E800E34F5400F9FF3600E4FF370003
:104BB0006011B800D0C8B300DBFD0700180020006A
